:100000000C9446000C946DE80C94E5E80C945DE9C2
:10001000189500001895000018950000189500002C
:1000200018950000189500000C945CEC18950000E1
:1000300018950000189500000C94E3F51895000041
:100040000C9401F418950000189500001895000014
:1000500018950000189500001895000018950000EC
:1000600018950000189500001895000018950000DC
:1000700018950000189500001895000018950000CC
:100080001895000018950000189500008FEF8DBF9F
:10009000C0EEECE34E2E80E18EBFDDE0FBE05F2E94
:1000A000EEEFFFE0A0E0B1E088278D933197E9F70C
:1000B00087E689B980E08093900088E18AB9662458
:1000C0008FE181BD87E181BD81B5886081BD80916F
:1000D000010180688093010185E085BD87B7806458
:1000E00087BF789489B7816089BF89B7826089BFEB
:1000F00089B7846089BF80916A008C7F8360809318
:100100006A0080916A00837F8C6080936A0080918E
:100110006A008F7C806380936A0088E080BF85E0FE
:1001200083BF87B7816087BF80EC8ABB80EB87BBCA
:100130008FEF84BB80E081BB84E082B980E0809354
:100140006400E2E7FFE0A8E5B6E094E00E948DF5E8
:10015000E7E7FFE0ADE5B6E091E00E948DF5E9E369
:10016000F0E0A5E7B6E00E9485F51B9A1C9A1D9A5F
:100170001E9A1F9A909ADA9ADB9ADC9ADD9ADE9A96
:10018000939A80E080931F06E1E9FFE0AAE1B5E0E1
:1001900097E00E948DF5E1EEFFE0AFE1B1E00E9453
:1001A00083F5AFE1B1E08C91A3E2B5E08D938827B0
:1001B0008C93A3E2B5E00D911C91013050E015073E
:1001C0000CF402C00C94EA0081E090E0A3E2B5E0F8
:1001D0008D939C93EBEEFFE0A7E2B5E00E9483F5E0
:1001E000E6E1F8E0A5E2B5E00E9483F5009125057F
:1001F000013010F00C94FF0084E08093250580E02E
:100200008093F003E0EBF6E0AFE1B1E00E9483F50C
:10021000AFE1B1E00D9111274CE350E00E948DF168
:10022000ADECB4E00D931C93E6E2F8E0A2EFB6E08B
:100230000E9483F5EEE3F0E0A5E1B7E094E00E94D0
:100240008DF5EBE6FFE0AAE1B7E00E9483F581E0DF
:100250008093840400918404033018F011F00C940E
:100260007503E4E8F4E0A190BB24E2E1F0E0EA0DDC
:10027000FB1DAFE1B1E00E9483F5AFE1B1E00D916C
:1002800011274CE350E00E948DF1A4E8B4E0AD905A
:10029000BB24AFE9B4E0AA0CBB1CAA0DBB1D0D9397
:1002A0001C93E4E8F4E0A190BB24E5E1F0E0EA0D62
:1002B000FB1DAFE1B1E00E9483F5AFE1B1E00D912C
:1002C00011274CE350E00E948DF1A4E8B4E0AD901A
:1002D000BB24A5EAB4E0AA0CBB1CAA0DBB1D0D9360
:1002E0001C93E4E8F4E0A190BB24E6E9F0E0EA0D19
:1002F000FB1DAFE1B1E00E9483F5AFE1B1E00D91EC
:1003000011274CE350E00E948DF1A4E8B4E0AD90D9
:10031000BB24AAEBB4E0AA0CBB1CAA0DBB1D0D9319
:100320001C93E4E8F4E0A190BB24EEE1F8E0AA0C11
:10033000BB1CEA0DFB1DA4E8B4E0AD90BB24AFE705
:10034000B6E0AA0CBB1CAA0DBB1D0E9485F5E4E813
:10035000F4E0A190BB24E6E8FFE0AA0CBB1CEA0D88
:10036000FB1DA4E8B4E0AD90BB24A6E6B6E0AA0C61
:10037000BB1CAA0DBB1D0E9485F5E4E8F4E0A1902A
:10038000BB24EDE8FFE0EA0DFB1DA4E8B4E0AD906E
:10039000BB24A0E7B6E0AA0DBB1D0E9483F5E4E8EC
:1003A000F4E0A190BB24E4EAF0E0AA0CBB1CEA0D47
:1003B000FB1DA4E8B4E0AD90BB24A4E2B4E0AA0C19
:1003C000BB1CAA0DBB1D0E9485F5A4E8B4E0AD904E
:1003D000BB24A4E2B4E0AA0CBB1CAA0DBB1D8D91EA
:1003E0009C91A4E8B4E0AD90BB24AEE1B4E0AA0CCB
:1003F000BB1CAA0DBB1D8D939C93E4E8F4E0A19077
:10040000BB24EFE0F0E0EA0DFB1DA4E8B4E0AD9002
:10041000BB24A6E0B4E0AA0DBB1D0E9483F5E4E86E
:10042000F4E0A190BB24EFE9F0E0EA0DFB1DA4E8A5
:10043000B4E0AD90BB24ACE0B4E0AA0DBB1D0E94BB
:1004400083F5E4E8F4E0A190BB24EDE1F0E0AA0C30
:10045000BB1CEA0DFB1DA4E8B4E0AD90BB24A3ECEB
:10046000B4E0AA0CBB1CAA0DBB1D0E9485F5E4E8F4
:10047000F4E0A190BB24EFE8F0E0AA0CBB1CEA0D6D
:10048000FB1DA4E8B4E0AD90BB24A9E4B5E0AA0C40
:10049000BB1CAA0DBB1D0E9485F581E0A4E8B4E059
:1004A000AD90BB24A8E0B5E0AA0DBB1D8C9381E004
:1004B000A4E8B4E0AD90BB24A1E4B5E0AA0DBB1D57
:1004C0008C93E4E8F4E0A190BB24E2EAF0E0EA0DCA
:1004D000FB1DA4E8B4E0AD90BB24AEE0B6E0AA0DED
:1004E000BB1D0E9483F581E0A4E8B4E0AD90BB247D
:1004F000ACEFB4E0AA0DBB1D8C9381E0A4E8B4E09E
:10050000AD90BB24AFEFB4E0AA0DBB1D8C93E4E823
:10051000F4E0A190BB24ECE9F0E0EA0DFB1DA4E8B7
:10052000B4E0AD90BB24ABE1B6E0AA0DBB1D0E94C8
:1005300083F5E4E8F4E0A190BB24E9E6F0E0EA0DFD
:10054000FB1DA4E8B4E0AD90BB24AFE1B6E0AA0D7A
:10055000BB1D0E9483F581E0A4E8B4E0AD90BB240C
:10056000A2E2B6E0AA0DBB1D8C93E4E8F4E0A190F2
:10057000BB24E4E2F0E0EA0DFB1DA4E8B4E0AD909A
:10058000BB24A5E2B6E0AA0DBB1D0E9483F5E4E8FA
:10059000F4E0A190BB24E6E2F0E0AA0CBB1CEA0D5B
:1005A000FB1DA4E8B4E0AD90BB24A7E2B6E0AA0C22
:1005B000BB1CAA0DBB1D0E9485F5E4E8F4E0A190E8
:1005C000BB24E7E6FFE0EA0DFB1DA4E8B4E0AD9034
:1005D000BB24A3E4B6E0AA0DBB1D0E9483F5E4E8AA
:1005E000F4E0A190BB24E0E6FFE0AA0CBB1CEA0DFE
:1005F000FB1DA4E8B4E0AD90BB24A0E5B6E0AA0CD6
:10060000BB1CAA0DBB1D0E9485F5E4E8F4E0A19097
:10061000BB24E4E3F0E0EA0DFB1DA4E8B4E0AD90F8
:10062000BB24AAE8B6E0AA0DBB1D0E9483F5E4E84E
:10063000F4E0A190BB24EEE2F0E0EA0DFB1DA4E89B
:10064000B4E0AD90BB24ABE7B6E0AA0DBB1D0E94A1
:1006500083F5A4E8B4E00D91112748E450E00E942E
:100660008DF1A5E2B1E0A00FB11F0E94BFF3A4E895
:10067000B4E00D91112748E450E00E948DF1A5E40B
:10068000B2E0A00FB11F0E94BFF3E4E8F4E0A19034
:10069000BB24E9E0F0E0EA0DFB1DA4E8B4E0AD9076
:1006A000BB24ABEFB6E0AA0DBB1D0E9483F5E4E8C6
:1006B000F4E0A190BB24E6E2F8E0AA0CBB1CEA0D32
:1006C000FB1DA4E8B4E0AD90BB24A4EFB6E0AA0CF7
:1006D000BB1CAA0DBB1D0E9485F5A4E8B4E08C915B
:1006E0008F5F8C9310F40C942A0181E080931F019A
:1006F00000911F01053018F011F00C94B103EFE1E7
:10070000F1E0A190BB24EEEAF0E0EA0DFB1DAFE1C1
:10071000B1E0AD90BB24A3E0B6E0AA0DBB1D0E94E2
:1007200083F5AFE1B1E0AD90BB24A2E5B5E0AA0C42
:10073000BB1CAA0DBB1D0E94BFF3AFE1B1E0AD90A1
:10074000BB24ACE5B5E0AA0CBB1CAA0DBB1D0E94E6
:10075000BFF3AFE1B1E08C918F5F8C9310F40C94F8
:10076000780381E08093840400918404043118F0BC
:1007700011F00C94D503E4E8F4E0A190BB24E9ED7A
:10078000F2E0EA0DFB1DA4E8B4E0AD90BB24A4E5C3
:10079000B4E0AA0DBB1D0E9483F5A4E8B4E08C91DF
:1007A0008F5F8C9310F40C94B4030E9428DF87E0D1
:1007B00086B980E487B9379AA0E2B1E0E4EAFDEEB9
:1007C0000E94DDF30E9497F1809119058F7B809341
:1007D0001905E0E2F1E0FA93EA930E9431D42296FF
:1007E000E0E2F1E0FA93EA930E9498D322960E9405
:1007F0004FF080E08093860480E28093870492E04B
:10080000A6E8B4E00E9445F080ED97E00E94EBF08E
:10081000A0E2B1E00E94BFF30B990C9449040E9B37
:100820000C94490484EF91E00E94EBF00B990C9436
:1008300049040E9B0C944904A42DB52DE6EAFDEE67
:100840000E94DDF30E9497F1EFE4F0E0A42DB52DB6
:100850007BE70E9478F5A42DB52DECEAFDEE0E9411
:10086000DDF30E9497F1E8E5F0E0A42DB52D7BE7DC
:100870000E9478F5A42DB52DE2EBFDEE0E94DDF38C
:100880000E9497F1E1E6F0E0A42DB52D7BE70E94F0
:1008900078F50E9493EB81E090E0ACE0B5E08D93B9
:1008A0009C9381E080931F0681E08093380481E06F
:1008B0008093510481E08093940480E08093F2035C
:1008C00080E08093F30380E08093F4030E9401C1F1
:1008D00081E08093940400919404053018F011F0A5
:1008E0000C94A8040091940441E0040FA9E4B4E03E
:1008F0000C93A9E4B4E08C91A9E3B0E00E94D7F393
:100900000E94CDF30C900822689409F4E89416F044
:100910000C94960481E0A4E9B4E0AD90BB24A9E076
:10092000B7E0AA0DBB1D8C930C94A00480E0A4E951
:10093000B4E0AD90BB24A9E0B7E0AA0DBB1D8C9339
:10094000A4E9B4E08C918F5F8C9310F40C946B0449
:1009500081E08093940480E08093490481E0809357
:10096000510481E08093380481E08093850481E024
:100970008093FE030E94B01080E991E00E94EBF0AA
:100980008AEB80936B040E94F11280E08093510403
:1009900080E08093380480E08093FE030E94B010D2
:1009A000809101018F7780930101709164007260E2
:1009B000709364007091650072607093650070912F
:1009C00064007E7F7093640088EC809353044091B0
:1009D000540400918A04041711F40C94F5040E9445
:1009E00025E780918A0480935404A9E6B4E08C91B1
:1009F00087FB16F40C9465050E9415F0082F013052
:100A000011F00C9465050E94D8E9AEEEB6E08C9129
:100A100082FB16F40C9465058091EE068460809349
:100A2000EE06A1E0B1E08C9185FBAFE0B7E088274E
:100A300080F98C93A1E0B1E08C9184FBA0E1B7E058
:100A4000882780F98C93A1E0B1E08C9183FBA1E130
:100A5000B7E0882780F98C93A1E0B1E08C9182FB0C
:100A6000A2E1B7E0882780F98C93A1E0B1E08C91F6
:100A700081FBA3E1B7E0882780F98C93A1E0B1E086
:100A80008C9180FBA4E1B7E0882780F98C9380915A
:100A900001018F7D80930101809101018F7E809300
:100AA000010180910101877F809301018091010103
:100AB0008B7F80930101809101018D7F80930101E3
:100AC000809101018E7F80930101A3E6B0E00C913B
:100AD00000FB16F00C94F506A1E9B6E036E40E949E
:100AE000B2F084E690E00E94EBF0A1E9B6E00E944B
:100AF000A7F5EA2FFB2F3297F0400FEFA2E2B7E005
:100B00000E9459F5A2E2B7E00E94FEF4AAE1B1E02A
:100B10000C93E1E9F6E002E0A2E2B7E00E9459F5A9
:100B2000A2E2B7E0E8EBFDEE0E94DDF30E94ADF536
:100B300011F00C94B90580E0AAE1B1E0AD90BB24BE
:100B4000A6E8B6E0AA0DBB1D8C9380E0AAE1B1E057
:100B5000AD90BB24ADEFB3E0AA0DBB1D8C9380918B
:100B60001A018093F0030E94717E0E94B0100C94D1
:100B7000F106ECEBFDEE0E94DDF30E94ADF511F005
:100B80000C94190683E0E1E9F6E001E00A93A2E2A1
:100B9000B7E00E9452F5A2E2B7E00E94FEF4A0EF97
:100BA000B3E00C935A924A9281E0A42DB52D8C9318
:100BB00081E00E9485EF5A924A9288E0A42DB52DDB
:100BC0008C9381E00E9485EF5A924A928091F003C3
:100BD000A42DB52D8C9381E00E9485EF0E9421DE2B
:100BE000269683E00E9481EF81E0A0EFB3E0AD9014
:100BF000BB24A6E8B6E0AA0DBB1D8C935A924A927C
:100C00008091F003A42DB52D8C9381E00E9485EF97
:100C10005A924A9281E0A42DB52D8C9381E00E94D6
:100C200085EF0E94BB2A249682E00E9481EF0C94FB
:100C3000F106E0ECFDEE0E94DDF30E94ADF511F04F
:100C40000C9481068091EE0680618093EE0681E02F
:100C50008093EF03A1E9B6E00E94A7F5AAE1B1E015
:100C60008C93AAE1B1E08C9182508C93A1E9B6E01B
:100C70000E94A7F5EA2FFB2F00911A013197E01B84
:100C8000F0400FEFA5E4B2E00E9459F5E5E4F2E090
:100C9000FA93EA93E8E4F8E4FA93EA93E5E6F3E0FA
:100CA000FA93EA93E8E4F8E4FA93EA93E0EDF3E0E8
:100CB000FA93EA93EFEEF3E0FA93EA930E9421DDD0
:100CC0002C9680E08093D403A0E2B1E00E94A7F5C7
:100CD000082F003018F011F00C9470060C947F0669
:100CE0000E94BC3E8091B7038F778093B703A5E441
:100CF000B2E00E94BFF3A5E6B3E00E94BFF30C94FC
:100D0000F106E4ECFDEE0E94DDF30E94ADF511F07A
:100D10000C94B2068091EE0688608093EE06809176
:100D20001A018093F00380E0AAE1B1E0AD90BB240A
:100D3000ADEFB3E0AA0DBB1D8C9380E0AAE1B1E05A
:100D4000AD90BB24A6E8B6E0AA0DBB1D8C930E9413
:100D5000717E8091EE06877F8093EE060E94B01030
:100D60000C94F106E8ECFDEE0E94DDF30E94ADF577
:100D700011F00C94BF060E9403EF0C94F106ECEC0A
:100D8000FDEE0E94DDF30E94ADF511F00C94CC064F
:100D90000E9403EF0C94F106E0EDFDEE0E94DDF3FE
:100DA0000E94ADF511F00C94D9060E9403EF0C944B
:100DB000F106E4EDFDEE0E94DDF30E94ADF511F0C9
:100DC0000C94E6060E9403EF0C94F106E8EDFDEEAC
:100DD0000E94DDF30E94ADF511F00C94F1060E9423
:100DE00003EFA1E9B6E00E94BFF30091D003013008
:100DF00011F00C94810780910101806480930101BE
:100E00008091B70380648093B70380912605886042
:100E1000809326058091690480618093690480E055
:100E2000809374068091260584608093260581E076
:100E30008093EF03E5E4F2E0FA93EA93E8E4F8E460
:100E4000FA93EA93E5E6F3E0FA93EA93E8E4F8E448
:100E5000FA93EA93E0EDF3E0FA93EA93EFEEF3E02E
:100E6000FA93EA930E9421DD2C9680E08093D403CC
:100E7000A0E2B1E00E94A7F5082F003018F011F0B1
:100E80000C9444070C9481070E94BC3EE0E2F1E020
:100E900005E0ADEAB3E00E9459F5A7EBB3E08C9111
:100EA00087FB16F00C946607A2E2B7E0ECEDFDEECE
:100EB0000E94DDF30E9497F1EDEAF3E0A2E2B7E0D1
:100EC0000E940EF00E9447F50C947607A2E2B7E06C
:100ED000EEEDFDEE0E94DDF30E9497F1EDEAF3E006
:100EE000A2E2B7E00E940EF00E9447F5A2E2B7E04E
:100EF0000E9423F00E9435F08091B7038F77809392
:100F0000B70300917406023010F40C94F30780913B
:100F100026058B7F80932605809101018F7B80932E
:100F200001018091B7038F7B8093B70381E08093A9
:100F3000420581E08093430581E0809344058091E0
:100F40002605877F80932605809169048F7E809394
:100F5000690480E0809374068091EE068B7F809315
:100F6000EE0600910F07013011F00C94BC07809140
:100F7000010180628093010100911007013011F09E
:100F80000C94C70780910101806180930101009159
:100F90001107013011F00C94D20780910101886093
:100FA0008093010100911207013011F00C94DD07CC
:100FB0008091010184608093010100911307013049
:100FC00011F00C94E8078091010182608093010187
:100FD00000911407013011F00C94F3078091010186
:100FE0008160809301010E947D18A4E9B4E0AD9076
:100FF000BB24A6E8B6E0AA0DBB1D0C91003011F091
:101000000C94FD0CA6E2B5E08C9182FB16F40C94D6
:10101000FD0CA4E9B4E0AD90BB24ADE8B4E0AA0DAA
:10102000BB1D0C91003081E010F009F080E08F933F
:10103000A4E9B4E0AD90BB24ADE8B4E0AA0DBB1DBB
:101040000C91083080E010F009F081E09F91892B2D
:10105000882311F40C94360881E0A4E9B4E0AD9043
:10106000BB24ADE8B4E0AA0DBB1D8C93A4E9B4E0A9
:10107000AD90BB24A1EFB3E0AA0DBB1D0C910030D5
:1010800018F011F00C9446080C945208A4E9B4E04E
:10109000AD90BB24A0E1B6E0AA0CBB1CAA0DBB1D01
:1010A0000E94BFF3A4E9B4E0AD90BB24ADE8B4E086
:1010B000AA0DBB1D0C91013011F00C94A408A4E9F9
:1010C000B4E0AD90BB24A3E9B4E0AA0CBB1CAA0D0C
:1010D000BB1D0E94BFF3A4E9B4E0AD90BB24A9E915
:1010E000B4E0AA0CBB1CAA0DBB1D0E94BFF380E09C
:1010F000A4E9B4E0AD90BB24ACEAB4E0AA0DBB1DFA
:101100008C9380E0A4E9B4E0AD90BB24AFEAB4E0F6
:10111000AA0DBB1D8C93A4E9B4E0AD90BB24A0E95B
:10112000B4E0AA0DBB1D0C91013011F00C94A20883
:1011300082E0A4E9B4E0AD90BB24ADE8B4E0AA0D30
:10114000BB1D8C930C94E30B023011F00C945309EB
:10115000A4E9B4E0AD90BB24ABE7B6E0AA0DBB1D9B
:101160000C91003011F00C94C5085A924A9280916B
:101170009404A42DB52D8C9381E00E9485EF0E94EC
:101180000F2C229681E00E9481EF84E0A4E9B4E074
:10119000AD90BB24A4E4B5E0AA0DBB1D8C93A4E9DB
:1011A000B4E0AD90BB24A1EFB3E0AA0DBB1D0C9140
:1011B000003011F00C945109A4E9B4E0AD90BB24C7
:1011C000AEE0B6E0AA0DBB1D0C91013081E009F044
:1011D00080E08F93A4E9B4E0AD90BB24AAE8B6E028
:1011E000AA0DBB1D0C91013081E009F080E09F91B8
:1011F000892B882311F40C942E09A4E9B4E0AD9056
:10120000BB24A3E4B6E0AA0DBB1D0C91013011F084
:101210000C94180981E0A4E9B4E0AD90BB24A5E0EA
:10122000B5E0AA0DBB1D8C930E94D2400C942409FA
:1012300081E0A4E9B4E0AD90BB24A2E0B5E0AA0D42
:10124000BB1D8C930E94D88081E0A4E9B4E0AD90EE
:10125000BB24A4E4B5E0AA0DBB1D8C93A4E9B4E0C3
:10126000AD90BB24A0E9B4E0AA0DBB1D0C910130E8
:1012700011F00C94470983E0A4E9B4E0AD90BB24DD
:10128000ADE8B4E0AA0DBB1D8C930C94510986E027
:10129000A4E9B4E0AD90BB24ADE8B4E0AA0DBB1D59
:1012A0008C930C94E30B033011F00C948F09A4E998
:1012B000B4E0AD90BB24A3E9B4E0AA0CBB1CAA0D1A
:1012C000BB1D0E94BFF3A4E9B4E0AD90BB24A9E923
:1012D000B4E0AA0CBB1CAA0DBB1D0E94BFF380E0AA
:1012E000A4E9B4E0AD90BB24ACEAB4E0AA0DBB1D08
:1012F0008C9381E0A4E9B4E0AD90BB24AFEAB4E004
:10130000AA0DBB1D8C9384E0A4E9B4E0AD90BB248E
:10131000ADE8B4E0AA0DBB1D8C930C94E30B043034
:1013200011F00C94100A00919404013011F00C9407
:10133000BE09A7EAB4E04D915C91ABE9B4E00D9130
:101340001C91041715070CF002C00C94BC09009105
:101350000405003011F00C94BC0900910505003023
:1013600011F00C94BC090091F503003011F00C94BD
:10137000BC0985E080938E040C940E0A023011F0B3
:101380000C94E709A9EAB4E04D915C91ADE9B4E0B1
:101390000D911C91041715070CF002C00C94E5097F
:1013A00000910305003011F00C94E509009105054A
:1013B000003011F00C94E5090091F603003011F0B3
:1013C0000C94E50985E080938F040C940E0A033099
:1013D00011F00C940E0AABEAB4E04D915C91AFE9C8
:1013E000B4E00D911C91041715070CF002C00C9489
:1013F0000E0A00910405003011F00C940E0A0091C1
:101400000305003011F00C940E0A0091F703003030
:1014100011F00C940E0A85E0809390040C94E30B79
:10142000053011F00C94A50AA4E9B4E0AD90BB24FA
:10143000AEE0B6E0AA0DBB1D0C91013081E009F0D1
:1014400080E08F93A4E9B4E0AD90BB24AAE8B6E0B5
:10145000AA0DBB1D0C91013081E009F080E09F9145
:10146000892B882311F40C94800AA4E9B4E0AD9090
:10147000BB24A0E5B6E0AA0CBB1CAA0DBB1D4D9178
:101480005C91A4E9B4E0AD90BB24A0E1B6E0AA0C65
:10149000BB1CAA0DBB1D0D911C910417150780E004
:1014A0000CF481E08F93A4E9B4E0AD90BB24A3E4F5
:1014B000B6E0AA0DBB1D0C91003081E009F080E080
:1014C0009F91892B882311F40C94740A81E0A4E97C
:1014D000B4E0AD90BB24A2E0B5E0AA0DBB1D8C9397
:1014E0000E94D8800C94800A81E0A4E9B4E0AD9019
:1014F000BB24A5E0B5E0AA0DBB1D8C930E94D24091
:10150000A4E9B4E0AD90BB24A0E9B4E0AA0DBB1DF2
:101510000C91013011F00C94990A83E0A4E9B4E035
:10152000AD90BB24ADE8B4E0AA0DBB1D8C930C9428
:10153000A30A86E0A4E9B4E0AD90BB24ADE8B4E032
:10154000AA0DBB1D8C930C94E30B063011F00C9488
:10155000CB0AA4E9B4E0AD90BB24A3E9B4E0AA0CA3
:10156000BB1CAA0DBB1D0E94BFF381E0A4E9B4E03F
:10157000AD90BB24ACEAB4E0AA0DBB1D8C9387E010
:10158000A4E9B4E0AD90BB24ADE8B4E0AA0DBB1D66
:101590008C930C94E30B073011F00C949D0BA4E991
:1015A000B4E0AD90BB24A0E9B4E0AA0DBB1D0C9142
:1015B000013011F00C94200BA4E9B4E0AD90BB24F1
:1015C000A3E9B4E0AA0CBB1CAA0DBB1D8D919C9194
:1015D000A4E9B4E0AD90BB24A9E9B4E0AA0CBB1C1B
:1015E000AA0DBB1D8D939C93A4E9B4E0AD90BB24E0
:1015F000A3E9B4E0AA0CBB1CAA0DBB1D0E94BFF35B
:1016000080E0A4E9B4E0AD90BB24ACEAB4E0AA0D5C
:10161000BB1D8C9381E0A4E9B4E0AD90BB24AFEA9C
:10162000B4E0AA0DBB1D8C9384E0A4E9B4E0AD90B6
:10163000BB24ADE8B4E0AA0DBB1D8C930C949B0BAE
:1016400000919404013011F00C944B0BA1EAB4E02A
:101650004D915C91A5E9B4E00D911C91041715071B
:101660000CF002C00C94490B00910405003011F0FD
:101670000C94490B00910505003011F00C94490BB6
:101680000091F203003011F00C94490B81E080933B
:101690008E040C949B0B023011F00C94740BA3EA93
:1016A000B4E04D915C91A7E9B4E00D911C91041751
:1016B00015070CF002C00C94720B0091030500306A
:1016C00011F00C94720B00910505003011F00C9490
:1016D000720B0091F303003011F00C94720B81E057
:1016E00080938F040C949B0B033011F00C949B0B94
:1016F000A5EAB4E04D915C91A9E9B4E00D911C918B
:10170000041715070CF002C00C949B0B0091040504
:10171000003011F00C949B0B00910305003011F088
:101720000C949B0B0091F403003011F00C949B0B74
:1017300081E0809390040C94E30B083011F00C943A
:10174000E30BA4E9B4E0AD90BB24A6E4B6E0AA0D97
:10175000BB1D0C91003018F011F00C94E30BA4E9C0
:10176000B4E0AD90BB24AFEAB4E0AA0DBB1D8C91F0
:10177000A4E9B4E0AD90BB24ADE8B4E0AA0DBB1D74
:101780008C93A4E9B4E0AD90BB24A4E2B4E0AA0C2D
:10179000BB1CAA0DBB1D8D919C91A4E9B4E0AD903A
:1017A000BB24AEE1B4E0AA0CBB1CAA0DBB1D8D93FB
:1017B0009C9380E0A4E9B4E0AD90BB24A9E4B6E03A
:1017C000AA0DBB1D8C9380E0A4E9B4E0AD90BB24CE
:1017D000A0E9B4E0AA0DBB1D8C93A4E9B4E0AD90E0
:1017E000BB24A4E4B5E0AA0DBB1D0C91003081E040
:1017F00010F009F080E08F93A4E9B4E0AD90BB2431
:10180000A4E4B5E0AA0DBB1D0C91043080E010F0FB
:1018100009F081E09F91892B882311F40C941A0C14
:1018200080E0A4E9B4E0AD90BB24A4E4B5E0AA0D47
:10183000BB1D8C93A4E9B4E0AD90BB24A4E4B5E057
:10184000AA0DBB1D0C91013011F00C94C20CA4E93F
:10185000B4E0AD90BB24A1E4B5E0AA0DBB1D0C9192
:10186000003011F00C94400C84E0A4E9B4E0AD9099
:10187000BB24A4E4B5E0AA0DBB1D8C930C94C00C52
:10188000A4E9B4E0AD90BB24AEE0B6E0AA0DBB1D68
:101890000C91013081E009F080E08F93A4E9B4E07D
:1018A000AD90BB24A1EFB3E0AA0DBB1D0C9100309D
:1018B00081E009F080E09F918923882311F40C9442
:1018C0009D0C00919404013011F00C946B0C0E945B
:1018D000452F0C94790C023011F00C94730C0E947B
:1018E000B9330C94790C033011F00C94790C0E94EC
:1018F0000C385A924A9280E0A42DB52D8C9381E049
:101900000E9485EF5A924A9285E0A42DB52D8C93C2
:1019100081E00E9485EF5A924A9280919404A42D0E
:10192000B52D8C9381E00E9485EF0E9421DE2696E2
:1019300083E00E9481EF0C94C00CA4E9B4E0AD9068
:10194000BB24A1EFB3E0AA0DBB1D0C91013011F037
:101950000C94B60C84E0A4E9B4E0AD90BB24A4E4FC
:10196000B5E0AA0DBB1D8C930C94C00C83E0A4E9D8
:10197000B4E0AD90BB24A4E4B5E0AA0DBB1D8C93EC
:101980000C94FD0C043011F00C94DF0CA4E9B4E0CD
:10199000AD90BB24A1E4B5E0AA0DBB1D0C910130B4
:1019A00011F00C94DD0C81E0A4E9B4E0AD90BB240F
:1019B000A4E4B5E0AA0DBB1D8C930C94FD0C023081
:1019C00011F00C94EF0C80E0A4E9B4E0AD90BB24DE
:1019D000A4E4B5E0AA0DBB1D8C930C94FD0C033060
:1019E00011F00C94FD0C80E0A4E9B4E0AD90BB24B0
:1019F000A4E4B5E0AA0DBB1D8C93E4E9F4E0A1904A
:101A0000BB24E1E3F0E0EA0DFB1DA0E1B0E00E94A1
:101A100083F5013011F00C94400DA4E9B4E0AD90D1
:101A2000BB24A4E4B5E0AA0DBB1D0C91003011F05D
:101A30000C94400DA4E9B4E0AD90BB24ACE0B4E05C
:101A4000AA0DBB1D0C91003011F40C94400D5A925C
:101A50004A9280919404A42DB52D8C9381E00E942C
:101A600085EF5A924A9280E0A42DB52D8C9381E0A7
:101A70000E9485EF0E94BB2A249682E00E9481EF9B
:101A8000ADECB4E04D915C91ABECB4E00D911C91E8
:101A9000041715070CF002C00C945C0DABECB4E01D
:101AA0000E94BFF380E080933F04809169048F7BA4
:101AB000809369040E94B01081E0809349040091F2
:101AC0004904053018F011F00C947D0DA9E4B4E040
:101AD000AD90BB24A3E0B6E0AA0DBB1D0C91013074
:101AE00011F00C94750D0E944DB6A9E4B4E08C91F0
:101AF0008F5F8C9310F40C945F0DA4E9B4E0AD906B
:101B0000BB24AAEBB4E0AA0CBB1CAA0DBB1D0D9113
:101B10001C91003050E0150711F40C94D50DA4E988
:101B2000B4E0AD90BB24AAEBB4E0AA0CBB1CAA0D98
:101B3000BB1D4D915C91A4E9B4E0AD90BB24A1EB39
:101B4000B4E0AA0CBB1CAA0DBB1D0D911C9104177F
:101B500015070CF002C00C94D50DA4E9B4E0AD90CB
:101B6000BB24AFE7B6E0AA0CBB1CAA0DBB1D8D9130
:101B70009C91ACE0B5E08D939C930E9401C180E004
:101B8000A4E9B4E0AD90BB24A8EBB4E0AA0DBB1D62
:101B90008C93A4E9B4E0AD90BB24A1EBB4E0AA0C13
:101BA000BB1CAA0DBB1D0E94BFF3A4E9B4E0AD901D
:101BB000BB24A4E2B4E0AA0CBB1CAA0DBB1D0D9172
:101BC0001C91003050E0150711F40C94BD0EA4E9EF
:101BD000B4E0AD90BB24A9E4B6E0AA0DBB1D0C9106
:101BE000003011F00C94BD0EA4E9B4E0AD90BB241C
:101BF000AEE1B4E0AA0CBB1CAA0DBB1D0D911C915B
:101C00000F3F5FEF15070CF402C00C94BD0E5A9203
:101C10004A9280E0A42DB52D8C9381E00E9485EF3F
:101C20005A924A9280919404A42DB52D8C9381E010
:101C30000E9485EF5A924A9280919404A42DB52D6A
:101C40008C9381E00E9485EF0E9421DE269683E03E
:101C50000E9481EF809194048093510481E0A4E973
:101C6000B4E0AD90BB24A1E3B4E0AA0DBB1D8C93FE
:101C70008EEB80936B0483ED80936C0482E0809301
:101C800085040E94F11281E0A4E9B4E0AD90BB2488
:101C9000ABE2B4E0AA0DBB1D8C93E8E3F0E0A0E159
:101CA000B0E00E9483F5013011F00C94A50E009174
:101CB0009404013011F00C94730EA1E0B1E08C910A
:101CC00085FB16F00C94670E81E080933004A1E050
:101CD000B1E08C9184FB16F00C94710E81E080933E
:101CE00031040C94A50E023011F00C948D0EA1E07D
:101CF000B1E08C9183FB16F00C94810E81E080930F
:101D00002F04A1E0B1E08C9182FB16F00C948B0EB5
:101D100081E0809331040C94A50E033011F00C94F3
:101D2000A50EA1E0B1E08C9181FB16F00C949B0E06
:101D300081E080932F04A1E0B1E08C9180FB16F04C
:101D40000C94A50E81E080933004A4E9B4E0AD903A
:101D5000BB24A4E2B4E0AA0CBB1CAA0DBB1D8D9150
:101D60009C91A4E9B4E0AD90BB24AEE1B4E0AA0C30
:101D7000BB1CAA0DBB1D8D939C93A4E9B4E0AD9050
:101D8000BB24A9E4B5E0AA0CBB1CAA0DBB1D4D9158
:101D90005C91A4E9B4E0AD90BB24A7E4B5E0AA0D42
:101DA000BB1D0D911127041715071CF011F00C94A1
:101DB000DB0E0C940C0F80E0A4E9B4E0AD90BB24E2
:101DC000A7E4B5E0AA0DBB1D8C9380E0A4E9B4E0C4
:101DD000AD90BB24ADEFB3E0AA0DBB1D8C9380E0AA
:101DE000A4E9B4E0AD90BB24A0E5B5E0AA0DBB1D0D
:101DF0008C93E4E9F4E0FA93EA935A924A9280E0F1
:101E0000A42DB52D8C9381E00E9485EF0E946ADF9E
:101E1000249681E00E9481EFA4E9B4E0AD90BB2458
:101E2000A4EFB6E0AA0CBB1CAA0DBB1D0D911C9122
:101E3000003050E0150711F40C94670FA4E9B4E0EA
:101E4000AD90BB24A2EFB6E0AA0DBB1D0C910130F2
:101E500011F00C94670FA4E9B4E0AD90BB24A4EF9B
:101E6000B6E0AA0CBB1CAA0DBB1D4D915C91A4E968
:101E7000B4E0AD90BB24ADEFB6E0AA0CBB1CAA0D3C
:101E8000BB1D0D911C91041715071CF011F00C944B
:101E90004B0F0C94670FA4E9B4E0AD90BB24ADEFF9
:101EA000B6E0AA0CBB1CAA0DBB1D0E94BFF3A4E99F
:101EB000B4E0AD90BB24ABEFB6E0AA0DBB1D8C9196
:101EC000ACE0B5E08D9388278C930E9401C1A4E912
:101ED000B4E0AD90BB24ACECB3E0AA0DBB1D0C91FB
:101EE000013011F00C942A10A4E9B4E0AD90BB24A9
:101EF000A0EDB3E0AA0DBB1D8C918093EF03009180
:101F00009404013011F00C948A0F89B78E7F89BF39
:101F10000C949A0F023011F00C94930F89B78D7FB7
:101F200089BF0C949A0F033011F00C949A0F89B763
:101F30008B7F89BFE4E9F4E00191112748E450E088
:101F40000E948DF1E5E2F1E0E00FF11FFA93EA93D0
:101F5000E8E4F8E4FA93EA93E4E9F4E00191112764
:101F600048E450E00E948DF1E5E4F2E0E00FF11F5B
:101F7000FA93EA93E8E4F8E4FA93EA93E4E9F4E004
:101F8000A190BB24ECECF3E0EA0DFB1DFA93EA937D
:101F9000EFEEF3E0FA93EA930E9421DD2C9680E0C5
:101FA000A4E9B4E0AD90BB24A0EDB3E0AA0DBB1D45
:101FB0008C9300919404013011F00C94E40F89B7D4
:101FC000816089BF0C94F40F023011F00C94ED0F76
:101FD00089B7826089BF0C94F40F033011F00C9420
:101FE000F40F89B7846089BFA0E2B1E00E94A7F531
:101FF000082F003018F011F00C9400100C942A10E7
:1020000080E0A4E9B4E0AD90BB24A5E4B4E0AA0D5F
:10201000BB1D8C930E94BC3E81E0A4E9B4E0AD906E
:10202000BB24A1E4B5E0AA0DBB1D8C9380E0A4E91C
:10203000B4E0AD90BB24A5E3B6E0AA0DBB1D8C9324
:1020400080E0A4E9B4E0AD90BB24A2E4B4E0AA0D22
:10205000BB1D8C9381E080933506009134060530DA
:1020600018F011F00C9436100C947B10A5E3B6E038
:10207000AD90BB24A4E5B4E0AA0DBB1D0C910130CA
:1020800011F00C946810E5E3F6E0A190BB24E5ECB8
:10209000F2E0EA0DFB1DA9E4B4E00E9483F5A9E497
:1020A000B4E08C91ACE0B5E08D9388278C930E94CE
:1020B00001C180E08093340680E0A5E3B6E0AD90F6
:1020C000BB24A4E5B4E0AA0DBB1D8C930E94B01004
:1020D000A5E3B6E08C918F5F8C93009135060431B7
:1020E00018F011F00C9476100C94791080E0809325
:1020F00034060C942D1000919404013011F00C94CE
:1021000085100E94A62C0C949310023011F00C94B0
:102110008D100E945C2D0C949310033011F00C94E0
:1021200093100E94122EA9E6B4E08C9185FB16F460
:102130000C94A01080E08093380480E080935104D8
:10214000A4E9B4E08C918F5F8C93009194040430E7
:1021500010F40C94AE1081E0809394040C94E40489
:1021600081E00E94FAF081E00E94FAF081E00E9492
:10217000FAF081E00E94FAF081E00E94FAF081E03A
:10218000A885B9858C93A885B9850C91033018F082
:1021900011F00C94C911A1E0B1E08C9187FB16F409
:1021A0000C94EC10E885F985A190BB24E8E1F0E0FF
:1021B000EA0DFB1DA0E1B0E00E9483F5003011F0B4
:1021C0000C94EC1080E0A885B985AD90BB24ADEFF0
:1021D000B3E0AA0DBB1D8C93A885B985AD90BB2437
:1021E000ADE8B6E0AA0DBB1D0C91013081E009F00D
:1021F00080E08F93A885B985AD90BB24A6E8B6E0B2
:10220000AA0DBB1D0C91013081E009F080E09F9187
:10221000892B8F93A885B985AD90BB24AEEEB6E02F
:10222000AA0DBB1D0C91013081E009F080E09F9167
:10223000892B882311F40C943911A885B9850C9148
:10224000013011F00C94291181E08093FE030C946D
:102250003911023011F00C94321182E08093FF03A7
:102260000C943911033011F00C94391184E08093EF
:102270000004A885B985AD90BB24ADEFB3E0AA0DED
:10228000BB1D0C91003011F40C94B71181E0A885AE
:10229000B985AD90BB24ABE4B4E0AA0DBB1D8C9313
:1022A000E9EBF6E0A0E1B0E00E9483F5013011F027
:1022B0000C94A911A885B985AD90BB24A8E3B4E01E
:1022C000AA0DBB1D0C91013081E009F080E08F93D5
:1022D000A885B985AD90BB24ADE8B6E0AA0DBB1DBD
:1022E0000C91013081E009F080E09F91892B8F9360
:1022F000A885B985AD90BB24A6E8B6E0AA0DBB1DA4
:102300000C91013081E009F080E09F91892B8F933F
:10231000A885B985AD90BB24AEEEB6E0AA0DBB1D75
:102320000C91013081E009F080E09F91892B882396
:1023300011F40C94A711809169048064809369045E
:10234000ABECB4E00E94BFF380E480933F040C94B4
:10235000B51180916904806480936904ABECB4E0AA
:102360000E94BFF380E480933F040C94C11180E08D
:10237000A885B985AD90BB24ABE4B4E0AA0DBB1D24
:102380008C93A885B9858C918F5F8C9310F40C94F5
:10239000C3108091FE03AE81BF818C93AE81BF815B
:1023A0000C914091FF03042BAE81BF810C93AE8151
:1023B000BF810C9140910004042BAE81BF810C932E
:1023C000AE81BF810C9140910104042BAE81BF818D
:1023D0000C93AE81BF810C9140910204042BAE811D
:1023E000BF810C93AE81BF810C9140910304042BFB
:1023F000AE81BF810C93AE81BF810C9140913F04AF
:10240000042BAE81BF810C9380912A05AC81BD81E4
:102410008C9380913205AA81BB818C9382E0A88540
:10242000B9858C93A885B9850C91083018F011F006
:102430000C944212AC81BD810C91A885B985AD90F8
:10244000BB24A9E2B5E0AA0DBB1D4C91042BAC81C5
:10245000BD810C93AA81BB810C91A885B985AD90F3
:10246000BB24A1E3B5E0AA0DBB1D4C91042BAA81AE
:10247000BB810C93A885B9858C918F5F8C9310F4E8
:102480000C94121280913A05A881B9818C938AE04C
:10249000A885B9858C93A885B9850C91003118F071
:1024A00011F00C946B12A881B9810C91A885B985A3
:1024B000AD90BB24A1E3B5E0AA0DBB1D4C91042B4C
:1024C000A881B9810C93A885B9858C918F5F8C9375
:1024D00010F40C944B12C798D898D19AD09AD89AE5
:1024E000A881B981119698E08E91983018F4392F0F
:1024F000992702C038E09850881FD99808F4D99AD3
:1025000000000000D89800000000D89A00000000E9
:102510003A9591F7992341F7D19AD09AD89AAA81FE
:10252000BB81119698E08E91983018F4392F992735
:1025300002C038E09850881FD99808F4D99A000052
:102540000000D89800000000D89A000000003A95DA
:1025500091F7992341F7D19AD09AD89AAC81BD814D
:10256000119698E08E91983018F4392F992702C06F
:1025700038E09850881FD99808F4D99A00000000D4
:10258000D89800000000D89A000000003A9591F712
:10259000992341F7D19AD09AD89AAE81BF811196EA
:1025A00098E08E91983018F4392F992702C038E0BE
:1025B0009850881FD99808F4D99A00000000D8983C
:1025C00000000000D89A000000003A9591F7992386
:1025D00041F7C79AC79885E0481A8827580A2A966B
:1025E000089581E00E94FAF081E00E94FAF081E013
:1025F0000E94FAF085E00E94FAF082E00E94FAF070
:1026000081E00E94FAF081E00E94FAF081E00E94ED
:10261000FAF08091B70380688093B703A7EBB3E02B
:102620008C9186FB16F00C941E13AEEEB6E08C91E6
:1026300084FB16F40C941E130C94B41681E0AE8542
:10264000BF858C93AE85BF850C91033018F011F0D7
:102650000C945F135A924A9280E0A42DB52D8C936E
:1026600081E00E9485EF5A924A9284E0A42DB52D14
:102670008C9381E00E9485EF5A924A92AC89BD8981
:102680008C91A42DB52D8C9381E00E9485EF0E9442
:1026900021DE269683E00E9481EF80E0AE85BF8533
:1026A000AD90BB24ACE2B7E0AA0DBB1D8C93AE8508
:1026B000BF858C918F5F8C9310F40C942213009142
:1026C0005104013081E008F080E08F9300915104C3
:1026D000033080E010F009F081E09F91892B88237E
:1026E00011F40C94A31300913804003018F011F089
:1026F0000C947C130C949213A885B985E8E3F4E05C
:102700000E94B4F4E885F98501E0AE81BF810E94A2
:1027100059F5AE81BF810E94FEF4A1E5B4E00C93AF
:102720000C94A3130091F003003018F011F00C94F6
:102730009B130C94A3138091F00380935104809118
:10274000F0038093380481E08093840440918504F1
:1027500000918404041718F011F00C943A16A4E8C0
:10276000B4E0AD90BB24AAE6B4E0AA0DBB1D8C91E9
:1027700080936A0400916A040B3E18F011F00C94E7
:10278000C3130C941A14AAE6B4E08C918B5E8C935C
:1027900080916A04AA85BB858C9381E08093500464
:1027A0005A924A9281E0A42DB52D8C9381E00E942B
:1027B00085EF0E94BA16229681E00E9481EFA7EB76
:1027C000B3E08C9185FB16F00C94FD13AEEEB6E0F1
:1027D0008C9185FB16F40C94FD13A5E7B6E08D9162
:1027E0009C910E94EBF08091B7038F7D8093B7039B
:1027F0008091EE0680628093EE06EA85FB85FA936F
:10280000EA930E940BCA22965A924A9280E0A42D23
:10281000B52D8C9381E00E9485EF0E94BA16229616
:1028200081E00E9481EF8091EE0681608093EE0648
:102830000C943216AEEEB6E08C9180FB16F00C9440
:102840002E148091EE068E7F8093EE0680E38093B7
:10285000870492E0A6E8B4E00E9445F080E080930F
:10286000860488EE8093870400916A04003018F093
:1028700011F00C943D140C946D1492E0A6E8B4E0B1
:102880000E9445F088EF8093870481E0AE85BF8584
:102890008C9340916A04AE85BF850C91041718F0A3
:1028A00011F00C946D1492E0A6E8B4E00E9445F09B
:1028B000A6E8B4E08C918F5F8C93A3E6B0E00C9116
:1028C00002FB0EF002C00C945D14AE85BF858C91A6
:1028D0008F5F8C9310F40C94491480EF80938704DD
:1028E00000916A04003011F00C94791480EE80930A
:1028F00087045A924A9281E0A42DB52D8C9381E0F1
:102900000E9485EF0E94BA16229681E00E9481EF14
:10291000A7EBB3E08C9185FB16F00C94A614AEEEF9
:10292000B6E08C9185FB16F40C94A614A5E7B6E0EE
:102930008D919C910E94EBF08091B7038F7D8093E5
:10294000B7038091EE0680628093EE0692E0A6E8DF
:10295000B4E00E9445F0A3E6B0E00C9102FB0EF05B
:1029600072C10E94AC8480E0A881B9818C9381E01F
:10297000AA81BB818C93AA81BB810C91053018F090
:1029800011F00C940315AA81BB81AD90BB24AEE37A
:10299000B6E0AA0DBB1D0C91013011F00C94FB1494
:1029A000AA81BB81AD90BB24A8E0B6E0AA0DBB1DF7
:1029B0000C91003011F00C94FB14AA81BB81AD90F6
:1029C000BB24A3E0B6E0AA0DBB1D0C91013011F0B1
:1029D0000C94FB1480E08093860480E3809387044A
:1029E00092E0A6E8B4E00E9445F081E0A881B981B8
:1029F0008C930C940315AA81BB818C918F5F8C936F
:102A000010F40C94BB14A881B9810C91013011F021
:102A10000C941B155A924A9280E0A42DB52D8C93EC
:102A200081E00E9485EF0E94BA16229681E00E9402
:102A300081EF0C943A1680E0AC81BD818C9381E0EB
:102A4000AE85BF858C93AE85BF850C91033018F0A1
:102A500011F00C941416AE85BF85AD90BB24A1E394
:102A6000B4E0AA0DBB1D0C91003011F00C941416AB
:102A7000AE85BF85AD90BB24ACE2B7E0AA0DBB1D0F
:102A80000C91013011F00C940C1600911F060130CE
:102A900011F40C940C1680E0AC85BD858C93AE854A
:102AA000BF85AD90BB24A5E0B5E0AA0DBB1D0C9180
:102AB000013011F00C946D15AE85BF85AD90BB242F
:102AC000AFE1B6E0AA0DBB1D0C91013011F00C94E2
:102AD0006D1581E0AC85BD858C93AE85BF85AD90CD
:102AE000BB24ABE1B6E0AA0DBB1D0C91013011F087
:102AF0000C948B15AE85BF85AD90BB24A5E0B5E0E9
:102B0000AA0DBB1D0C91003011F00C948B1581E0C7
:102B1000AC85BD858C9300911F06023011F00C949A
:102B2000951581E0AC85BD858C93AEEEB6E08C91B9
:102B300087FB16F40C940C16AC85BD850C91013006
:102B400011F00C940C160E947D18AE85BF85AD90D7
:102B5000BB24A1EFB3E0AA0DBB1D0C91013011F015
:102B60000C940C1680E08093860480E380938704A5
:102B70005A924A9280E0A42DB52D8C9381E00E9458
:102B800085EF0E94BA16229681E00E9481EF92E0C2
:102B9000A6E8B4E00E9445F0AE85BF85AD90BB24A9
:102BA000A5E0B5E0AA0DBB1D0C91013011F00C940D
:102BB0000616AE85BF85AD90BB24A6E7B6E0AA0D8C
:102BC000BB1D0C91013011F00C94061680E0AE850F
:102BD000BF85AD90BB24A6E7B6E0AA0DBB1D8C93C4
:102BE00080E0AE85BF85AD90BB24A5E0B5E0AA0D21
:102BF000BB1D8C9381E0AE85BF85AD90BB24A2E068
:102C0000B5E0AA0DBB1D8C930E94D88081E0AC81F9
:102C1000BD818C930C941416AE85BF858C918F5F0B
:102C20008C9310F40C942315AC81BD810C91013070
:102C300011F00C94211680E0AC81BD818C930C9432
:102C40003A160C94AB145A924A9280E0A42DB52DFA
:102C50008C9381E00E9485EF0E94BA16229681E053
:102C60000E9481EFA4E8B4E08C918F5F8C9310F404
:102C70000C94A61380E08093CF0480E08093D0046E
:102C800080E08093D1045A924A9280E0A42DB52D21
:102C90008C9381E00E9485EF0E94BA16229681E013
:102CA0000E9481EF00911B06003018F011F00C9487
:102CB0005B160C94671681E0ABE1B6E0AD90BB24E7
:102CC000A2E0B5E0AA0DBB1D8C930E94D8800091B4
:102CD0005104003018F011F00C9470160C949316F7
:102CE000A1E5B4E0AD90BB24AEE0B6E0AA0DBB1DFB
:102CF0000C91003011F00C949316A1E5B4E0AD9066
:102D0000BB24A1EFB3E0AA0DBB1D0C91003011F064
:102D10000C949316A6E2B5E08C9184FB16F40C9407
:102D200093160E94B0105A924A9280E0A42DB52DBD
:102D30008C9381E00E9485EF5A924A9284E0A42D00
:102D4000B52D8C9381E00E9485EF5A924A9284E0DF
:102D5000A42DB52D8C9381E00E9485EF0E9421DE89
:102D6000269683E00E9481EF8DE0481A8827580A52
:102D700060960895AEEEB6E08C9184FB16F40C9448
:102D80005B1800910605013081E009F080E08F9327
:102D900000915104013081E009F080E09F91892B7E
:102DA0008F9300913804013081E009F080E09F9119
:102DB000892B8F93009138040C3081E009F080E07A
:102DC0009F91892B8F93009138040D3081E009F099
:102DD00080E09F91892B8F93009138040B3781E01D
:102DE00009F080E09F91892B882311F40C944917F6
:102DF00081E080932D075A924A92AA81BB818C91DF
:102E0000A42DB52D8C9381E00E9485EF5A924A92B1
:102E100084E0A42DB52D8C9381E00E9485EF5A9219
:102E20004A9281E0A42DB52D8C9381E00E9485EF1C
:102E30000E9421DE269683E00E9481EFA881B9815D
:102E40000C91013011F00C943A1781E08093CF047B
:102E500081E08093FE0300914C04003011F00C944B
:102E600038178091B70380628093B7030E94B01037
:102E70000C9449170091CF04003011F00C944917BD
:102E800000913904003011F00C94491780E08093D0
:102E9000FE0300910705013081E009F080E08F9387
:102EA00000915104023081E009F080E09F91892B6C
:102EB0008F9300913804023081E009F080E09F9107
:102EC000892B8F93009138040C3081E009F080E069
:102ED0009F91892B8F9300913804073181E009F08D
:102EE00080E09F91892B8F93009138040B3781E00C
:102EF00009F080E09F91892B882311F40C94D1175D
:102F000081E080932E075A924A92AA81BB818C91CC
:102F1000A42DB52D8C9381E00E9485EF5A924A92A0
:102F200084E0A42DB52D8C9381E00E9485EF5A9208
:102F30004A9282E0A42DB52D8C9381E00E9485EF0A
:102F40000E9421DE269683E00E9481EFA881B9814C
:102F50000C91013011F00C94C21781E08093D004E1
:102F600082E08093FF0300914D04003011F00C9437
:102F7000C0178091B70380628093B7030E94B0109E
:102F80000C94D1170091D004003011F00C94D1179B
:102F900000913A04003011F00C94D11780E0809336
:102FA000FF0300910805013081E009F080E08F9374
:102FB00000915104033081E009F080E09F91892B5A
:102FC0008F9300913804033081E009F080E09F91F5
:102FD000892B8F93009138040D3081E009F080E057
:102FE0009F91892B8F9300913804073181E009F07C
:102FF00080E09F91892B8F93009138040B3781E0FB
:1030000009F080E09F91892B882311F40C945918C2
:1030100081E080932F075A924A92AA81BB818C91BA
:10302000A42DB52D8C9381E00E9485EF5A924A928F
:1030300084E0A42DB52D8C9381E00E9485EF5A92F7
:103040004A9283E0A42DB52D8C9381E00E9485EFF8
:103050000E9421DE269683E00E9481EFA881B9813B
:103060000C91013011F00C944A1881E08093D10446
:1030700084E08093000400914E04003011F00C9421
:1030800048188091B70380628093B7030E94B01004
:103090000C9459180091D104003011F00C94591877
:1030A00000913B04003011F00C94591880E080939B
:1030B00000040C947C185A924A9281E0A42DB52DFC
:1030C0008C9381E00E9485EF5A924A9284E0A42D6D
:1030D000B52D8C9381E00E9485EF5A924A9284E04C
:1030E000A42DB52D8C9381E00E9485EF0E9421DEF6
:1030F000269683E00E9481EF08950E948E29A1E226
:10310000B0E08C9187FB882780F9082F41E00427E5
:10311000ACE3B6E00C93A0E3B0E08C9183FB88278E
:1031200080F9082F41E00427ADE3B6E00C93A1E25B
:10313000B0E08C9183FB882780F9082F41E00427B9
:10314000AEE3B6E00C9381E080933A0700913A0732
:10315000033018F011F00C94F11BEAE3F7E0A190B2
:10316000BB24EAE8F0E0EA0DFB1DA0E1B0E00E941C
:1031700083F5003081E009F080E08F93AAE3B7E0A7
:10318000AD90BB24A8E3B6E0AA0DBB1D0C910130A5
:1031900081E009F080E09F918923882311F40C9449
:1031A000DA18EAE3F7E0FA93EA930E944A2C2296AF
:1031B0000C946C19EAE3F7E0A190BB24EAE8F0E094
:1031C000EA0DFB1DA0E1B0E00E9483F5013081E033
:1031D00009F080E08F93AAE3B7E0AD90BB24ABE3A6
:1031E000B6E0AA0DBB1D0C91013081E009F080E032
:1031F0009F9189238F93AAE3B7E0AD90BB24A8E306
:10320000B6E0AA0DBB1D0C91013081E009F080E011
:103210009F918923882311F40C941719EAE3F7E0AE
:10322000FA93EA930E944A2C22960C946C19EAE3D2
:10323000F7E0A190BB24EAE8F0E0EA0DFB1DA0E175
:10324000B0E00E9483F5023081E009F080E08F93C6
:10325000AAE3B7E0AD90BB24ABE3B6E0AA0DBB1D7B
:103260000C91013081E009F080E09F91892388234F
:1032700011F40C944419EAE3F7E0FA93EA930E94FC
:103280004A2C22960C946C1980E0AAE3B7E0AD902A
:10329000BB24A4EFB3E0AA0DBB1D8C9380E0AAE38E
:1032A000B7E0AD90BB24AFE3B4E0AA0DBB1D8C9397
:1032B00080E0AAE3B7E0AD90BB24A2E4B4E0AA0D9D
:1032C000BB1D8C9380E0AAE3B7E0AD90BB24A5E4DE
:1032D000B4E0AA0DBB1D8C93AAE3B7E0AD90BB246C
:1032E000A4EFB3E0AA0DBB1D0C91003011F00C94BB
:1032F000131AAAE3B7E0AD90BB24A4E2B4E0AA0C91
:10330000BB1CAA0DBB1D8D919C91AAE3B7E0AD90AB
:10331000BB24AEE1B4E0AA0CBB1CAA0DBB1D8D936F
:103320009C93AAE3B7E0AD90BB24A7EFB3E0AA0D4E
:10333000BB1D0C91003011F00C94131AAAE3B7E0F6
:10334000AD90BB24AAEFB3E0AA0DBB1D0C910030D9
:1033500011F00C94131A80E0AAE3B7E0AD90BB24FF
:10336000A1EFB3E0AA0DBB1D8C93AAE3B7E0AD902B
:10337000BB24ABE2B4E0AA0DBB1D0C91013011F0EF
:103380000C94E81980E0AAE3B7E0AD90BB24ABE26F
:10339000B4E0AA0DBB1D8C9383E0809385048091DB
:1033A0003A07809351048EEB80936B0483ED8093F6
:1033B0006C0482E580936D040E94F11280E0AAE320
:1033C000B7E0AD90BB24A1E3B4E0AA0DBB1D8C9384
:1033D00080E0AAE3B7E0AD90BB24A4E3B4E0AA0D7B
:1033E000BB1D8C93AAE3B7E0AD90BB24AEE2B4E082
:1033F000AA0DBB1D0C91013011F00C94131A80E042
:10340000AAE3B7E0AD90BB24AEE2B4E0AA0DBB1DC9
:103410008C9380E0AAE3B7E0AD90BB24ABE2B4E0CC
:10342000AA0DBB1D8C93AAE3B7E0AD90BB24AEE020
:10343000B6E0AA0DBB1D0C91003011F00C94701A6F
:10344000AAE3B7E0AD90BB24A7EFB3E0AA0DBB1D84
:103450000C91003011F00C94701AAAE3B7E0AD9013
:10346000BB24AAEFB3E0AA0DBB1D0C91003011F0F4
:103470000C94701A80E0AAE3B7E0AD90BB24A1EFF2
:10348000B3E0AA0DBB1D8C9380E0AAE3B7E0AD903A
:10349000BB24ABE2B4E0AA0DBB1D8C9380E0AAE391
:1034A000B7E0AD90BB24A4E3B4E0AA0DBB1D8C93A0
:1034B000AAE3B7E0AD90BB24A4E2B4E0AA0CBB1C25
:1034C000AA0DBB1D8D919C91AAE3B7E0AD90BB24E2
:1034D000AEE1B4E0AA0CBB1CAA0DBB1D8D939C935E
:1034E000EAE3F7E0A190BB24E2E4F0E0EA0DFB1D83
:1034F000A0E1B0E00E9483F5013011F00C94941A21
:10350000AAE3B7E0AD90BB24A4EFB3E0AA0DBB1DC6
:103510008C91AAE3B7E0AD90BB24A6E3B7E0AA0D77
:10352000BB1D8C930C94A61AAAE3B7E0AD90BB2404
:10353000A8E3B6E0AA0DBB1D8C91AAE3B7E0AD905D
:10354000BB24A6E3B7E0AA0DBB1D8C93AAE3B7E0AA
:10355000AD90BB24A6E3B7E0AA0DBB1D4C91AAE336
:10356000B7E0AD90BB24A0E3B7E0AA0DBB1D0C9162
:10357000041711F40C94851BAAE3B7E0AD90BB24AB
:10358000A6E3B7E0AA0DBB1D4C91AAE3B7E0AD904E
:10359000BB24A0E3B7E0AA0DBB1D0C91041718F0E3
:1035A00011F00C94D51A0C944F1BAAE3B7E00D91BF
:1035B000112748E450E00E948DF1A5E2B1E0A00F90
:1035C000B11F0E94A7F5082F003018F011F00C94DD
:1035D000EB1A0C94451B89E40E94FAF0AAE3B7E0C9
:1035E0000D91112748E450E00E948DF1A5E2B1E071
:1035F000A00FB11F0E94A7F5EA2FFB2F3297F040D2
:103600000FEFA881B9810E9459F5EDE5F6E0A88198
:10361000B9810E94AFF50FB689E4481A8827580A85
:1036200022960FBE11F40C94451BAAE3B7E00D914E
:10363000112748E450E00E948DF1A5E2B1E0A00F0F
:10364000B11F0E940EF0E0EEFDEE0E94DDF30E943D
:1036500097F1EDE5F6E0AAE3B7E00D91112748E414
:1036600050E00E948DF1A5E2B1E0A00FB11F0E94D1
:103670000EF00E9447F581E0AAE3B7E0AD90BB24CD
:10368000ACECB3E0AA0DBB1D8C9381E0AAE3B7E0DC
:10369000AD90BB24A0EDB3E0AA0DBB1D8C93EAE373
:1036A000F7E0A190BB24E2E4F0E0EA0DFB1DA0E10D
:1036B000B0E00E9483F5013011F00C94731BAAE373
:1036C000B7E0AD90BB24A4EFB3E0AA0DBB1D8C9175
:1036D000AAE3B7E0AD90BB24A0E3B7E0AA0DBB1D01
:1036E0008C930C94851BAAE3B7E0AD90BB24A8E3B0
:1036F000B6E0AA0DBB1D8C91AAE3B7E0AD90BB2448
:10370000A0E3B7E0AA0DBB1D8C93EAE3F7E0A1901C
:10371000BB24E1E3F0E0EA0DFB1DA0E1B0E00E9474
:1037200083F5003081E009F080E08F93AAE3B7E0F1
:10373000AD90BB24ACE0B4E0AA0DBB1D0C910030F1
:1037400081E009F080E09F91892B882311F40C948B
:10375000E91B0091F003003011F00C94E91BA9E67D
:10376000B4E08C9185FB16F40C94E91BAAE3B7E056
:10377000AD90BB24AEECB4E0AA0DBB1D0C910030A3
:1037800011F00C94E91BAAE3B7E0AD90BB24A4EFC1
:10379000B3E0AA0DBB1D0C91003011F00C94E91B95
:1037A0005A924A9280913A07A42DB52D8C9381E0CC
:1037B0000E9485EF5A924A9280E0A42DB52D8C93F9
:1037C00081E00E9485EF0E94BB2A249682E00E943D
:1037D00081EFAAE3B7E08C918F5F8C9310F40C9487
:1037E000A618A1E0B1E08C9183FB16F00C94601C4C
:1037F0000091F603013011F00C94351C00918B06FA
:10380000013011F00C94071C81E08093910481E059
:103810008093F80381E08093F20380E080930404B6
:1038200081E080933904A5EBB4E00E94BFF3A2E6E7
:10383000B6E00E94BFF35A924A9281E0A42DB52DC2
:103840008C9381E00E9485EF5A924A9281E0A42DE8
:10385000B52D8C9381E00E9485EF0E94BB2A2496AF
:1038600082E00E9481EF0C94601C80E08093F8035A
:103870000091F503003011F00C94601CE2E3F0E0DD
:10388000A0E1B0E00E9483F5003011F00C94601CC0
:103890005A924A9281E0A42DB52D8C9381E00E942A
:1038A00085EF5A924A9280E0A42DB52D8C9381E049
:1038B0000E9485EF0E94BB2A249682E00E9481EF3D
:1038C000A1E0B1E08C9181FB16F00C94CF1C00912B
:1038D000F703013011F00C94A41C00918B06013009
:1038E00011F00C94761C81E08093910481E0809328
:1038F000FB0381E08093F20380E08093040481E085
:1039000080933904A7EBB4E00E94BFF3A2E6B6E0CF
:103910000E94BFF35A924A9281E0A42DB52D8C9358
:1039200081E00E9485EF5A924A9281E0A42DB52D44
:103930008C9381E00E9485EF0E94BB2A249682E04E
:103940000E9481EF0C94CF1C80E08093FB030091D8
:10395000F503003011F00C94CF1CE2E3F0E0A0E19D
:10396000B0E00E9483F5003011F00C94CF1C5A9205
:103970004A9281E0A42DB52D8C9381E00E9485EFC1
:103980005A924A9280E0A42DB52D8C9381E00E943A
:1039900085EF0E94BB2A249682E00E9481EF40912D
:1039A000F50300913407041711F40C94061D40919F
:1039B000F50300913407041718F011F00C94E21C81
:1039C0000C94021D81E080933C0480E080933D04D0
:1039D00080E080933E0481E080934505A1E0B1E062
:1039E0008C9185FB16F00C94F81C81E080934605C1
:1039F000A1E0B1E08C9184FB16F00C94021D81E0F3
:103A0000809347058091F50380933407A5EFB3E0D9
:103A10008C9180FBA0E3B7E08C9187F98C93002711
:103A2000A0E3B7E08C9186FB0EF401E04427A0E30D
:103A3000B7E08C9187FB0EF44395041711F40C94B6
:103A4000621E00910F06013011F00C94B31D00911D
:103A5000F503013011F00C94541D00914004003026
:103A600011F00C94541D5A924A9281E0A42DB52D68
:103A70008C9381E00E9485EF5A924A9281E0A42DB6
:103A8000B52D8C9381E00E9485EF5A924A9281E095
:103A9000A42DB52D8C9381E00E9485EF0E9421DE3C
:103AA000269683E00E9481EF0091F503003081E0CB
:103AB00009F080E08F9300914004013081E009F02B
:103AC00080E09F91892B882311F40C94B31D5A92A6
:103AD0004A9280E0A42DB52D8C9381E00E9485EF61
:103AE0005A924A9281E0A42DB52D8C9381E00E94D8
:103AF00085EF5A924A9281E0A42DB52D8C9381E0F6
:103B00000E9485EF0E9421DE269683E00E9481EFCD
:103B100081E080935F06A9E1B5E08C9187FB16F008
:103B20000C94B31D5A924A9280E0A42DB52D8C932B
:103B300081E00E9485EF5A924A9281E0A42DB52D32
:103B40008C9381E00E9485EF5A924A9284E0A42DE2
:103B5000B52D8C9381E00E9485EF0E9421DE269690
:103B600083E00E9481EF0091F503013011F00C9485
:103B7000071E00914004003011F00C94071E0091C4
:103B80008706013011F00C94071E5A924A9281E088
:103B9000A42DB52D8C9381E00E9485EF5A924A9214
:103BA00081E0A42DB52D8C9381E00E9485EF5A927F
:103BB0004A9284E0A42DB52D8C9381E00E9485EF7C
:103BC0000E9421DE269683E00E9481EF5A924A925B
:103BD00080E0A42DB52D8C9381E00E9485EF5A9250
:103BE0004A9288E0A42DB52D8C9381E00E9485EF48
:103BF0005A924A9281E0A42DB52D8C9381E00E94C7
:103C000085EF0E9421DE269683E00E9481EF0091DD
:103C1000F503003081E009F080E08F9300914004CB
:103C2000013081E009F080E09F91892B882311F415
:103C30000C94621E00918706013011F00C94621EF4
:103C40005A924A9280E0A42DB52D8C9381E00E9477
:103C500085EF5A924A9281E0A42DB52D8C9381E094
:103C60000E9485EF5A924A9284E0A42DB52D8C9340
:103C700081E00E9485EF0E9421DE269683E00E946B
:103C800081EF5A924A9281E0A42DB52D8C9381E068
:103C90000E9485EF5A924A9288E0A42DB52D8C930C
:103CA00081E00E9485EF5A924A9281E0A42DB52DC1
:103CB0008C9381E00E9485EF0E9421DE269683E0AE
:103CC0000E9481EFA0E3B7E08C9187FBA0E3B7E00F
:103CD0008C9186F98C93A1E0B1E08C9185FB16F074
:103CE0000C94771FEFE8F0E0A0E1B0E00E9483F5CC
:103CF000013011F00C94F31E0091F503013011F026
:103D00000C94B01E00914304003011F00C94B01ECE
:103D1000AEEEB6E08C9187FB16F40C94B01E5A926E
:103D20004A9281E0A42DB52D8C9381E00E9485EF0D
:103D30005A924A9281E0A42DB52D8C9381E00E9485
:103D400085EF5A924A9282E0A42DB52D8C9381E0A2
:103D50000E9485EF0E9421DE269683E00E9481EF7B
:103D6000EDEAF0E0A0E1B0E00E9483F5013081E0EF
:103D700009F080E08F9300914304013081E009F065
:103D800080E09F9189238F930091F503003081E0BB
:103D900009F080E09F91892B882311F40C94F11E87
:103DA0005A924A9280E0A42DB52D8C9381E00E9416
:103DB00085EF5A924A9281E0A42DB52D8C9381E033
:103DC0000E9485EF5A924A9282E0A42DB52D8C93E1
:103DD00081E00E9485EF0E9421DE269683E00E940A
:103DE00081EF0C94771F0091F503013011F00C94D2
:103DF0002D1F00914304003011F00C942D1F0091F1
:103E0000F603003011F00C942D1FAEEEB6E08C914D
:103E100087FB16F40C942D1F5A924A9281E0A42D30
:103E2000B52D8C9381E00E9485EF5A924A9281E0F1
:103E3000A42DB52D8C9381E00E9485EF5A924A9271
:103E400082E0A42DB52D8C9381E00E9485EF0E9425
:103E500021DE269683E00E9481EFEDEAF0E0A0E10A
:103E6000B0E00E9483F5013081E009F080E08F939B
:103E700000914304013081E009F080E09F918923A3
:103E80008F930091F503003081E009F080E09F916D
:103E9000892B8F930091F603013081E009F080E0D7
:103EA0009F91892B882311F40C94771F5A924A9280
:103EB00080E0A42DB52D8C9381E00E9485EF5A926D
:103EC0004A9281E0A42DB52D8C9381E00E9485EF6C
:103ED0005A924A9282E0A42DB52D8C9381E00E94E3
:103EE00085EF0E9421DE269683E00E9481EFA1E00B
:103EF000B1E08C9184FB16F00C948320E0E9F0E0B3
:103F0000A0E1B0E00E9483F5013011F00C94FF1F96
:103F10000091F503013011F00C94BC1F0091430493
:103F2000003011F00C94BC1FAEEEB6E08C9187FB14
:103F300016F40C94BC1F5A924A9281E0A42DB52D20
:103F40008C9381E00E9485EF5A924A9281E0A42DE1
:103F5000B52D8C9381E00E9485EF5A924A9283E0BE
:103F6000A42DB52D8C9381E00E9485EF0E9421DE67
:103F7000269683E00E9481EFEEEAF0E0A0E1B0E057
:103F80000E9483F5013081E009F080E08F93009179
:103F90004304013081E009F080E09F9189238F93F1
:103FA0000091F503003081E009F080E09F91892BBA
:103FB000882311F40C94FD1F5A924A9280E0A42D9C
:103FC000B52D8C9381E00E9485EF5A924A9281E050
:103FD000A42DB52D8C9381E00E9485EF5A924A92D0
:103FE00083E0A42DB52D8C9381E00E9485EF0E9483
:103FF00021DE269683E00E9481EF0C9483200091BD
:10400000F503013011F00C94392000914304003085
:1040100011F00C9439200091F703003011F00C944A
:104020003920AEEEB6E08C9187FB16F40C94392063
:104030005A924A9281E0A42DB52D8C9381E00E9482
:1040400085EF5A924A9281E0A42DB52D8C9381E0A0
:104050000E9485EF5A924A9283E0A42DB52D8C934D
:1040600081E00E9485EF0E9421DE269683E00E9477
:1040700081EFEEEAF0E0A0E1B0E00E9483F50130CC
:1040800081E009F080E08F9300914304013081E0EA
:1040900009F080E09F9189238F930091F503003010
:1040A00081E009F080E09F91892B8F930091F703C5
:1040B000013081E009F080E09F91892B882311F481
:1040C0000C9483205A924A9280E0A42DB52D8C93B3
:1040D00081E00E9485EF5A924A9281E0A42DB52D8D
:1040E0008C9381E00E9485EF5A924A9283E0A42D3E
:1040F000B52D8C9381E00E9485EF0E9421DE2696EB
:1041000083E00E9481EFA1E0B1E08C9185FB16F085
:104110000C94F2200091F503013011F00C94C720AB
:1041200000918C06013011F00C94992081E080936D
:10413000920481E08093F90381E08093F30380E0AF
:104140008093050481E080933A04A3EBB4E00E94DD
:10415000BFF3A4E6B6E00E94BFF35A924A9282E00F
:10416000A42DB52D8C9381E00E9485EF5A924A923E
:1041700081E0A42DB52D8C9381E00E9485EF0E94F3
:10418000BB2A249682E00E9481EF0C94F22080E00A
:104190008093F9030091F603003011F00C94F220A3
:1041A000E3E3F0E0A0E1B0E00E9483F5003011F01D
:1041B0000C94F2205A924A9282E0A42DB52D8C9351
:1041C00081E00E9485EF5A924A9280E0A42DB52D9D
:1041D0008C9381E00E9485EF0E94BB2A249682E0A6
:1041E0000E9481EFA1E0B1E08C9180FB16F00C946D
:1041F00061210091F703013011F00C9436210091F8
:104200008C06013011F00C94082181E08093920417
:1042100081E08093FC0381E08093F30380E080934E
:10422000050481E080933A04A7EBB4E00E94BFF359
:10423000A4E6B6E00E94BFF35A924A9282E0A42D0F
:10424000B52D8C9381E00E9485EF5A924A9281E0CD
:10425000A42DB52D8C9381E00E9485EF0E94BB2A8E
:10426000249682E00E9481EF0C9461210091F60374
:10427000003011F00C945E21E3E3F0E0A0E1B0E047
:104280000E9483F5003011F00C945E215A924A92FC
:1042900082E0A42DB52D8C9381E00E9485EF5A9287
:1042A0004A9280E0A42DB52D8C9381E00E9485EF89
:1042B0000E94BB2A249682E00E9481EF80E08093D6
:1042C000FC034091F60300913507041711F40C9498
:1042D00098214091F60300913507041718F011F06A
:1042E0000C9474210C94942180E080933C0481E030
:1042F00080933D0480E080933E0481E080934605F6
:10430000A1E0B1E08C9183FB16F00C948A2181E04E
:1043100080934505A1E0B1E08C9182FB16F00C94EE
:10432000942181E0809347058091F60380933507BF
:10433000A6EFB3E08C9180FBA0E3B7E08C9185F908
:104340008C930027A0E3B7E08C9184FB0EF401E08E
:104350004427A0E3B7E08C9185FB0EF44395041746
:1043600011F40C94E72200911006013011F00C9426
:1043700038220091F603013011F00C94E6210091EF
:104380004104003011F00C94E6215A924A9281E0E7
:10439000A42DB52D8C9381E00E9485EF5A924A920C
:1043A00082E0A42DB52D8C9381E00E9485EF5A9276
:1043B0004A9282E0A42DB52D8C9381E00E9485EF76
:1043C0000E9421DE269683E00E9481EF0091F60391
:1043D000003011F00C9438225A924A9280E0A42DB9
:1043E000B52D8C9381E00E9485EF5A924A9282E02B
:1043F000A42DB52D8C9381E00E9485EF5A924A92AC
:1044000082E0A42DB52D8C9381E00E9485EF0E945F
:1044100021DE269683E00E9481EF81E08093600692
:10442000A9E1B5E08C9187FB16F00C9438225A92E2
:104430004A9280E0A42DB52D8C9381E00E9485EFF7
:104440005A924A9282E0A42DB52D8C9381E00E946D
:1044500085EF5A924A9284E0A42DB52D8C9381E089
:104460000E9485EF0E9421DE269683E00E9481EF64
:104470000091F603013011F00C948C22009141045C
:10448000003011F00C948C2200918806013011F05C
:104490000C948C225A924A9281E0A42DB52D8C93D3
:1044A00081E00E9485EF5A924A9282E0A42DB52DB8
:1044B0008C9381E00E9485EF5A924A9284E0A42D69
:1044C000B52D8C9381E00E9485EF0E9421DE269617
:1044D00083E00E9481EF5A924A9280E0A42DB52D8C
:1044E0008C9381E00E9485EF5A924A9288E0A42D35
:1044F000B52D8C9381E00E9485EF5A924A9282E01A
:10450000A42DB52D8C9381E00E9485EF0E9421DEC1
:10451000269683E00E9481EF0091F603003081E04F
:1045200009F080E08F9300914104013081E009F0AF
:1045300080E09F91892B882311F40C94E72200914D
:104540008806013011F00C94E7225A924A9280E0DA
:10455000A42DB52D8C9381E00E9485EF5A924A924A
:1045600082E0A42DB52D8C9381E00E9485EF5A92B4
:104570004A9284E0A42DB52D8C9381E00E9485EFB2
:104580000E9421DE269683E00E9481EF5A924A9291
:1045900081E0A42DB52D8C9381E00E9485EF5A9285
:1045A0004A9288E0A42DB52D8C9381E00E9485EF7E
:1045B0005A924A9282E0A42DB52D8C9381E00E94FC
:1045C00085EF0E9421DE269683E00E9481EFA0E322
:1045D000B7E08C9185FBA0E3B7E08C9184F98C93D4
:1045E000A1E0B1E08C9183FB16F00C94FC23EEE883
:1045F000F0E0A0E1B0E00E9483F5013011F00C94EE
:1046000078230091F603013011F00C9435230091CA
:104610004404003011F00C943523AEEEB6E08C91DA
:1046200087FB16F40C9435235A924A9281E0A42D0C
:10463000B52D8C9381E00E9485EF5A924A9282E0D8
:10464000A42DB52D8C9381E00E9485EF5A924A9259
:1046500081E0A42DB52D8C9381E00E9485EF0E940E
:1046600021DE269683E00E9481EFECEAF0E0A0E1F3
:10467000B0E00E9483F5013081E009F080E08F9383
:1046800000914404013081E009F080E09F9189238A
:104690008F930091F603003081E009F080E09F9154
:1046A000892B882311F40C9476235A924A9280E045
:1046B000A42DB52D8C9381E00E9485EF5A924A92E9
:1046C00082E0A42DB52D8C9381E00E9485EF5A9253
:1046D0004A9281E0A42DB52D8C9381E00E9485EF54
:1046E0000E9421DE269683E00E9481EF0C94FC2339
:1046F0000091F603013011F00C94B22300914404B0
:10470000003011F00C94B2230091F503003011F049
:104710000C94B223AEEEB6E08C9187FB16F40C94A9
:10472000B2235A924A9281E0A42DB52D8C9381E058
:104730000E9485EF5A924A9282E0A42DB52D8C9367
:1047400081E00E9485EF5A924A9281E0A42DB52D16
:104750008C9381E00E9485EF0E9421DE269683E003
:104760000E9481EFECEAF0E0A0E1B0E00E9483F566
:10477000013081E009F080E08F9300914404013022
:1047800081E009F080E09F9189238F930091F603E7
:10479000003081E009F080E09F91892B8F93009198
:1047A000F503013081E009F080E09F91892B882397
:1047B00011F40C94FC235A924A9280E0A42DB52D5A
:1047C0008C9381E00E9485EF5A924A9282E0A42D58
:1047D000B52D8C9381E00E9485EF5A924A9281E038
:1047E000A42DB52D8C9381E00E9485EF0E9421DEDF
:1047F000269683E00E9481EFA1E0B1E08C9182FBDC
:1048000016F00C940825E0E9F0E0A0E1B0E00E9489
:1048100083F5013011F00C9484240091F6030130EB
:1048200011F00C94412400914404003011F00C94D8
:104830004124AEEEB6E08C9187FB16F40C94412433
:104840005A924A9281E0A42DB52D8C9381E00E946A
:1048500085EF5A924A9282E0A42DB52D8C9381E087
:104860000E9485EF5A924A9283E0A42DB52D8C9335
:1048700081E00E9485EF0E9421DE269683E00E945F
:1048800081EFEEEAF0E0A0E1B0E00E9483F50130B4
:1048900081E009F080E08F9300914404013081E0D1
:1048A00009F080E09F9189238F930091F6030030F7
:1048B00081E009F080E09F91892B882311F40C940A
:1048C00082245A924A9280E0A42DB52D8C9381E0E7
:1048D0000E9485EF5A924A9282E0A42DB52D8C93C6
:1048E00081E00E9485EF5A924A9283E0A42DB52D73
:1048F0008C9381E00E9485EF0E9421DE269683E062
:104900000E9481EF0C9408250091F603013011F00C
:104910000C94BE2400914404003011F00C94BE2489
:104920000091F703003011F00C94BE24AEEEB6E017
:104930008C9187FB16F40C94BE245A924A9281E023
:10494000A42DB52D8C9381E00E9485EF5A924A9256
:1049500082E0A42DB52D8C9381E00E9485EF5A92C0
:104960004A9283E0A42DB52D8C9381E00E9485EFBF
:104970000E9421DE269683E00E9481EFEEEAF0E0BD
:10498000A0E1B0E00E9483F5013081E009F080E011
:104990008F9300914404013081E009F080E09F9101
:1049A00089238F930091F603003081E009F080E0C5
:1049B0009F91892B8F930091F703013081E009F0DB
:1049C00080E09F91892B882311F40C9408255A923A
:1049D0004A9280E0A42DB52D8C9381E00E9485EF52
:1049E0005A924A9282E0A42DB52D8C9381E00E94C8
:1049F00085EF5A924A9283E0A42DB52D8C9381E0E5
:104A00000E9485EF0E9421DE269683E00E9481EFBE
:104A1000A1E0B1E08C9184FB16F00C947725009115
:104A2000F503013011F00C944C2500918D060130F6
:104A300011F00C941E2581E08093930481E0809313
:104A4000FA0381E08093F40380E08093060481E020
:104A500080933B04A3EBB4E00E94BFF3A6E6B6E06C
:104A60000E94BFF35A924A9283E0A42DB52D8C93F5
:104A700081E00E9485EF5A924A9281E0A42DB52DE3
:104A80008C9381E00E9485EF0E94BB2A249682E0ED
:104A90000E9481EF0C94772580E08093FA030091C7
:104AA000F703003011F00C947725E4E3F0E0A0E187
:104AB000B0E00E9483F5003011F00C9477255A92F3
:104AC0004A9283E0A42DB52D8C9381E00E9485EF5E
:104AD0005A924A9280E0A42DB52D8C9381E00E94D9
:104AE00085EF0E94BB2A249682E00E9481EFA1E01C
:104AF000B1E08C9182FB16F00C94E6250091F60350
:104B0000013011F00C94BB2500918D06013011F09D
:104B10000C948D2581E08093930481E08093FD03C4
:104B200081E08093F40380E08093060481E0809329
:104B30003B04A5EBB4E00E94BFF3A6E6B6E00E94FA
:104B4000BFF35A924A9283E0A42DB52D8C9381E055
:104B50000E9485EF5A924A9281E0A42DB52D8C9344
:104B600081E00E9485EF0E94BB2A249682E00E9489
:104B700081EF0C94E62580E08093FD030091F7031C
:104B8000003011F00C94E625E4E3F0E0A0E1B0E0A1
:104B90000E9483F5003011F00C94E6255A924A9257
:104BA00083E0A42DB52D8C9381E00E9485EF5A926D
:104BB0004A9280E0A42DB52D8C9381E00E9485EF70
:104BC0000E94BB2A249682E00E9481EF4091F70365
:104BD00000913607041711F40C941D264091F70339
:104BE00000913607041718F011F00C94F9250C9475
:104BF000192680E080933C0480E080933D0481E0AE
:104C000080933E0481E080934705A1E0B1E08C9160
:104C100081FB16F00C940F2681E080934505A1E0FE
:104C2000B1E08C9180FB16F00C94192681E0809302
:104C300046058091F70380933607A7EFB3E08C9188
:104C400080FBA0E3B7E08C9183F98C930027A0E36D
:104C5000B7E08C9182FB0EF401E04427A0E3B7E0BB
:104C60008C9183FB0EF44395041711F40C946C277C
:104C700000911106013011F00C94BD260091F7034C
:104C8000013011F00C946B2600914204003011F0B9
:104C90000C946B265A924A9281E0A42DB52D8C93E8
:104CA00081E00E9485EF5A924A9283E0A42DB52DAF
:104CB0008C9381E00E9485EF5A924A9283E0A42D62
:104CC000B52D8C9381E00E9485EF0E9421DE26960F
:104CD00083E00E9481EF0091F703003011F00C9403
:104CE000BD265A924A9280E0A42DB52D8C9381E086
:104CF0000E9485EF5A924A9283E0A42DB52D8C93A1
:104D000081E00E9485EF5A924A9283E0A42DB52D4E
:104D10008C9381E00E9485EF0E9421DE269683E03D
:104D20000E9481EF81E080936106A9E1B5E08C915A
:104D300087FB16F00C94BD265A924A9280E0A42D6F
:104D4000B52D8C9381E00E9485EF5A924A9283E0C0
:104D5000A42DB52D8C9381E00E9485EF5A924A9242
:104D600084E0A42DB52D8C9381E00E9485EF0E94F4
:104D700021DE269683E00E9481EF0091F703013047
:104D800011F00C94112700914204003011F00C94A2
:104D9000112700918906013011F00C9411275A92C5
:104DA0004A9281E0A42DB52D8C9381E00E9485EF7D
:104DB0005A924A9283E0A42DB52D8C9381E00E94F3
:104DC00085EF5A924A9284E0A42DB52D8C9381E010
:104DD0000E9485EF0E9421DE269683E00E9481EFEB
:104DE0005A924A9280E0A42DB52D8C9381E00E94C6
:104DF00085EF5A924A9288E0A42DB52D8C9381E0DC
:104E00000E9485EF5A924A9283E0A42DB52D8C938F
:104E100081E00E9485EF0E9421DE269683E00E94B9
:104E200081EF0091F703003081E009F080E08F937B
:104E300000914204013081E009F080E09F91892BCC
:104E4000882311F40C946C2700918906013011F02D
:104E50000C946C275A924A9280E0A42DB52D8C9325
:104E600081E00E9485EF5A924A9283E0A42DB52DED
:104E70008C9381E00E9485EF5A924A9284E0A42D9F
:104E8000B52D8C9381E00E9485EF0E9421DE26964D
:104E900083E00E9481EF5A924A9281E0A42DB52DC1
:104EA0008C9381E00E9485EF5A924A9288E0A42D6B
:104EB000B52D8C9381E00E9485EF5A924A9283E04F
:104EC000A42DB52D8C9381E00E9485EF0E9421DEF8
:104ED000269683E00E9481EFA0E3B7E08C9183FBEC
:104EE000A0E3B7E08C9182F98C93A1E0B1E08C91C2
:104EF00081FB16F00C948128EEE8F0E0A0E1B0E030
:104F00000E9483F5013011F00C94FD270091F70306
:104F1000013011F00C94BA2700914504003011F0D3
:104F20000C94BA27AEEEB6E08C9187FB16F40C9485
:104F3000BA275A924A9281E0A42DB52D8C9381E034
:104F40000E9485EF5A924A9283E0A42DB52D8C934E
:104F500081E00E9485EF5A924A9281E0A42DB52DFE
:104F60008C9381E00E9485EF0E9421DE269683E0EB
:104F70000E9481EFECEAF0E0A0E1B0E00E9483F54E
:104F8000013081E009F080E08F9300914504013009
:104F900081E009F080E09F9189238F930091F703CE
:104FA000003081E009F080E09F91892B882311F483
:104FB0000C94FB275A924A9280E0A42DB52D8C9335
:104FC00081E00E9485EF5A924A9283E0A42DB52D8C
:104FD0008C9381E00E9485EF5A924A9281E0A42D41
:104FE000B52D8C9381E00E9485EF0E9421DE2696EC
:104FF00083E00E9481EF0C9481280091F703013037
:1050000011F00C94372800914504003011F00C94F5
:1050100037280091F503003011F00C943728AEEEDC
:10502000B6E08C9187FB16F40C9437285A924A927A
:1050300081E0A42DB52D8C9381E00E9485EF5A92DA
:105040004A9283E0A42DB52D8C9381E00E9485EFD8
:105050005A924A9281E0A42DB52D8C9381E00E9452
:1050600085EF0E9421DE269683E00E9481EFECEA24
:10507000F0E0A0E1B0E00E9483F5013081E009F0AA
:1050800080E08F9300914504013081E009F080E0D9
:105090009F9189238F930091F703003081E009F0FD
:1050A00080E09F91892B8F930091F503013081E07F
:1050B00009F080E09F91892B882311F40C948128BA
:1050C0005A924A9280E0A42DB52D8C9381E00E94E3
:1050D00085EF5A924A9283E0A42DB52D8C9381E0FE
:1050E0000E9485EF5A924A9281E0A42DB52D8C93AF
:1050F00081E00E9485EF0E9421DE269683E00E94D7
:1051000081EFA1E0B1E08C9180FB16F00C948D2929
:10511000EFE8F0E0A0E1B0E00E9483F5013011F08B
:105120000C9409290091F703013011F00C94C62862
:1051300000914504003011F00C94C628AEEEB6E0A4
:105140008C9187FB16F40C94C6285A924A9281E0FF
:10515000A42DB52D8C9381E00E9485EF5A924A923E
:1051600083E0A42DB52D8C9381E00E9485EF5A92A7
:105170004A9282E0A42DB52D8C9381E00E9485EFA8
:105180000E9421DE269683E00E9481EFEDEAF0E0A6
:10519000A0E1B0E00E9483F5013081E009F080E0F9
:1051A0008F9300914504013081E009F080E09F91E8
:1051B00089238F930091F703003081E009F080E0AC
:1051C0009F91892B882311F40C9407295A924A92B3
:1051D00080E0A42DB52D8C9381E00E9485EF5A923A
:1051E0004A9283E0A42DB52D8C9381E00E9485EF37
:1051F0005A924A9282E0A42DB52D8C9381E00E94B0
:1052000085EF0E9421DE269683E00E9481EF0C94B8
:105210008D290091F703013011F00C94432900917E
:105220004504003011F00C9443290091F60300303E
:1052300011F00C944329AEEEB6E08C9187FB16F486
:105240000C9443295A924A9281E0A42DB52D8C9357
:1052500081E00E9485EF5A924A9283E0A42DB52DF9
:105260008C9381E00E9485EF5A924A9282E0A42DAD
:10527000B52D8C9381E00E9485EF0E9421DE269659
:1052800083E00E9481EFEDEAF0E0A0E1B0E00E944F
:1052900083F5013081E009F080E08F9300914504AF
:1052A000013081E009F080E09F9189238F93009184
:1052B000F703003081E009F080E09F91892B8F9304
:1052C0000091F603013081E009F080E09F91892B85
:1052D000882311F40C948D295A924A9280E0A42DCF
:1052E000B52D8C9381E00E9485EF5A924A9283E01B
:1052F000A42DB52D8C9381E00E9485EF5A924A929D
:1053000082E0A42DB52D8C9381E00E9485EF0E9450
:1053100021DE269683E00E9481EF089581E00E94BD
:10532000FAF082E00E94FAF082E00E94FAF0A9E628
:10533000B4E08C9185FB81E00EF080E08F93A9E6CC
:10534000B4E08C9184FB81E00EF080E09F91892B8A
:10535000882311F40C94F02981E0809332060091A7
:105360003206033018F011F00C94EE290091320649
:1053700043E0040FAC81BD810C93A2E3B6E0AD9095
:10538000BB24A2E2B6E0AA0DBB1D0C91013011F0C6
:105390000C94E629AC81BD818C91A1E2B0E00E9421
:1053A000D7F30E94CDF30C900822689409F4E89496
:1053B000882780F9082F41E00427A2E3B6E0AD90EA
:1053C000BB24A8E3B6E0AA0DBB1D0C93A2E3B6E094
:1053D0008C918F5F8C9310F40C94AF290C94B52AA8
:1053E00081E08093320600913206033018F011F00C
:1053F0000C94B52A0091320643E0040FAC81BD81C4
:105400000C93A2E3B6E0AD90BB24A2E2B6E0AA0DF5
:10541000BB1D0C91013011F00C94AD2AAC81BD8103
:105420008C91A1E2B0E00E94D7F30E94CDF30C90E2
:105430000822689409F4E89416F40C94A32A81E0F5
:10544000A2E3B6E0AD90BB24A8E3B6E0AA0DBB1D75
:105450008C93A2E3B6E0AD90BB24A5E2B6E0AA0D22
:10546000BB1D0C91013081E009F080E08F93A2E335
:10547000B6E0AD90BB24ABE4B4E0AA0DBB1D0C912B
:10548000003081E009F080E09F9189238F93A2E3AF
:10549000B6E0AD90BB24AEE0B6E0AA0DBB1D0C910A
:1054A000013081E009F080E09F918923882311F485
:1054B0000C94762A09E110E0A2E3B6E0AD90BB249B
:1054C000A7E2B6E0AA0CBB1CAA0DBB1D4D915C91D6
:1054D000040F151FA881B9810D931C93A881B98170
:1054E0008D919C910E94EBF00C947A2A89E190E0D6
:1054F0000E94EBF0AC81BD818C91A1E2B0E00E94F2
:10550000D7F30E94CDF30C900822689409F4E89434
:1055100016F40C94972A81E0A2E3B6E0AD90BB2488
:10552000A8E3B6E0AA0DBB1D8C930C94A12A80E0E1
:10553000A2E3B6E0AD90BB24A8E3B6E0AA0DBB1D84
:105540008C930C94AD2A80E0A2E3B6E0AD90BB242E
:10555000A8E3B6E0AA0DBB1D8C93A2E3B6E08C9144
:105560008F5F8C9310F40C94F32985E0481A8827F8
:10557000580A26960895A881B9810C91013011F03E
:105580000C943E2B80E0AA81BB81AD90BB24A9E0A6
:10559000B4E0AA0DBB1D8C93EA81FB81A190BB24D2
:1055A000EAE3F0E0EA0DFB1DA0E1B0E00E9483F524
:1055B000013011F00C94132BAA81BB81AD90BB2458
:1055C000ACE0B4E0AA0DBB1D0C910E3F11F40C949D
:1055D000F52A80E0AA81BB81AD90BB24A0E0B4E0B5
:1055E000AA0DBB1D8C930C94112BAA81BB810C912D
:1055F000013011F00C94012B88E0809301040C948D
:10560000112B023011F00C940A2B80E180930204DC
:105610000C94112B033011F00C94112B80E2809329
:1056200003040C943C2BAA81BB81AD90BB24ACE05D
:10563000B4E0AA0DBB1D0C910E3F11F40C943C2B51
:10564000AA81BB810C91013011F00C942C2B88E0C5
:10565000809301040C943C2B023011F00C94352BF8
:1056600080E1809302040C943C2B033011F00C94E5
:105670003C2B80E2809303040C940C2CAA81BB8108
:10568000AD90BB24ABE7B6E0AA0DBB1D0C9100307A
:1056900011F00C948F2BAA81BB81AD90BB24A5E0A7
:1056A000B5E0AA0DBB1D0C91013081E009F080E04E
:1056B0008F93AA81BB81AD90BB24A2E0B5E0AA0D77
:1056C000BB1D0C91013081E009F080E09F91892B96
:1056D000882311F40C948F2BAA81BB81AD90BB243D
:1056E000ACE0B4E0AA0DBB1D8C91AA81BB81AD904A
:1056F000BB24A9E0B4E0AA0DBB1D8C935A924A9238
:10570000AC81BD818C91A42DB52D8C9381E00E943C
:1057100085EF0E940F2C229681E00E9481EFA9E67E
:10572000B4E08C9185FB16F40C940C2CAEEEB6E034
:105730008C9186FB16F40C940C2CAA81BB81AD9045
:10574000BB24AEEEB6E0AA0DBB1D0C91003011F0EB
:105750000C940C2CAA81BB81AD90BB24A6E8B6E0CA
:10576000AA0DBB1D0C91003011F00C940C2CAA81D9
:10577000BB81AD90BB24ACE0B4E0AA0DBB1D0C9185
:105780000F3F10F00C940C2CAA81BB81AD90BB2470
:10579000ACE0B4E0AA0DBB1D0C91003011F00C94EC
:1057A000DB2B80E0AA81BB81AD90BB24A9E0B4E0F3
:1057B000AA0DBB1D8C93AA81BB81AD90BB24ACE02C
:1057C000B4E0AA0DBB1D4C91AA81BB81AD90BB2456
:1057D000A9E0B4E0AA0DBB1D0C91041710F40C94C1
:1057E0000C2C80E0AA81BB81AD90BB24A9E0B4E081
:1057F000AA0DBB1D8C935A924A92AC81BD818C91AB
:10580000A42DB52D8C9381E00E9485EF0E940F2C72
:10581000229681E00E9481EF0E94B0100895E881F5
:10582000F981A190BB24EAE3F0E0EA0DFB1DA0E1C1
:10583000B0E00E9483F5013011F00C943D2CA8815A
:10584000B9810C91013011F00C942B2C88E08093DD
:1058500001040C943B2C023011F00C94342C80E1A8
:10586000809302040C943B2C033011F00C943B2CDD
:1058700080E2809303040C94472C80E0A881B981D6
:10588000AD90BB24A0E0B4E0AA0DBB1D8C930E9498
:10589000B010089581E0A881B981AD90BB24A4EF38
:1058A000B3E0AA0DBB1D8C935A924A92AA81BB8188
:1058B0008C91A42DB52D8C9381E00E9485EF5A9296
:1058C0004A9281E0A42DB52D8C9381E00E9485EF52
:1058D0000E94BB2A249682E00E9481EFA881B981B0
:1058E000AD90BB24AEE0B6E0AA0DBB1D0C9101301B
:1058F00011F00C94A52C81E0A881B981AD90BB2456
:10590000A1EFB3E0AA0DBB1D8C9380E0A881B98103
:10591000AD90BB24A3E0B4E0AA0DBB1D8C9381E045
:10592000A881B981AD90BB24A8E3B4E0AA0DBB1D4A
:105930008C93A881B981AD90BB24A0E6B6E0AA0CF7
:10594000BB1CAA0DBB1D0E94BFF3089500912C043F
:10595000013081E009F080E08F9300912F04013045
:1059600081E009F080E09F91892B882311F40C9449
:10597000C02C80E08093FE030E94B0100C945B2D3D
:10598000A2EFB3E08C9180FBA9E1B5E08C9185F9A1
:105990008C930027A9E1B5E08C9182FB0EF401E025
:1059A0004427A9E1B5E08C9185FB0EF443950417DB
:1059B00011F40C943A2D0091F203013011F00C9483
:1059C000F52C0091F503013011F00C94EA2C81E0E4
:1059D0008093350480E080930A0481E080939104F1
:1059E00081E08093FE030E94B01000910F0600300A
:1059F00011F00C94142D0091F203003011F00C946E
:105A0000142D80E08093390480E08093FE030E948F
:105A1000B010A9E1B5E08C9185FBA9E1B5E08C91CE
:105A200082F98C930C945B2D00913904013011F0B4
:105A30000C943A2D0091F203003011F00C943A2DA1
:105A400081E08093FE030E94B0100091CF040030EB
:105A500011F00C943A2D5A924A9281E0A42DB52D62
:105A60008C9381E00E9485EF0E94C82E229681E0EF
:105A70000E9481EFA9E1B5E08C9185FBA9E1B5E039
:105A80008C9182F98C9300913B07013011F00C94BA
:105A90005B2D80E080933B075A924A9281E0A42DCF
:105AA000B52D8C9381E00E9485EF0E943BE4229605
:105AB00081E00E9481EF089500912D04013081E082
:105AC00009F080E08F9300913004013081E009F00B
:105AD00080E09F91892B882311F40C94762D80E02F
:105AE0008093FF030E94B0100C94112EA3EFB3E03B
:105AF0008C9180FBA9E1B5E08C9184F98C9300270F
:105B0000A9E1B5E08C9181FB0EF401E04427A9E105
:105B1000B5E08C9184FB0EF44395041711F40C94BA
:105B2000F02D0091F303013011F00C94AB2D81E0C6
:105B3000809392040091F603013011F00C94A32D90
:105B400081E08093360480E080930B0482E08093B0
:105B5000FF030E94B01000911006003011F00C9469
:105B6000CA2D0091F303003011F00C94CA2D80E08F
:105B700080933A0480E08093FF030E94B010A9E173
:105B8000B5E08C9184FBA9E1B5E08C9181F98C930F
:105B90000C94112E00913A04013011F00C94F02D68
:105BA0000091F303003011F00C94F02D82E080930B
:105BB000FF030E94B0100091D004003011F00C944B
:105BC000F02D5A924A9282E0A42DB52D8C9381E05B
:105BD0000E9485EF0E94C82E229681E00E9481EFEC
:105BE000A9E1B5E08C9184FBA9E1B5E08C9181F944
:105BF0008C9300913C07013011F00C94112E80E041
:105C000080933C075A924A9282E0A42DB52D8C9342
:105C100081E00E9485EF0E943BE4229681E00E9491
:105C200081EF089500912E04013081E009F080E0B9
:105C30008F9300913104013081E009F080E09F9161
:105C4000892B882311F40C942C2E80E0809300047F
:105C50000E94B0100C94C72EA4EFB3E08C9180FB8F
:105C6000A9E1B5E08C9183F98C930027A9E1B5E017
:105C70008C9180FB0EF401E04427A9E1B5E08C9102
:105C800083FB0EF44395041711F40C94A62E009197
:105C9000F403013011F00C94612E81E080939304A1
:105CA0000091F703013011F00C94592E81E080939C
:105CB000370480E080930C0484E0809300040E9409
:105CC000B01000911106003011F00C94802E00915C
:105CD000F403003011F00C94802E80E080933B049C
:105CE00080E0809300040E94B010A9E1B5E08C919F
:105CF00083FBA9E1B5E08C9180F98C930C94C72EBD
:105D000000913B04013011F00C94A62E0091F40395
:105D1000003011F00C94A62E84E0809300040E94C1
:105D2000B0100091D104003011F00C94A62E5A92BC
:105D30004A9283E0A42DB52D8C9381E00E9485EFDB
:105D40000E94C82E229681E00E9481EFA9E1B5E071
:105D50008C9183FBA9E1B5E08C9180F98C93009143
:105D60003D07013011F00C94C72E80E080933D0771
:105D70005A924A9283E0A42DB52D8C9381E00E9423
:105D800085EF0E943BE4229681E00E9481EF089516
:105D9000A881B9810C91013011F00C94E02E809112
:105DA00030078D7F8093300780913007816080932A
:105DB000300780913E07806880933E070C94082F3F
:105DC000023011F00C94F52E8091300782608093A0
:105DD0003007809130078E7F8093300780913E0797
:105DE000806880933E070C94082F033011F00C94C8
:105DF000082F8091300782608093300780913007B0
:105E000081608093300780913E078F7780933E07B3
:105E100000910F06003011F00C94172FA0E3B7E0AB
:105E20008C9181FB16F00C94172F0E94A62C0091E8
:105E30001006003011F00C94262FA0E3B7E08C91EF
:105E400080FB16F00C94262F0E945C2D0091110609
:105E5000003011F00C94352FAEE3B7E08C9187FB46
:105E600016F00C94352F0E94122E809130078D7FF2
:105E700080933007809130078E7F80933007809128
:105E80003E078F7780933E07089582E00E94FAF0E4
:105E900082E00E94FAF081E00E94FAF081E00E9424
:105EA000FAF05A924A9281E0A42DB52D8C9381E0AC
:105EB0000E9485EF5A924A9285E0A42DB52D8C93CD
:105EC00081E00E9485EF5A924A9281E0A42DB52D7F
:105ED0008C9381E00E9485EF0E9421DE269683E06C
:105EE0000E9481EF5A924A9280E0A42DB52D8C93A6
:105EF00081E00E9485EF5A924A9285E0A42DB52D4B
:105F00008C9381E00E9485EF5A924A9282E0A42D00
:105F1000B52D8C9381E00E9485EF0E9421DE2696AC
:105F200083E00E9481EF5A924A9280E0A42DB52D21
:105F30008C9381E00E9485EF5A924A9285E0A42DCD
:105F4000B52D8C9381E00E9485EF5A924A9283E0AE
:105F5000A42DB52D8C9381E00E9485EF0E9421DE57
:105F6000269683E00E9481EF00910905003011F030
:105F70000C94BF2F82E0809345050C94B33381E0ED
:105F8000AA81BB818C93AA81BB810C91033018F04C
:105F900011F00C94A63380E0A881B9818C93AA817A
:105FA000BB810C91013011F00C94DC2F81E0A881B1
:105FB000B9818C930C94FC2F023011F00C94ED2FCE
:105FC000A1E0B1E08C9183FB16F00C94EB2F81E003
:105FD000A881B9818C930C94FC2F033011F00C94A0
:105FE000FC2FA1E0B1E08C9181FB16F00C94FC2F0A
:105FF00081E0A881B9818C93AA81BB81AD90BB243B
:10600000ABE3B4E0AA0DBB1D0C91013011F00C9470
:106010009E33A9E6B4E08C9185FB16F40C949E3374
:10602000A881B9810C91013011F00C949E335A92E1
:106030004A9281E0A42DB52D8C9381E00E9485EFDA
:106040005A924A9285E0A42DB52D8C9381E00E944E
:1060500085EF5A924A9281E0A42DB52D8C9381E070
:106060000E9485EF0E9421DE269683E00E9481EF48
:1060700080916904806180936904AA81BB810C913D
:10608000013011F00C947E30E9E0F5E0A190BB24E2
:10609000ECECF4E0AA0CBB1CEA0DFB1DAE81BF8149
:1060A0000E9485F5E9E0F5E0A190BB24ECEEF2E07A
:1060B000AA0CBB1CEA0DFB1DA3EDB4E00E9485F504
:1060C000E9E0F5E0A190BB24E8E2F3E0AA0CBB1CF8
:1060D000EA0DFB1DA5EDB4E00E9485F5E9E0F5E0D1
:1060E000A190BB24ECEBF5E0AA0CBB1CEA0DFB1D58
:1060F000A7EDB4E00E9485F50C94B830023011F0A1
:106100000C949C30EEEDF4E0AE81BF810E9485F5E9
:10611000EEEFF2E0A3EDB4E00E9485F5EAE3F3E0F0
:10612000A5EDB4E00E9485F5EEECF5E0A7EDB4E056
:106130000E9485F50C94B830033011F00C94B830FF
:10614000E0EEF4E0AE81BF810E9485F5E0E0F3E08F
:10615000A3EDB4E00E9485F5ECE3F3E0A5EDB4E037
:106160000E9485F5E0EDF5E0A7EDB4E00E9485F52D
:10617000AE81BF810D911C914AE050E00E94C5EFB5
:10618000AE81BF814D935C9381E090E0AC81BD8195
:106190008D939C93AC81BD810D911C910A3050E090
:1061A00015071CF011F00C940E31AE81BF818D915A
:1061B0009C910E94EBF00E947D185A924A92AC8109
:1061C000BD818C91A42DB52D8C9381E00E9485EF2B
:1061D0000E94C82E229681E00E9481EF0091F50373
:1061E000013011F00C94F6300C94B333A1E0B1E01F
:1061F0008C9185FB16F00C94FF300E945C2DA1E081
:10620000B1E08C9184FB16F00C9408310E94122EA0
:10621000AC81BD810E948DEF0C94CA30AE81BF81EC
:106220008D919C91AFE3B7E08D939C93A3EDB4E087
:106230000D911C91093250E015070CF402C00C942A
:106240004131A3EDB4E00D911C91003050E01507F1
:1062500011F40C944131A3EDB4E00D911C914AEB83
:1062600050E0040F151FACE0B5E00D931C9381E0E6
:10627000809351040E943B8580913E078064809307
:106280003E070E94373DAA81BB810C91013011F07D
:106290000C948431E9E0F5E0A190BB24E8E0F5E05E
:1062A000AA0CBB1CEA0DFB1DAE81BF810E9485F5C7
:1062B000E9E0F5E0A190BB24E4E6F3E0AA0CBB1C06
:1062C000EA0DFB1DA3EDB4E00E9485F5E9E0F5E0E1
:1062D000A190BB24E0EAF3E0AA0CBB1CEA0DFB1D75
:1062E000A5EDB4E00E9485F5E9E0F5E0A190BB24BE
:1062F000E8EFF5E0AA0CBB1CEA0DFB1DA7EDB4E02E
:106300000E9485F50C94BE31023011F00C94A2313C
:10631000EAE1F5E0AE81BF810E9485F5E6E7F3E0B2
:10632000A3EDB4E00E9485F5E2EBF3E0A5EDB4E067
:106330000E9485F5EAE0F6E0A7EDB4E00E9485F55D
:106340000C94BE31033011F00C94BE31ECE1F5E059
:10635000AE81BF810E9485F5E8E7F3E0A3EDB4E0EC
:106360000E9485F5E4EBF3E0A5EDB4E00E9485F52D
:10637000ECE0F6E0A7EDB4E00E9485F5AE81BF81C8
:106380000D911C914AE050E00E94C5EFAE81BF81A3
:106390004D935C9381E090E0AC81BD818D939C93A3
:1063A000AC81BD810D911C910A3050E015071CF0A5
:1063B00011F00C940232AE81BF818D919C910E94AC
:1063C000EBF00E947D180091F503013011F00C9460
:1063D000EB310C94B3335A924A92AC81BD818C91CB
:1063E000A42DB52D8C9381E00E9485EF0E94C82ECC
:1063F000229681E00E9481EFAC81BD810E948DEFE9
:106400000C94D031AE81BF818D919C91AFE3B7E008
:106410008D939C930E94373DAA81BB810C910130E2
:1064200011F00C944D32E9E0F5E0A190BB24E4E4D6
:10643000F5E0AA0CBB1CEA0DFB1DAE81BF810E94DA
:1064400085F5E9E0F5E0A190BB24ECEDF3E0AA0CC2
:10645000BB1CEA0DFB1DA3EDB4E00E9485F5E9E04D
:10646000F5E0A190BB24E8E1F4E0AA0CBB1CEA0D26
:10647000FB1DA5EDB4E00E9485F5E9E0F5E0A190F3
:10648000BB24E4E3F6E0AA0CBB1CEA0DFB1DA7ED60
:10649000B4E00E9485F50C948732023011F00C9420
:1064A0006B32E6E5F5E0AE81BF810E9485F5EEEE48
:1064B000F3E0A3EDB4E00E9485F5EAE2F4E0A5ED97
:1064C000B4E00E9485F5E6E4F6E0A7EDB4E00E94B2
:1064D00085F50C948732033011F00C948732E8E58F
:1064E000F5E0AE81BF810E9485F5E0EFF3E0A3ED1A
:1064F000B4E00E9485F5ECE2F4E0A5EDB4E00E9482
:1065000085F5E8E4F6E0A7EDB4E00E9485F5AE81FC
:10651000BF810D911C914AE050E00E94C5EFAE8111
:10652000BF814D935C9381E090E0AC81BD818D9300
:106530009C93AC81BD810D911C910A3050E01507F0
:106540001CF011F00C94CB32AE81BF818D919C91E7
:106550000E94EBF00E947D180091F503013011F0CC
:106560000C94B4320C94B3335A924A92AC81BD81EC
:106570008C91A42DB52D8C9381E00E9485EF0E9413
:10658000C82E229681E00E9481EFAC81BD810E94DD
:106590008DEF0C949932AE81BF818D919C91AFE3C8
:1065A000B7E08D939C930E94373DAA81BB810C91EB
:1065B000013011F00C941633E9E0F5E0A190BB2412
:1065C000E0E8F5E0AA0CBB1CEA0DFB1DAE81BF8123
:1065D0000E9485F5E9E0F5E0A190BB24E4E5F4E054
:1065E000AA0CBB1CEA0DFB1DA3EDB4E00E9485F5CF
:1065F000E9E0F5E0A190BB24E0E9F4E0AA0CBB1CC3
:10660000EA0DFB1DA5EDB4E00E9485F5E9E0F5E09B
:10661000A190BB24E0E7F6E0AA0CBB1CEA0DFB1D31
:10662000A7EDB4E00E9485F50C945033023011F0D0
:106630000C943433E2E9F5E0AE81BF810E9485F528
:10664000E6E6F4E0A3EDB4E00E9485F5E2EAF4E0CA
:10665000A5EDB4E00E9485F5E2E8F6E0A7EDB4E030
:106660000E9485F50C945033033011F00C94503394
:10667000E4E9F5E0AE81BF810E9485F5E8E6F4E04B
:10668000A3EDB4E00E9485F5E4EAF4E0A5EDB4E002
:106690000E9485F5E4E8F6E0A7EDB4E00E9485F5F8
:1066A000AE81BF810D911C914AE050E00E94C5EF80
:1066B000AE81BF814D935C9381E090E0AC81BD8160
:1066C0008D939C93AC81BD810D911C910A3050E05B
:1066D00015071CF011F00C949433AE81BF818D919D
:1066E0009C910E94EBF00E947D180091F50301300F
:1066F00011F00C947D330C94B3335A924A92AC81CE
:10670000BD818C91A42DB52D8C9381E00E9485EFE5
:106710000E94C82E229681E00E9481EFAC81BD814B
:106720000E948DEF0C946233AE81BF818D919C915C
:10673000AFE3B7E08D939C930E94373DAA81BB8164
:106740008C918F5F8C9310F40C94C32F809169040B
:106750008F7E8093690482E08093450580913E0797
:106760008F7B80933E0786E0481A8827580A289630
:10677000089582E00E94FAF082E00E94FAF081E03F
:106780000E94FAF081E00E94FAF000910A050030C0
:1067900011F00C94D03382E0809346050C940638B7
:1067A0005A924A9281E0A42DB52D8C9381E00E94EB
:1067B00085EF5A924A9285E0A42DB52D8C9381E005
:1067C0000E9485EF5A924A9282E0A42DB52D8C93B7
:1067D00081E00E9485EF0E9421DE269683E00E94E0
:1067E00081EF5A924A9280E0A42DB52D8C9381E0DE
:1067F0000E9485EF5A924A9285E0A42DB52D8C9384
:1068000081E00E9485EF5A924A9281E0A42DB52D35
:106810008C9381E00E9485EF0E9421DE269683E022
:106820000E9481EF5A924A9280E0A42DB52D8C935C
:1068300081E00E9485EF5A924A9285E0A42DB52D01
:106840008C9381E00E9485EF5A924A9283E0A42DB6
:10685000B52D8C9381E00E9485EF0E9421DE269663
:1068600083E00E9481EF81E0AA81BB818C93AA81A1
:10687000BB810C91033018F011F00C94F93780E0D3
:10688000A881B9818C93AA81BB810C91013011F050
:106890000C945734A1E0B1E08C9185FB16F00C9478
:1068A000553481E0A881B9818C930C947034023006
:1068B00011F00C94613481E0A881B9818C930C941F
:1068C0007034033011F00C947034A1E0B1E08C917D
:1068D00080FB16F00C94703481E0A881B9818C9310
:1068E000AA81BB81AD90BB24ABE3B4E0AA0DBB1D74
:1068F0000C91013011F00C94F137A9E6B4E08C91C1
:1069000085FB16F40C94F137A881B9810C91013004
:1069100011F00C94F13780916904806180936904CF
:10692000AA81BB810C91013011F00C94B134E4EFD9
:10693000F4E0AE81BF810E9485F5E4E1F3E0A3EDD0
:10694000B4E00E9485F5E0E5F3E0A5EDB4E00E9437
:1069500085F5E4EEF5E0A7EDB4E00E9485F50C9432
:106960000B35023011F00C94EF34EAE0F5E0A19021
:10697000BB24E0EEF4E0AA0CBB1CEA0DFB1DAE81CB
:10698000BF810E9485F5EAE0F5E0A190BB24E0E03C
:10699000F3E0AA0CBB1CEA0DFB1DA3EDB4E00E94C2
:1069A00085F5EAE0F5E0A190BB24ECE3F3E0AA0C66
:1069B000BB1CEA0DFB1DA5EDB4E00E9485F5EAE0E5
:1069C000F5E0A190BB24E0EDF5E0AA0CBB1CEA0DBC
:1069D000FB1DA7EDB4E00E9485F50C940B35033048
:1069E00011F00C940B35E2EFF4E0AE81BF810E9410
:1069F00085F5E2E1F3E0A3EDB4E00E9485F5EEE475
:106A0000F3E0A5EDB4E00E9485F5E2EEF5E0A7ED38
:106A1000B4E00E9485F5AE81BF810D911C914AE0E2
:106A200050E00E94C5EFAE81BF814D935C9381E041
:106A300090E0AC81BD818D939C93AC81BD810D9123
:106A40001C910A3050E015071CF011F00C946135D0
:106A5000AE81BF818D919C910E94EBF00E947D18C8
:106A60000091F603013011F00C9438350C9406387F
:106A70005A924A92AC81BD818C91A42DB52D8C93F4
:106A800081E00E9485EF0E94C82E229681E00E943C
:106A900081EFA1E0B1E08C9183FB16F00C945235AC
:106AA0000E94A62CA1E0B1E08C9182FB16F00C9420
:106AB0005B350E94122EAC81BD810E948DEF0C943B
:106AC0001D35AE81BF818D919C91AFE3B7E08D9371
:106AD0009C93A3EDB4E00D911C91093250E0150791
:106AE0000CF402C00C949435A3EDB4E00D911C910C
:106AF000003050E0150711F40C949435A3EDB4E088
:106B00000D911C914AEB50E0040F151FACE0B5E06D
:106B10000D931C9382E0809351040E943B858091E9
:106B20003E07806480933E070E94373DAA81BB8167
:106B30000C91013011F00C94B735E0E3F5E0AE8133
:106B4000BF810E9485F5ECE8F3E0A3EDB4E00E947C
:106B500085F5E8ECF3E0A5EDB4E00E9485F5E0E210
:106B6000F6E0A7EDB4E00E9485F50C9411360230F2
:106B700011F00C94F535EAE0F5E0A190BB24ECE1CE
:106B8000F5E0AA0CBB1CEA0DFB1DAE81BF810E9483
:106B900085F5EAE0F5E0A190BB24E8E7F3E0AA0C74
:106BA000BB1CEA0DFB1DA3EDB4E00E9485F5EAE0F5
:106BB000F5E0A190BB24E4EBF3E0AA0CBB1CEA0DCA
:106BC000FB1DA5EDB4E00E9485F5EAE0F5E0A1909B
:106BD000BB24ECE0F6E0AA0CBB1CEA0DFB1DA7ED04
:106BE000B4E00E9485F50C941136033011F00C943A
:106BF0001136EEE2F5E0AE81BF810E9485F5EAE84C
:106C0000F3E0A3EDB4E00E9485F5E6ECF3E0A5ED3A
:106C1000B4E00E9485F5EEE1F6E0A7EDB4E00E9455
:106C200085F5AE81BF810D911C914AE050E00E9434
:106C3000C5EFAE81BF814D935C9381E090E0AC8164
:106C4000BD818D939C93AC81BD810D911C910A30C7
:106C500050E015071CF011F00C945536AE81BF8141
:106C60008D919C910E94EBF00E947D180091F6039B
:106C7000013011F00C943E360C9406385A924A9228
:106C8000AC81BD818C91A42DB52D8C9381E00E94A7
:106C900085EF0E94C82E229681E00E9481EFAC8190
:106CA000BD810E948DEF0C942336AE81BF818D9102
:106CB0009C91AFE3B7E08D939C930E94373DAA81EE
:106CC000BB810C91013011F00C948036ECE6F5E0BC
:106CD000AE81BF810E9485F5E4E0F4E0A3EDB4E06D
:106CE0000E9485F5E0E4F4E0A5EDB4E00E9485F5AE
:106CF000ECE5F6E0A7EDB4E00E9485F50C94DA36F9
:106D0000023011F00C94BE36EAE0F5E0A190BB240D
:106D1000E8E5F5E0AA0CBB1CEA0DFB1DAE81BF81C6
:106D20000E9485F5EAE0F5E0A190BB24E0EFF3E0F6
:106D3000AA0CBB1CEA0DFB1DA3EDB4E00E9485F577
:106D4000EAE0F5E0A190BB24ECE2F4E0AA0CBB1C65
:106D5000EA0DFB1DA5EDB4E00E9485F5EAE0F5E043
:106D6000A190BB24E8E4F6E0AA0CBB1CEA0DFB1DD5
:106D7000A7EDB4E00E9485F50C94DA36033011F0EB
:106D80000C94DA36EAE6F5E0AE81BF810E9485F523
:106D9000E2E0F4E0A3EDB4E00E9485F5EEE3F4E078
:106DA000A5EDB4E00E9485F5EAE5F6E0A7EDB4E0D4
:106DB0000E9485F5AE81BF810D911C914AE050E0A3
:106DC0000E94C5EFAE81BF814D935C9381E090E05E
:106DD000AC81BD818D939C93AC81BD810D911C9143
:106DE0000A3050E015071CF011F00C941E37AE81EC
:106DF000BF818D919C910E94EBF00E947D180091C3
:106E0000F603013011F00C9407370C9406385A92AF
:106E10004A92AC81BD818C91A42DB52D8C9381E0DB
:106E20000E9485EF0E94C82E229681E00E9481EF89
:106E3000AC81BD810E948DEF0C94EC36AE81BF8198
:106E40008D919C91AFE3B7E08D939C930E94373D69
:106E5000AA81BB810C91013011F00C944937E8EA0A
:106E6000F5E0AE81BF810E9485F5ECE7F4E0A3ED8B
:106E7000B4E00E9485F5E8EBF4E0A5EDB4E00E94F3
:106E800085F5E8E9F6E0A7EDB4E00E9485F50C94FD
:106E9000A337023011F00C948737EAE0F5E0A190B7
:106EA000BB24E4E9F5E0AA0CBB1CEA0DFB1DAE8196
:106EB000BF810E9485F5EAE0F5E0A190BB24E8E6F9
:106EC000F4E0AA0CBB1CEA0DFB1DA3EDB4E00E948C
:106ED00085F5EAE0F5E0A190BB24E4EAF4E0AA0C31
:106EE000BB1CEA0DFB1DA5EDB4E00E9485F5EAE0B0
:106EF000F5E0A190BB24E4E8F6E0AA0CBB1CEA0D87
:106F0000FB1DA7EDB4E00E9485F50C94A337033078
:106F100011F00C94A337E6EAF5E0AE81BF810E9440
:106F200085F5EAE7F4E0A3EDB4E00E9485F5E6EB31
:106F3000F4E0A5EDB4E00E9485F5E6E9F6E0A7ED02
:106F4000B4E00E9485F5AE81BF810D911C914AE0AD
:106F500050E00E94C5EFAE81BF814D935C9381E00C
:106F600090E0AC81BD818D939C93AC81BD810D91EE
:106F70001C910A3050E015071CF011F00C94E73713
:106F8000AE81BF818D919C910E94EBF00E947D1893
:106F90000091F603013011F00C94D0370C940638B0
:106FA0005A924A92AC81BD818C91A42DB52D8C93BF
:106FB00081E00E9485EF0E94C82E229681E00E9407
:106FC00081EFAC81BD810E948DEF0C94B537AE810D
:106FD000BF818D919C91AFE3B7E08D939C930E940C
:106FE000373DAA81BB818C918F5F8C9310F40C94F8
:106FF000373482E080934605809169048F7E8093C8
:10700000690480913E078F7B80933E0786E0481A93
:107010008827580A2896089582E00E94FAF082E0B4
:107020000E94FAF081E00E94FAF081E00E94FAF0FA
:1070300000910B05003011F00C94233882E080930E
:1070400047050C94593C5A924A9281E0A42DB52DE3
:107050008C9381E00E9485EF5A924A9285E0A42D9C
:10706000B52D8C9381E00E9485EF5A924A9283E07D
:10707000A42DB52D8C9381E00E9485EF0E9421DE26
:10708000269683E00E9481EF5A924A9280E0A42DD6
:10709000B52D8C9381E00E9485EF5A924A9285E04B
:1070A000A42DB52D8C9381E00E9485EF5A924A92CF
:1070B00082E0A42DB52D8C9381E00E9485EF0E9483
:1070C00021DE269683E00E9481EF5A924A9280E068
:1070D000A42DB52D8C9381E00E9485EF5A924A929F
:1070E00085E0A42DB52D8C9381E00E9485EF5A9206
:1070F0004A9281E0A42DB52D8C9381E00E9485EF0A
:107100000E9421DE269683E00E9481EF81E0AA8121
:10711000BB818C93AA81BB810C91033018F011F0D4
:107120000C944C3C80E0A881B9818C93AA81BB81EE
:107130000C91013011F00C94AA38A1E0B1E08C91CF
:1071400084FB16F00C94A83881E0A881B9818C9357
:107150000C94C338023011F00C94BB38A1E0B1E0BC
:107160008C9182FB16F00C94B93881E0A881B9812A
:107170008C930C94C338033011F00C94C33881E025
:10718000A881B9818C93AA81BB81AD90BB24ABE36C
:10719000B4E0AA0DBB1D0C91013011F00C94443CDD
:1071A000A9E6B4E08C9185FB16F40C94443CA881CC
:1071B000B9810C91013011F00C94443C8091690428
:1071C000806180936904AA81BB810C91013011F028
:1071D0000C940439E6E0F5E0AE81BF810E9485F5AC
:1071E000E6E2F3E0A3EDB4E00E9485F5E2E6F3E029
:1071F000A5EDB4E00E9485F5E6EFF5E0A7EDB4E07B
:107200000E9485F50C945E39023011F00C942239FD
:10721000E8E0F5E0AE81BF810E9485F5E8E2F3E0A9
:10722000A3EDB4E00E9485F5E4E6F3E0A5EDB4E05B
:107230000E9485F5E8EFF5E0A7EDB4E00E9485F542
:107240000C945E39033011F00C945E39EBE0F5E0FC
:10725000A190BB24E4EFF4E0AA0CBB1CEA0DFB1DDB
:10726000AE81BF810E9485F5EBE0F5E0A190BB24E3
:10727000E4E1F3E0AA0CBB1CEA0DFB1DA3EDB4E0B6
:107280000E9485F5EBE0F5E0A190BB24E0E5F3E09A
:10729000AA0CBB1CEA0DFB1DA5EDB4E00E9485F510
:1072A000EBE0F5E0A190BB24E4EEF5E0AA0CBB1CFA
:1072B000EA0DFB1DA7EDB4E00E9485F5AE81BF810C
:1072C0000D911C914AE050E00E94C5EFAE81BF8154
:1072D0004D935C9381E090E0AC81BD818D939C9354
:1072E000AC81BD810D911C910A3050E015071CF056
:1072F00011F00C94B439AE81BF818D919C910E94A4
:10730000EBF00E947D180091F703013011F00C940E
:107310008B390C94593C5A924A92AC81BD818C9124
:10732000A42DB52D8C9381E00E9485EF0E94C82E7C
:10733000229681E00E9481EFA1E0B1E08C9180FB78
:1073400016F00C94A5390E945C2DA1E0B1E08C915F
:1073500081FB16F00C94AE390E94A62CAC81BD8145
:107360000E948DEF0C947039AE81BF818D919C91FC
:10737000AFE3B7E08D939C93A3EDB4E00D911C9126
:10738000093250E015070CF402C00C94E739A3ED64
:10739000B4E00D911C91003050E0150711F40C94ED
:1073A000E739A3EDB4E00D911C914AEB50E0040FD6
:1073B000151FACE0B5E00D931C9383E0809351045E
:1073C0000E943B8580913E07806480933E070E9427
:1073D000373DAA81BB810C91013011F00C940A3A1F
:1073E000E2E4F5E0AE81BF810E9485F5EEE9F3E0CD
:1073F000A3EDB4E00E9485F5EAEDF3E0A5EDB4E07D
:107400000E9485F5E2E3F6E0A7EDB4E00E9485F581
:107410000C94643A023011F00C94283AE4E4F5E05C
:10742000AE81BF810E9485F5E0EAF3E0A3EDB4E010
:107430000E9485F5ECEDF3E0A5EDB4E00E9485F542
:10744000E4E3F6E0A7EDB4E00E9485F50C94643A1D
:10745000033011F00C94643AEBE0F5E0A190BB240A
:10746000E0E3F5E0AA0CBB1CEA0DFB1DAE81BF8179
:107470000E9485F5EBE0F5E0A190BB24ECE8F3E099
:10748000AA0CBB1CEA0DFB1DA3EDB4E00E9485F520
:10749000EBE0F5E0A190BB24E8ECF3E0AA0CBB1C08
:1074A000EA0DFB1DA5EDB4E00E9485F5EBE0F5E0EB
:1074B000A190BB24E0E2F6E0AA0CBB1CEA0DFB1D88
:1074C000A7EDB4E00E9485F5AE81BF810D911C91BE
:1074D0004AE050E00E94C5EFAE81BF814D935C93BE
:1074E00081E090E0AC81BD818D939C93AC81BD81A6
:1074F0000D911C910A3050E015071CF011F00C940E
:10750000A83AAE81BF818D919C910E94EBF00E94C0
:107510007D180091F703013011F00C94913A0C940E
:10752000593C5A924A92AC81BD818C91A42DB52DC3
:107530008C9381E00E9485EF0E94C82E229681E004
:107540000E9481EFAC81BD810E948DEF0C94763A50
:10755000AE81BF818D919C91AFE3B7E08D939C93F9
:107560000E94373DAA81BB810C91013011F00C942F
:10757000D33AEEE7F5E0AE81BF810E9485F5E6E102
:10758000F4E0A3EDB4E00E9485F5E2E5F4E0A5EDBA
:10759000B4E00E9485F5EEE6F6E0A7EDB4E00E94C7
:1075A00085F50C942D3B023011F00C94F13AE0E893
:1075B000F5E0AE81BF810E9485F5E8E1F4E0A3ED3E
:1075C000B4E00E9485F5E4E5F4E0A5EDB4E00E94A6
:1075D00085F5E0E7F6E0A7EDB4E00E9485F50C94B0
:1075E0002D3B033011F00C942D3BEBE0F5E0A19026
:1075F000BB24ECE6F5E0AA0CBB1CEA0DFB1DAE813A
:10760000BF810E9485F5EBE0F5E0A190BB24E4E0AA
:10761000F4E0AA0CBB1CEA0DFB1DA3EDB4E00E9434
:1076200085F5EBE0F5E0A190BB24E0E4F4E0AA0CE2
:10763000BB1CEA0DFB1DA5EDB4E00E9485F5EBE057
:10764000F5E0A190BB24ECE5F6E0AA0CBB1CEA0D2A
:10765000FB1DA7EDB4E00E9485F5AE81BF810D91C1
:107660001C914AE050E00E94C5EFAE81BF814D936E
:107670005C9381E090E0AC81BD818D939C93AC8163
:10768000BD810D911C910A3050E015071CF011F0DE
:107690000C94713BAE81BF818D919C910E94EBF067
:1076A0000E947D180091F703013011F00C945A3BB1
:1076B0000C94593C5A924A92AC81BD818C91A42D74
:1076C000B52D8C9381E00E9485EF0E94C82E2296F2
:1076D00081E00E9481EFAC81BD810E948DEF0C940E
:1076E0003F3BAE81BF818D919C91AFE3B7E08D931D
:1076F0009C930E94373DAA81BB810C91013011F00F
:107700000C949C3BEAEBF5E0AE81BF810E9485F5CD
:10771000EEE8F4E0A3EDB4E00E9485F5EAECF4E0D5
:10772000A5EDB4E00E9485F5EAEAF6E0A7EDB4E045
:107730000E9485F50C94F63B023011F00C94BA3B94
:10774000ECEBF5E0AE81BF810E9485F5E0E9F4E065
:10775000A3EDB4E00E9485F5ECECF4E0A5EDB4E017
:107760000E9485F5ECEAF6E0A7EDB4E00E9485F50D
:107770000C94F63B033011F00C94F63BEBE0F5E093
:10778000A190BB24E8EAF5E0AA0CBB1CEA0DFB1DA6
:10779000AE81BF810E9485F5EBE0F5E0A190BB24AE
:1077A000ECE7F4E0AA0CBB1CEA0DFB1DA3EDB4E072
:1077B0000E9485F5EBE0F5E0A190BB24E8EBF4E056
:1077C000AA0CBB1CEA0DFB1DA5EDB4E00E9485F5DB
:1077D000EBE0F5E0A190BB24E8E9F6E0AA0CBB1CC5
:1077E000EA0DFB1DA7EDB4E00E9485F5AE81BF81D7
:1077F0000D911C914AE050E00E94C5EFAE81BF811F
:107800004D935C9381E090E0AC81BD818D939C931E
:10781000AC81BD810D911C910A3050E015071CF020
:1078200011F00C943A3CAE81BF818D919C910E94E5
:10783000EBF00E947D180091F703013011F00C94D9
:10784000233C0C94593C5A924A92AC81BD818C9154
:10785000A42DB52D8C9381E00E9485EF0E94C82E47
:10786000229681E00E9481EFAC81BD810E948DEF64
:107870000C94083CAE81BF818D919C91AFE3B7E041
:107880008D939C930E94373DAA81BB818C918F5F21
:107890008C9310F40C948A3882E080934705809191
:1078A00069048F7E8093690480913E078F7B80936B
:1078B0003E0786E0481A8827580A28960895A88126
:1078C000B981AD90BB24A6E0B4E0AA0DBB1D0C911C
:1078D000003011F40C94103DA881B981AD90BB2407
:1078E000A6E0B4E0AA0DBB1D4C91A881B981AD9072
:1078F000BB24A3E0B4E0AA0DBB1D0C91041710F447
:107900000C940E3D80E0A881B981AD90BB24A3E02A
:10791000B4E0AA0DBB1D8C93A881B981AD90BB24A6
:10792000ADE6B6E0AA0DBB1D8C918F5F8C93A8814C
:10793000B981AD90BB24A0E7B6E0AA0DBB1D0C91A8
:10794000003011F40C94DE3CE881F981A190BB2455
:10795000E4E8FFE0EA0DFB1DA0E1B0E00E9483F542
:10796000003011F40C94DE3CA881B981AD90BB24A9
:10797000A0E7B6E0AA0DBB1D4C91A881B981AD90DE
:10798000BB24ADE6B6E0AA0DBB1D0C91041710F4A4
:107990000C94DE3C80E0A881B981AD90BB24ADE6BB
:1079A000B6E0AA0DBB1D8C9381E0A881B981AD9092
:1079B000BB24AAE3B7E0AA0DBB1D8C93A881B981B3
:1079C000AD90BB24AEEEB6E0AA0DBB1D0C9100300D
:1079D00011F00C940E3D80E0A881B981AD90BB24DC
:1079E000A8E3B4E0AA0DBB1D8C93A881B981AD902A
:1079F000BB24AAE3B7E0AA0DBB1D0C91003011F027
:107A00000C940E3D80E0A881B981AD90BB24ADEF10
:107A1000B3E0AA0DBB1D8C930E94B0100C94363DB0
:107A2000A881B981AD90BB24A1EFB3E0AA0DBB1D25
:107A30000C91003011F00C94363DA881B981AD90C5
:107A4000BB24AEECB4E0AA0DBB1D0C91003011F0CC
:107A50000C94363D80E0A881B981AD90BB24ADEF98
:107A6000B3E0AA0DBB1D8C930E94B0100895AEE345
:107A7000B7E08C9186FB16F40C945B3DAFE3B7E066
:107A80000D911C91003050E0150781E009F480E071
:107A90008F93A7EDB4E00D911C91003050E01507D5
:107AA00081E009F480E09F91892B882311F40C94E4
:107AB0005B3D0E94427F089580E10E94FAF0AFE4AE
:107AC000B4E080B38C9394E0AFE4B4E00E94AEF1F4
:107AD000A881B981E2EEFDEE0E94DDF30E9497F1EC
:107AE00000914F04003011F00C94803DABE6B1E002
:107AF000E2EFFDEE0E94DDF30E9497F10C948A3DC7
:107B000080914F04E881F98101E00A93ABE6B1E08E
:107B10000E9452F5809B0C949C3D5A924A9281E0BF
:107B2000A42DB52D8C9381E00E9485EF0E94C63D67
:107B3000229681E00E9481EF819B0C94AE3D5A9287
:107B40004A9282E0A42DB52D8C9381E00E9485EFAE
:107B50000E94C63D229681E00E9481EF829B0C9498
:107B6000C03D5A924A9283E0A42DB52D8C9381E0BA
:107B70000E9485EF0E94C63D229681E00E9481EF1F
:107B800080E1481A8827580A2296089581E00E94C9
:107B9000FAF0E7E2F8E0A0E1B0E00E9483F50130FE
:107BA00011F00C94033EAA81BB81AD90BB24A6E8E2
:107BB000B6E0AA0DBB1D0C91013011F00C94033EF0
:107BC0005A924A9280E0A42DB52D8C9381E00E94B8
:107BD00085EF5A924A92AE81BF818C91A42DB52D2A
:107BE0008C9381E00E9485EF5A924A9284E0A42D02
:107BF000B52D8C9381E00E9485EF0E9421DE2696B0
:107C000083E00E9481EF81E0A881B9818C93A881F3
:107C1000B9810C91033018F011F00C94B63EE88154
:107C2000F981A190BB24EBEAF0E0EA0DFB1DA0E195
:107C3000B0E00E9483F5013011F00C94AE3EEEE20C
:107C4000F0E0A0E1B0E00E9483F5023011F00C9466
:107C5000663EAA81BB810D91112748E450E00E9445
:107C60008DF1A5E2B1E0A00FB11F0E94A7F5082F8A
:107C7000003018F011F00C943F3E0C94643E5A9280
:107C80004A9280E0A42DB52D8C9381E00E9485EF6F
:107C90005A924A92AE81BF818C91A42DB52D8C93BE
:107CA00081E00E9485EF5A924A92AE81BF818C9109
:107CB000A42DB52D8C9381E00E9485EF0E9421DEDA
:107CC000269683E00E9481EF0C948B3E5A924A9252
:107CD00080E0A42DB52D8C9381E00E9485EF5A920F
:107CE0004A92AE81BF818C91A42DB52D8C9381E0F9
:107CF0000E9485EF5A924A92AE81BF818C91A42D49
:107D0000B52D8C9381E00E9485EF0E9421DE26969E
:107D100083E00E9481EF81E0A881B981AD90BB240E
:107D2000AFE3B4E0AA0DBB1D8C93A881B981AD90DF
:107D3000BB24AEE0B6E0AA0DBB1D0C91003011F0E3
:107D40000C94AE3E80E0A881B981AD90BB24ADEF2C
:107D5000B3E0AA0DBB1D8C930E94B010A881B9811D
:107D60008C918F5F8C9310F40C94073E81E0481A3D
:107D70008827580A2296089589E00E94FAF084E044
:107D80000E94FAF081E00E94FAF081E00E94FAF08D
:107D900081E00E94FAF085E00E94FAF0A1E0B1E0F3
:107DA0008C9186FB16F40C94FE3EE0EFF3E0A1907C
:107DB000BB24EBE4F0E0EA0DFB1DA0E1B0E00E9483
:107DC00083F5013011F00C94FC3EA0EFB3E0AD90D0
:107DD000BB24A5E3B6E0AA0DBB1D0C91003011F049
:107DE0000C94FC3E80E08093F0038091B7038F7B7E
:107DF0008093B7030C94CC400C94273FA0E2B1E0F1
:107E00000E94A7F5082F41E0041BAE81BF810C93AF
:107E1000E0E2F1E001E0AA85BB850E9459F5AA8560
:107E2000BB850E94FEF4A2EDB4E00C93A0E2B1E0A9
:107E30000E94A7F5EA2FFB2FAE81BF810C913197ED
:107E4000E01BF0400FEFA0E2B1E00E9459F58CE496
:107E50000E94FAF0A0E2B1E00E94A7F5EA2FFB2F02
:107E60003297F0400FEFA881B9810E9459F5EDE5F6
:107E7000F6E0A881B9810E94AFF50FB68CE4481AEC
:107E80008827580A22960FBE11F00C94693FA0E291
:107E9000B1E00E94A7F5082F41E0041BAE81BF812D
:107EA0000C93E0E2F1E0AE81BF810C91A0E2B1E081
:107EB0000E9459F5E5E1F8E0A0E1B0E00E9483F509
:107EC000003011F00C94693F8091B7038064809377
:107ED000B7038CE40E94FAF0A0E2B1E00E94A7F59B
:107EE000EA2FFB2F3297F0400FEFA881B9810E9453
:107EF00059F5A881B981E0EEFDEE0E94DDF30E9404
:107F0000ADF50FB68CE4481A8827580A22960FBEA2
:107F100011F00C94A33FA0E2B1E00E94A7F5082F56
:107F200041E0041BAE81BF810C93E0E2F1E0AE8141
:107F3000BF810C91A0E2B1E00E9459F58091B70396
:107F40008F7B8093B703EEE2F8E0A881B98194E0DB
:107F50000E948DF5A881B9818C91803011F40C9428
:107F6000FB3FA881B9810E94A7F5AE81BF818C93A8
:107F700081E0E0E2F1E0AE81BF810C910A93AB8534
:107F8000BC850E9452F5E881F981AA85BB850E94D3
:107F9000AFF511F00C94FB3FA0E2B1E00E94A7F511
:107FA000082FAE81BF814C91041BAC81BD810C9325
:107FB000A0E2B1E00E94A7F5EA2FFB2FAC81BD81C2
:107FC0000C913197E01BF0400FEFA0E2B1E00E946E
:107FD00059F581E08093D2048091EE06826080930F
:107FE000EE060E946C4480E08093D2048091EE06FD
:107FF0008D7F8093EE060091D204003011F00C9436
:108000001140A0E2B1E00E94A7F5082F023118F05C
:1080100011F00C940D400C941140A0E2B1E00E94CC
:10802000BFF3A6E2B5E08C9182FB16F00C941D40E4
:108030008091B70380648093B70381E0AE81BF81F4
:108040008C93AE81BF810C91033018F011F00C9429
:108050005540EE81FF810191112749E050E00E94D7
:108060008DF1E6E4F0E0E00FF11FAA85BB8598E012
:108070000E948DF5EA85FB85A0E2B1E00E94AFF594
:1080800011F00C944D4080916904886080936904DC
:10809000AE81BF818C918093D204AE81BF818C91DF
:1080A0008F5F8C9310F40C9421408091EE068064D5
:1080B0008093EE060091D204003011F40C946840D5
:1080C000ACE8B4E00E94BFF30E946C440C94B7404B
:1080D000E0E0F0E0A885B98593E00E948DF5A885E1
:1080E000B9858C91803011F40C94B540A885B98580
:1080F0000E94A7F5AE81BF818C93E0E2F1E0AE81F2
:10810000BF810C91AA85BB850E9459F5E885F98548
:10811000AA85BB850E94AFF511F00C94B340A0E294
:10812000B1E00E94A7F5AC81BD818C93AC81BD818B
:108130000C91AE81BF814C91041BAA81BB810C9331
:10814000A0E2B1E00E94A7F5EA2FFB2FAA81BB8134
:108150000C913197E01BF0400FEFA0E2B1E00E94DC
:1081600059F50C94B5400C94CC400E94FFB680E0C9
:108170008093F00380E0809345048091B7038F7B68
:108180008093B7038091EE068F7B8093EE068091FB
:10819000EE068F7D8093EE0685E1481A8827580AFF
:1081A0002C96089581E00E94FAF081E00E94FAF096
:1081B00081E00E94FAF081E00E94FAF081E00E94E2
:1081C000FAF081E00E94FAF081E00E94FAF081E08A
:1081D000AE81BF818C93AE81BF810C91033018F0CA
:1081E00011F00C945C44AE81BF81AD90BB24ABE731
:1081F000B6E0AA0DBB1D0C91003011F00C94124199
:10820000AE81BF81AD90BB24ACE0B4E0AA0DBB1D34
:108210008C91AE81BF81AD90BB24A9E0B4E0AA0DE2
:10822000BB1D8C935A924A92A885B9858C91A42D36
:10823000B52D8C9381E00E9485EF5A924A92AA85CF
:10824000BB85AD90BB24ABE7B6E0AA0DBB1D8C91FE
:10825000A42DB52D8C9381E00E9485EF0E94BB2A4E
:10826000249682E00E9481EF80916904806280936D
:10827000690480E0AE81BF81AD90BB24A7E1B6E088
:10828000AA0DBB1D8C93AE81BF81AD90BB24A5E030
:10829000B5E0AA0DBB1D0C91013011F00C945444B3
:1082A00081E0AE81BF81AD90BB24A6E7B6E0AA0D08
:1082B000BB1D8C93AE81BF818C918093510481E072
:1082C000AE81BF81AD90BB24A7E1B6E0AA0DBB1D76
:1082D0008C93AE81BF810C9143E0049FAA81BB8146
:1082E0000C92AE81BF81AD90BB24AFEFB4E0AA0D7C
:1082F000BB1D0C91AA81BB814C91040FA881B9814F
:108300000C93A881B9810C9143E0041BAA81BB8125
:108310000C93EA81FB81A190BB24E2ECF9E0EA0D29
:10832000FB1DAC81BD810E9483F500910E060130DA
:1083300011F00C949F4180E0AC81BD818C93AC81A5
:10834000BD810C910B3011F00C94B3418AE090E0A8
:108350008A939A930E94ABEF2296002F41E0040F7C
:10836000AC81BD810C93AC81BD810C91013011F0C9
:108370000C94BE410E941E9E0C94E841033011F003
:108380000C94C6410E94159C0C94E841053011F0F4
:108390000C94D0410E941E9E0E94159C0C94E841B2
:1083A000073011F00C94D8410E941E9E0C94E841B5
:1083B000083011F00C94E0410E94159C0C94E841A7
:1083C000093011F00C94E8410E94159C0E941E9EF9
:1083D000AE81BF81AD90BB24A5E0B5E0AA0DBB1D69
:1083E0000C91003011F00C94064280E0AE81BF8108
:1083F000AD90BB24A6E7B6E0AA0DBB1D8C9380917F
:1084000069048F7D809369040C946644AE81BF81BA
:10841000AD90BB24A6E7B6E0AA0DBB1D0C910130C0
:1084200011F00C94D743AE81BF81AD90BB24AFEF68
:10843000B4E0AA0DBB1D0C91013011F00C94A442C4
:10844000EE81FF81A190BB24E1E8F0E0EA0DFB1D85
:10845000A5E8B4E00E9483F5EE81FF81A190BB24E2
:10846000E1E8F0E0EA0DFB1DA885B9850E9483F5DF
:1084700081E0AC85BD858C93A885B9854C91AC8590
:10848000BD850C91041718F011F00C949842AE8140
:10849000BF810C91013011F00C946242EC85FD8596
:1084A000A190BB24E3ECF1E0EA0DFB1DAC85BD859A
:1084B000AD90BB24AAE6B4E0AA0DBB1D0E9483F5D3
:1084C0000C949042023011F00C947A42EC85FD85B8
:1084D000A190BB24E9EDF1E0EA0DFB1DAC85BD8563
:1084E000AD90BB24AAE6B4E0AA0DBB1D0E9483F5A3
:1084F0000C949042033011F00C949042EC85FD8571
:10850000A190BB24EFEEF1E0EA0DFB1DAC85BD852B
:10851000AD90BB24AAE6B4E0AA0DBB1D0E9483F572
:10852000AC85BD858C918F5F8C9310F40C943C428C
:1085300082E0AE81BF81AD90BB24AFEFB4E0AA0D65
:10854000BB1D8C930C94B243023011F00C942C435D
:10855000EE81FF81A190BB24E4E8F0E0EA0DFB1D71
:10856000A5E8B4E00E9483F5EE81FF81A190BB24D1
:10857000E4E8F0E0EA0DFB1DA885B9850E9483F5CB
:1085800081E0AC85BD858C93A885B9854C91AC857F
:10859000BD850C91041718F011F00C942043AE81A6
:1085A000BF810C91013011F00C94EA42EC85FD85FD
:1085B000A190BB24E5E0F2E0EA0DFB1DAC85BD8592
:1085C000AD90BB24AAE6B4E0AA0DBB1D0E9483F5C2
:1085D0000C941843023011F00C940243EC85FD8595
:1085E000A190BB24EBE1F2E0EA0DFB1DAC85BD855B
:1085F000AD90BB24AAE6B4E0AA0DBB1D0E9483F592
:108600000C941843033011F00C941843EC85FD854D
:10861000A190BB24E1E3F2E0EA0DFB1DAC85BD8532
:10862000AD90BB24AAE6B4E0AA0DBB1D0E9483F561
:10863000AC85BD858C918F5F8C9310F40C94C442F3
:1086400083E0AE81BF81AD90BB24AFEFB4E0AA0D53
:10865000BB1D8C930C94B243033011F00C94B243C5
:10866000EE81FF81A190BB24E7E8F0E0EA0DFB1D5D
:10867000A5E8B4E00E9483F5EE81FF81A190BB24C0
:10868000E7E8F0E0EA0DFB1DA885B9850E9483F5B7
:1086900081E0AC85BD858C93A885B9854C91AC856E
:1086A000BD850C91041718F011F00C94A843AE810D
:1086B000BF810C91013011F00C947243EC85FD8563
:1086C000A190BB24E7E4F2E0EA0DFB1DAC85BD857B
:1086D000AD90BB24AAE6B4E0AA0DBB1D0E9483F5B1
:1086E0000C94A043023011F00C948A43EC85FD8574
:1086F000A190BB24EDE5F2E0EA0DFB1DAC85BD8544
:10870000AD90BB24AAE6B4E0AA0DBB1D0E9483F580
:108710000C94A043033011F00C94A043EC85FD852C
:10872000A190BB24E3E7F2E0EA0DFB1DAC85BD851B
:10873000AD90BB24AAE6B4E0AA0DBB1D0E9483F550
:10874000AC85BD858C918F5F8C9310F40C944C4359
:1087500081E0AE81BF81AD90BB24AFEFB4E0AA0D44
:10876000BB1D8C930E94F1128091EE068F7D809349
:10877000EE06AE81BF81AD90BB24A5E0B5E0AA0DA9
:10878000BB1D0C91003011F00C94D74380E0AE81FA
:10879000BF81AD90BB24A6E7B6E0AA0DBB1D8C93AC
:1087A000809169048F7D809369040C946644AE8146
:1087B000BF81AD90BB24A6E7B6E0AA0DBB1D0C910E
:1087C000013011F00C94544480E0AE81BF81AD9033
:1087D000BB24A6E7B6E0AA0DBB1D8C93AC81BD817E
:1087E0000C91023011F00C94F9430E941E9E0C94DF
:1087F0002344043011F00C9401440E94159C0C9405
:108800002344063011F00C940B440E941E9E0E94DB
:10881000159C0C942344073011F00C9413440E94CF
:10882000159C0C942344083011F00C941B440E94B6
:108830001E9E0C9423440A3011F00C9423440E9491
:10884000159C0E941E9E80E0AE81BF81AD90BB242E
:10885000A5E0B5E0AA0DBB1D8C93AE81BF81AD90A4
:10886000BB24ABE7B6E0AA0DBB1D0C91013011F0A3
:108870000C9454445A924A92A885B9858C91A42D9F
:10888000B52D8C9381E00E9485EF5A924A9280E048
:10889000A42DB52D8C9381E00E9485EF0E94BB2A08
:1088A000249682E00E9481EFAE81BF818C918F5F20
:1088B0008C9310F40C94EB4080E080930E060E94A1
:1088C0007D18809169048F7D8093690487E0481A40
:1088D0008827580A2E96089585E30E94FAF081E1D0
:1088E0000E94FAF084E00E94FAF086E00E94FAF01A
:1088F00083E00E94FAF083E40E94FAF081E00E9493
:10890000FAF081E00E94FAF081E00E94FAF081E042
:108910000E94FAF081E00E94FAF081E00E94FAF0F1
:1089200081E00E94FAF081E00E94FAF082E00E9469
:10893000FAF082E00E94FAF082E00E94FAF081E010
:108940000E94FAF082E00E94FAF081E00E94FAF0C0
:1089500081E00E94FAF081E00E94FAF081E00E943A
:10896000FAF081E00E94FAF0A7EBB3E08C9186FB6D
:1089700016F40C94BF4484EF91E00E94EBF0009158
:10898000F003003018F011F00C94C8440C94D64455
:108990000091F003043010F00C94D6448091F00361
:1089A000809338048091F00380935104A9E6B4E0E9
:1089B0008C9183FB16F00C94FA448091F003809321
:1089C000330684E08093850482E380936B0489E21C
:1089D00080936C048DE280936D048091D204809327
:1089E0006E0480916904877F809369040E94F1126C
:1089F0000C94A37C8AE090E00E94EBF0E8E5F6E0BE
:108A0000A0E2B1E00E94AFF511F00C9414458CE89F
:108A100080936B0481E0809385040E94F11280E0D2
:108A20008093D2040C94A37C8CE40E94FAF0E0E2E0
:108A3000F1E003E0A881B9810E9459F5A881B981CC
:108A4000E4EFFDEE0E94DDF30E94ADF50FB68CE47D
:108A5000481A8827580A22960FBE11F00C947545C3
:108A6000A0E2B1E00E94A7F5082F43E0041BA8850F
:108A7000B9850C93A0E2B1E00E94A7F5EA2FFB2F85
:108A8000A885B9850C913197E01BF0400FEFAEA59A
:108A9000BFA50E9459F5AEA5BFA50E94FEF4AA8904
:108AA000BB890D931C9381E080938504A885B985CB
:108AB0000C91033011F00C946645AA89BB898C9106
:108AC00080936B040E94F1120C94734581E08093B3
:108AD0005004AA89BB890C914BEE040FABE6B4E0BD
:108AE0000C930E94F1120C94A37CA0E2B1E0E8EF99
:108AF000FDEE0E94DDF30E94ADF511F00C94874568
:108B00000E9459E38091B70380688093B703A0E285
:108B1000B1E0E2E0FEEE0E94DDF30E94ADF511F05F
:108B20000C94AF45A8EDB6E0EEE0FEEE0E94DDF35A
:108B30000E9497F1A8EDB6E00E940EF0E2EFFDEE84
:108B40000E94DDF30E9497F1A8EDB6E00E948EF03E
:108B50000E9488F08091B70380688093B7038CE40B
:108B60000E94FAF0E0E2F1E002E0A881B9810E94FF
:108B700059F5A881B981E2E1FEEE0E94DDF30E9481
:108B8000ADF50FB68CE4481A8827580A22960FBE16
:108B900011F00C942946A0E2B1E00E94A7F5EA2F5B
:108BA000FB2F3297F0400FEFAC8DBD8D0E9459F531
:108BB000AC8DBD8D8C9180538C93AC8DBD8D0C9103
:108BC000053018F011F00C94E7450C94E9450C942D
:108BD0009B7CAC8DBD8D0C91033010F00C940A463B
:108BE000AC8DBD8D8C91A2EDB4E0AD90BB24ACEF0B
:108BF000B4E0AA0DBB1D8C9381E0A2EDB4E0AD9072
:108C0000BB24A2E0B5E0AA0DBB1D8C930E94D880C6
:108C10000C94274681E080930E0681E0A2EDB4E03B
:108C2000AD90BB24A5E0B5E0AA0DBB1D8C93AC8D27
:108C3000BD8D0C9142E0041BA2EDB4E0AD90BB24CD
:108C4000AFEFB4E0AA0DBB1D0C930E94D2400C9470
:108C5000A37C81E0A8A1B9A18C93A8A1B9A10C9192
:108C6000033018F011F00C94FE4CA8EBB3E0E8A12F
:108C7000F9A10E94B4F4A8EBB3E00E940EF0E6E183
:108C8000FEEE0E94DDF30E9497F18CE40E94FAF060
:108C9000E0E2F1E003E0A881B9810E9459F5E8EB38
:108CA000F3E0A881B9810E94AFF50FB68CE4481AB1
:108CB0008827580A22960FBE11F00C94D046A0E2E5
:108CC000B1E00E94A7F5EA2FFB2F3297F0400FEF9B
:108CD000AC8DBD8D0E9459F5AC8DBD8D8C918053AE
:108CE0008C93E8A1F9A1A190BB24E2EAF0E0EA0D9F
:108CF000FB1DA0E1B0E00E9483F5013081E009F0A6
:108D000080E08F93AC8DBD8D0C91013081E009F036
:108D100080E09F91892B882311F40C94B246AC8D8E
:108D2000BD8D8C91A8A1B9A1AD90BB24A2E2B6E003
:108D3000AA0DBB1D8C938BEB80936B04A8A1B9A1EA
:108D40008C9180936C040AEAAC8DBD8D4C91040F1C
:108D5000ADE6B4E00C9383E0809385040E94F112A9
:108D60000C94CE468FE680936B048DEB80936C045D
:108D700084E880936D048AEA80936E0484E0809393
:108D80006F0485EB80937004A8A1B9A18C918093A6
:108D9000710487E0809385040E94F1120C94A37CF7
:108DA000A8EBB3E0E8A1F9A10E94B4F4A8EBB3E00A
:108DB0000E940EF0EAE1FEEE0E94DDF30E9497F1C0
:108DC0008CE40E94FAF0E0E2F1E003E0A881B981CE
:108DD0000E9459F5E8EBF3E0A881B9810E94AFF554
:108DE0000FB68CE4481A8827580A22960FBE11F055
:108DF0000C943B47A0E2B1E00E94A7F5EA2FFB2FBD
:108E00003297F0400FEFAC8DBD8D0E9459F5AC8DBF
:108E1000BD8D8C9180538C934091F003A8A1B9A192
:108E20000C91041711F40C943947E8A1F9A1A19011
:108E3000BB24E8E4F0E0EA0DFB1DAC8DBD8D7BE7C3
:108E40000E9467F50E94EB7E85EB80936F04A8A1DA
:108E5000B9A18C91809370040AEAAC8DBD8D4C91C0
:108E6000040FA1E7B4E00C9387E0809385040E948F
:108E7000F1120C94A37CA8EBB3E0E8A1F9A10E9445
:108E8000B4F4A8EBB3E00E940EF0EEE1FEEE0E9417
:108E9000DDF30E9497F18CE40E94FAF0E0E2F1E049
:108EA00003E0A881B9810E9459F5E8EBF3E0A881BD
:108EB000B9810E94AFF50FB68CE4481A8827580A8A
:108EC00022960FBE11F00C949847A0E2B1E00E94E8
:108ED000A7F5EA2FFB2F3297F0400FEFAC8DBD8D39
:108EE0000E9459F5AC8DBD8D8C9180538C93E8A177
:108EF000F9A1A190BB24EBE4F0E0EA0DFB1DAC8DE1
:108F0000BD8D7BE70E9467F50E94EB7E87ED809325
:108F10006F040AEAAC8DBD8D4C91040FA0E7B4E05C
:108F20000C9386E0809385040E94F1120C94A37C3C
:108F3000A8EBB3E0E8A1F9A10E94B4F4A8EBB3E078
:108F40000E940EF0E2E2FEEE0E94DDF30E9497F135
:108F50008CE40E94FAF0E0E2F1E003E0A881B9813C
:108F60000E9459F5E8EBF3E0A881B9810E94AFF5C2
:108F70000FB68CE4481A8827580A22960FBE11F0C3
:108F80000C940048A0E2B1E00E94A7F5EA2FFB2F65
:108F90003297F0400FEFAC8DBD8D0E9459F5AC8D2E
:108FA000BD8D8C9180538C93E8A1F9A1A190BB2435
:108FB000E2E4F0E0EA0DFB1DAC8DBD8D7BE70E9485
:108FC00067F50E94EB7E80E280936F048CE28093D1
:108FD00070048FE28093710483E580937204AC8DFA
:108FE000BD8D0C91013011F00C94F94787ED809301
:108FF000720488E0809385040E94F1120C94A37C93
:109000008CE40E94FAF0E0E2F1E003E0A881B9818B
:109010000E9459F5A881B981E6E2FEEE0E94DDF3D7
:109020000E94ADF50FB68CE4481A8827580A22969C
:109030000FBE11F00C946048A0E2B1E00E94A7F5C9
:10904000EA2FFB2F3297F0400FEFAC8DBD8D0E94C1
:1090500059F5AC8DBD8D8C9180538C93AC8DBD8DAD
:109060000C91013018F011F00C9438480C943A48E7
:109070000C949B7CEBE6FFE0AC8DBD8D7BE70E9402
:1090800067F5AC8DBD8D8C9180931A078AE2809331
:109090006B0480E380936C048AEA80936D04AC8D4A
:1090A000BD8D0C91013011F00C9459488BEA8093DE
:1090B0006D0483E0809385040E94F1120C94A37CDC
:1090C000A8EBB3E0E8A1F9A10E94B4F4A8EBB3E0E7
:1090D0000E940EF0EAE2FEEE0E94DDF30E9497F19C
:1090E0008CE40E94FAF0E0E2F1E003E0A881B981AB
:1090F0000E9459F5E8EBF3E0A881B9810E94AFF531
:109100000FB68CE4481A8827580A22960FBE11F031
:109110000C94E948A0E2B1E00E94A7F5EA2FFB2FEA
:109120003297F0400FEFAC8DBD8D0E9459F5AC8D9C
:10913000BD8D8C9180538C93AC8DBD8D0C91023084
:1091400018F011F00C94A6480C94A8480C949B7C41
:10915000E8A1F9A1A190BB24EAE8F0E0EA0DFB1D2B
:10916000AC8DBD8D7BE70E9467F585EB80936B042A
:10917000A8A1B9A18C9180936C0483E580936D04C0
:1091800086EC80936E0484E080938504AC8DBD8D65
:109190000C91013011F00C94D24887ED80936D044E
:1091A0000C94E548AC8DBD8D0C91023011F00C94FF
:1091B000E54887ED80936D0488E980936E0486EC22
:1091C00080936F0485E0809385040E94F1120C94D3
:1091D000A37CA8EBB3E0E8A1F9A10E94B4F4A8EB4A
:1091E000B3E00E940EF0EEE2FEEE0E94DDF30E947C
:1091F00097F18CE40E94FAF0E0E2F1E004E0A8814B
:10920000B9810E9459F5E8EBF3E0A881B9810E9489
:10921000AFF50FB68CE4481A8827580A22960FBE7D
:1092200011F00C946D49A0E2B1E00E94A7F5082F5F
:1092300044E0041BAE8DBF8D0C93A0E2B1E00E9410
:10924000A7F5EA2FFB2FAE8DBF8D0C913197E01B58
:10925000F0400FEFAEA5BFA50E9459F5AEA5BFA582
:109260000E94FEF4AC8DBD8D0C93AC8DBD8D0C9128
:109270000A3018F011F00C943F490C9441490C94B9
:109280009B7CAC8DBD8D8C91A8A1B9A1AD90BB2468
:10929000A8E0B5E0AA0DBB1D8C9385E08093850402
:1092A00085EB80936B04A8A1B9A18C9180936C0489
:1092B00080E280936D0481E380936E04A8A1B9A13C
:1092C000AD90BB24A8E0B5E0AA0DBB1D8C918093A6
:1092D0006F040E94F1120C94A37CA8EBB3E0E8A108
:1092E000F9A10E94B4F4A8EBB3E00E940EF0E2E30F
:1092F000FEEE0E94DDF30E9497F18CE40E94FAF0EA
:10930000E0E2F1E003E0A881B9810E9459F5E8EBC1
:10931000F3E0A881B9810E94AFF50FB68CE4481A3A
:109320008827580A22960FBE11F00C94D649A0E265
:10933000B1E00E94A7F5EA2FFB2F3297F0400FEF24
:10934000AC8DBD8D0E9459F5AC8DBD8D8C91805337
:109350008C93E8A1F9A1A190BB24EBE1F0E0EA0D28
:10936000FB1DAC8DBD8D7BE70E9467F585EB80937F
:109370006B04A8A1B9A18C9180936C0481E38093C4
:109380006D0481E380936E0480E280936F040AEAA7
:10939000AC8DBD8D4C91040FA0E7B4E00C9386E03A
:1093A000809385040E94F1120C94A37CA8EBB3E097
:1093B000E8A1F9A10E94B4F4A8EBB3E00E940EF07A
:1093C000E6E3FEEE0E94DDF30E9497F18CE40E943A
:1093D000FAF0E0E2F1E003E0A881B9810E9459F5DA
:1093E000E8EBF3E0A881B9810E94AFF50FB68CE4F9
:1093F000481A8827580A22960FBE11F00C946F4A1B
:10940000A0E2B1E00E94A7F5EA2FFB2F3297F040CF
:109410000FEFAC8DBD8D0E9459F5AC8DBD8D8C913B
:1094200080538C93A8A1B9A1AD90BB24A4EFB3E065
:10943000AA0DBB1D0C91013011F00C944B4AAC8D60
:10944000BD8D0C91013011F00C944B4A5A924A9206
:1094500081E0A42DB52D8C9381E00E9485EF5A9276
:109460004A92ACA1BDA18C91A42DB52D8C9381E025
:109470000E9485EF5A924A92AEA1BFA18C91A42D71
:10948000B52D8C9381E00E9485EF0E9421DE269607
:1094900083E00E9481EF85EB80936B04A8A1B9A1C2
:1094A0008C9180936C040AEAAC8DBD8D4C91040FB5
:1094B000ADE6B4E00C9383E0809385040E94F11242
:1094C000E8A1F9A1A190BB24E8E1F0E0EA0DFB1DC1
:1094D000AC8DBD8D7BE70E9467F50C94A37CA8EB57
:1094E000B3E0E8A1F9A10E94B4F4A8EBB3E00E94B4
:1094F0000EF0EAE3FEEE0E94DDF30E9497F18CE4A9
:109500000E94FAF0E0E2F1E003E0A881B9810E9454
:1095100059F5E8EBF3E0A881B9810E94AFF50FB6E9
:109520008CE4481A8827580A22960FBE11F00C9432
:10953000D74AA0E2B1E00E94A7F5EA2FFB2F3297AD
:10954000F0400FEFAC8DBD8D0E9459F5AC8DBD8DF7
:109550008C9180538C93E8A1F9A1A190BB24EDE8F4
:10956000F0E0EA0DFB1DAC8DBD8D7BE70E9467F539
:1095700085EB80936B04A8A1B9A18C9180936C04B6
:109580008CE980936D048EE980936E04AC8DBD8D63
:109590000C91013011F00C94D04A8AE980936E044A
:1095A00084E0809385040E94F1120C94A37CA8EBC4
:1095B000B3E0E8A1F9A10E94B4F4A8EBB3E00E94E3
:1095C0000EF0EEE3FEEE0E94DDF30E9497F18CE4D4
:1095D0000E94FAF0E0E2F1E003E0A881B9810E9484
:1095E00059F5E8EBF3E0A881B9810E94AFF50FB619
:1095F0008CE4481A8827580A22960FBE11F00C9462
:10960000464BA0E2B1E00E94A7F5EA2FFB2F32976C
:10961000F0400FEFAC8DBD8D0E9459F5AC8DBD8D26
:109620008C9180538C9385EB80936B04A8A1B9A196
:109630008C9180936C048DEB80936D040AEAAC8D61
:10964000BD8D4C91040FAEE6B4E00C9384E08093A2
:1096500085040E94F112AC8DBD8D8C91A8A1B9A199
:10966000AD90BB24AEE0B6E0AA0DBB1D8C93E8A183
:10967000F9A1A190BB24E2EAF0E0EA0DFB1DAC8D5C
:10968000BD8D7BE70E9467F50C94A37CA8EBB3E04B
:10969000E8A1F9A10E94B4F4A8EBB3E00E940EF097
:1096A000E2E4FEEE0E94DDF30E9497F18CE40E945A
:1096B000FAF0E0E2F1E003E0A881B9810E9459F5F7
:1096C000E8EBF3E0A881B9810E94AFF50FB68CE416
:1096D000481A8827580A22960FBE11F00C94AC4BFA
:1096E000A0E2B1E00E94A7F5EA2FFB2F3297F040ED
:1096F0000FEFAC8DBD8D0E9459F5AC8DBD8D8C9159
:1097000080538C93E8A1F9A1A190BB24ECE9F0E08F
:10971000EA0DFB1DAC8DBD8D7BE70E9467F5AC8D1E
:10972000BD8D8C91A8A1B9A1AD90BB24ABE1B6E0F1
:10973000AA0DBB1D8C930E94F87E0AEAAC8DBD8DEC
:109740004C91040FA0E7B4E00C9386E0809385046D
:109750000E94F1120C94A37CA8EBB3E0E8A1F9A15C
:109760000E94B4F4A8EBB3E00E940EF0E6E4FEEE33
:109770000E94DDF30E9497F18CE40E94FAF0E0E28F
:10978000F1E003E0A881B9810E9459F5E8EBF3E02C
:10979000A881B9810E94AFF50FB68CE4481A8827DA
:1097A000580A22960FBE11F00C94184CA0E2B1E0BA
:1097B0000E94A7F5EA2FFB2F3297F0400FEFAC8DF8
:1097C000BD8D0E9459F5AC8DBD8D8C9180538C93CD
:1097D000E8A1F9A1A190BB24E9E6F0E0EA0DFB1DA8
:1097E000AC8DBD8D7BE70E9467F5AC8DBD8D8C91F6
:1097F000A8A1B9A1AD90BB24AFE1B6E0AA0DBB1DF5
:109800008C930E94F87E86E28093700481E28093BC
:1098100071040AEAAC8DBD8D4C91040FA2E7B4E04F
:109820000C9388E0809385040E94F1120C94A37C31
:10983000A8EBB3E0E8A1F9A10E94B4F4A8EBB3E06F
:109840000E940EF0EAE4FEEE0E94DDF30E9497F122
:109850008CE40E94FAF0E0E2F1E003E0A881B98133
:109860000E9459F5E8EBF3E0A881B9810E94AFF5B9
:109870000FB68CE4481A8827580A22960FBE11F0BA
:109880000C94814CA0E2B1E00E94A7F5EA2FFB2FD7
:109890003297F0400FEFAC8DBD8D0E9459F5AC8D25
:1098A000BD8D8C9180538C93E8A1F9A1A190BB242C
:1098B000EBEAF0E0EA0DFB1DAC8DBD8D7BE70E946D
:1098C00067F585EB80936B04A8A1B9A18C91809377
:1098D0006C0481E380936D0481E380936E048EE9D0
:1098E00080936F040AEAAC8DBD8D4C91040FA0E704
:1098F000B4E00C9386E0809385040E94F1120C94EE
:10990000A37CA8EBB3E0E8A1F9A10E94B4F4A8EB12
:10991000B3E00E940EF0EEE4FEEE0E94DDF30E9442
:1099200097F18CE40E94FAF0E0E2F1E003E0A88114
:10993000B9810E9459F5E8EBF3E0A881B9810E9452
:10994000AFF50FB68CE4481A8827580A22960FBE46
:1099500011F00C94F64CA0E2B1E00E94A7F5EA2FBA
:10996000FB2F3297F0400FEFAC8DBD8D0E9459F563
:10997000AC8DBD8D8C9180538C93E8A1F9A1A19001
:10998000BB24E4E2F0E0EA0DFB1DAC8DBD8D7BE76E
:109990000E9467F5AC8DBD8D8C91A8A1B9A1AD9049
:1099A000BB24A5E2B6E0AA0DBB1D8C9385EB80938A
:1099B0006B04A8A1B9A18C9180936C0488E2809378
:1099C0006D0480E280936E0483E280936F040AEA60
:1099D000AC8DBD8D4C91040FA0E7B4E00C9386E0F4
:1099E000809385040E94F1120C94A37CA8A1B9A1D4
:1099F0008C918F5F8C9310F40C942D4681E0A8A17C
:109A0000B9A18C93A8A1B9A10C91033018F011F061
:109A10000C94864DA8EBB3E0E8A1F9A10E94B4F440
:109A2000A8EBB3E00E940EF0E2E5FEEE0E94DDF34B
:109A30000E9497F18CE40E94FAF0E0E2F1E003E08A
:109A4000A881B9810E9459F5E8EBF3E0A881B981BA
:109A50000E94AFF50FB68CE4481A8827580A229660
:109A60000FBE11F00C947E4DA0E2B1E00E94A7F56C
:109A7000EA2FFB2F3297F0400FEFAC8DBD8D0E9487
:109A800059F5AC8DBD8D8C9180538C93AC8DBD8D73
:109A90008C91A8A1B9A1AD90BB24A0E5B5E0AA0D19
:109AA000BB1D8C9383E08093850487E480936B04D3
:109AB000A8A1B9A18C9180936C040AEAAC8DBD8DEC
:109AC0004C91040FADE6B4E00C930E94F112E8A1B2
:109AD000F9A1FA93EA935A924A92A8A1B9A18C915A
:109AE000A42DB52D8C9381E00E9485EF0E946ADF42
:109AF000249681E00E9481EF0C94A37CA8A1B9A1D7
:109B00008C918F5F8C9310F40C94024DA0E2B1E025
:109B10000E94FEF4AA89BB890D931C93AA89BB8974
:109B20000D911C910D3F58E0150711F00C94E14D7B
:109B3000A1E0B1E08C9185FB16F00C94C54D5A92D2
:109B40004A9280E0A42DB52D8C9381E00E9485EF90
:109B50005A924A9281E0A42DB52D8C9381E00E9407
:109B600085EF5A924A9282E0A42DB52D8C9381E024
:109B70000E9485EF0E9421DE269683E00E9481EFFD
:109B8000809101018F7D8093010187E0809385049E
:109B90000E94087F81E080936D040E940F7F82E025
:109BA000809370048BEA809371040E94F11283E128
:109BB00090E0ACE0B5E08D939C930E943B850C94C3
:109BC000994F0C3F58E0150711F00C94034E85E1B6
:109BD00090E0ACE0B5E08D939C930E943B8587E0DC
:109BE000809385040E94087F81E080936D040E9429
:109BF0000F7F82E0809370048AEA809371040E9450
:109C0000F1120C94994F053E5CE0150711F00C948D
:109C1000524EA1E0B1E08C9184FB16F00C94364ECC
:109C20005A924A9280E0A42DB52D8C9381E00E9437
:109C300085EF5A924A9281E0A42DB52D8C9381E054
:109C40000E9485EF5A924A9283E0A42DB52D8C9301
:109C500081E00E9485EF0E9421DE269683E00E942B
:109C600081EF809101018F7E8093010187E08093D5
:109C700085040E94087F81E080936D040E940F7F1D
:109C800083E0809370048BEA809371040E94F11248
:109C900084E190E0ACE0B5E08D939C930E943B851D
:109CA0000C94994F043E5CE0150711F00C94744E2F
:109CB00086E190E0ACE0B5E08D939C930E943B85FB
:109CC00087E0809385040E94087F81E080936D0483
:109CD0000E940F7F83E0809370048AEA809371046E
:109CE0000E94F1120C94994F053155E0150711F0BF
:109CF0000C94964E87E0809385040E94087F82E052
:109D000080936D040E940F7F81E0809370048BEA42
:109D1000809371040E94F11287E190E0ACE0B5E01D
:109D20008D939C930E943B850C94994F0F3E5CE071
:109D3000150711F00C94B84E87E0809385040E94BB
:109D4000087F82E080936D040E940F7F83E0809300
:109D500070048BEA809371040E94F11288E190E014
:109D6000ACE0B5E08D939C930E943B850C94994F99
:109D7000043155E0150711F00C94DA4E89E190E0BA
:109D8000ACE0B5E08D939C930E943B8587E0809387
:109D900085040E94087F82E080936D040E940F7FFB
:109DA00081E0809370048AEA809371040E94F1122A
:109DB0000C94994F0E3E5CE0150711F00C94FC4E8C
:109DC0008AE190E0ACE0B5E08D939C930E943B85E6
:109DD00087E0809385040E94087F82E080936D0471
:109DE0000E940F7F83E0809370048AEA809371045D
:109DF0000E94F1120C94994F0F3155E0150711F0A4
:109E00000C941E4F87E0809385040E94087F83E0B6
:109E100080936D040E940F7F81E0809370048BEA31
:109E2000809371040E94F1128BE190E0ACE0B5E008
:109E30008D939C930E943B850C94994F073059E079
:109E4000150711F00C94404F87E0809385040E9421
:109E5000087F83E080936D040E940F7F82E08093EF
:109E600070048BEA809371040E94F1128CE190E0FF
:109E7000ACE0B5E08D939C930E943B850C94994F88
:109E80000E3155E0150711F00C94624F8DE190E012
:109E9000ACE0B5E08D939C930E943B8587E0809376
:109EA00085040E94087F83E080936D040E940F7FE9
:109EB00081E0809370048AEA809371040E94F11219
:109EC0000C94994F063059E0150711F00C94874F08
:109ED0008EE190E0ACE0B5E08D939C930E943B85D1
:109EE00087E0809385040E94087F83E080936D045F
:109EF0000E940F7F85EB80936F0482E08093700453
:109F00008AEA809371040E94F1120C94994F043AEA
:109F100056E0150711F00C94914F0E94159C0C947B
:109F2000994F053A56E0150711F00C94994F0E948D
:109F3000E79EA0E2B1E0E6E5FEEE0E94DDF30E94BE
:109F4000ADF511F00C94C44F0E941D7F81E0809309
:109F50006D0482E080936E0485EB80936F0482E051
:109F6000809370048BEA8093710487E0809385046A
:109F70000E94F11286E790E0ACE0B5E08D939C93EF
:109F80000E943B850C94D750EAE5FEEE0E94DDF37B
:109F90000E94ADF511F00C94ED4F0E941D7F81E001
:109FA00080936D0482E080936E0485EB80936F0450
:109FB00083E0809370048BEA8093710487E0809340
:109FC00085040E94F11287E790E0ACE0B5E08D9344
:109FD0009C930E943B850C94D750EEE5FEEE0E94C8
:109FE000DDF30E94ADF511F00C9416500E941D7F18
:109FF00082E080936D0482E080936E0485EB809311
:10A000006F0483E0809370048BEA8093710487E08F
:10A01000809385040E94F11288E790E0ACE0B5E0FF
:10A020008D939C930E943B850C94D750E2E6FEEE04
:10A030000E94DDF30E94ADF511F00C943A508BE8CC
:10A0400080936B048CE380936C0485EB80936D04A8
:10A050008BEA80936E0484E0809385040E94F11261
:10A0600089E790E0ACE0B5E08D939C930E943B853E
:10A070000C94D750E6E6FEEE0E94DDF30E94ADF5AB
:10A0800011F00C9463508AE790E0ACE0B5E08D935A
:10A090009C930E943B850E941D7F81E080936D040C
:10A0A00082E080936E0485EB80936F0482E080935E
:10A0B00070048AEA8093710487E0809385040E948B
:10A0C000F1120C94D750EAE6FEEE0E94DDF30E94F6
:10A0D000ADF511F00C948C508BE790E0ACE0B5E05E
:10A0E0008D939C930E943B850E941D7F81E080930D
:10A0F0006D0482E080936E0485EB80936F0483E0AF
:10A10000809370048AEA8093710487E080938504C9
:10A110000E94F1120C94D750EEE6FEEE0E94DDF3A1
:10A120000E94ADF511F00C94B5508CE790E0ACE0D6
:10A13000B5E08D939C930E943B850E941D7F82E039
:10A1400080936D0482E080936E0485EB80936F04AE
:10A1500083E0809370048AEA8093710487E080939F
:10A1600085040E94F1120C94D750E2E7FEEE0E94A3
:10A17000DDF30E94ADF511F00C94D7508DE790E01F
:10A18000ACE0B5E08D939C930E943B858BE8809377
:10A190006B048CE380936C0485EB80936D048AEAF6
:10A1A00080936E0484E0809385040E94F1128CE415
:10A1B0000E94FAF0E0E2F1E004E0A881B9810E9497
:10A1C00059F5A881B981E6E7FEEE0E94DDF30E9411
:10A1D000ADF50FB68CE4481A8827580A22960FBEB0
:10A1E00011F00C941751A0E2B1E00E94A7F5082FDE
:10A1F00044E0041BAE8DBF8D0C93A0E2B1E00E9441
:10A20000A7F5EA2FFB2FAE8DBF8D0C913197E01B88
:10A21000F0400FEFAEA5BFA50E9459F5EEA5FFA532
:10A22000FA93EA930E944ED222960C94A37C8CE47B
:10A230000E94FAF0E0E2F1E004E0A881B9810E9416
:10A2400059F5A881B981ECE7FEEE0E94DDF30E948A
:10A25000ADF50FB68CE4481A8827580A22960FBE2F
:10A2600011F00C945C51A0E2B1E00E94A7F5082F18
:10A2700044E0041BAE8DBF8D0C93A0E2B1E00E94C0
:10A28000A7F5EA2FFB2FAE8DBF8D0C913197E01B08
:10A29000F0400FEFAEA5BFA50E9459F580911905BA
:10A2A000806480931905EEA5FFA5FA93EA930E94B6
:10A2B00098D322960C94A37C8CE40E94FAF0E0E2FE
:10A2C000F1E004E0A881B9810E9459F5A881B98123
:10A2D000E2E8FEEE0E94DDF30E94ADF50FB68CE4DD
:10A2E000481A8827580A22960FBE11F00C94A151E3
:10A2F000A0E2B1E00E94A7F5082F44E0041BAE8D58
:10A30000BF8D0C93A0E2B1E00E94A7F5EA2FFB2FCE
:10A31000AE8DBF8D0C913197E01BF0400FEFAEA5D5
:10A32000BFA50E9459F58091190580648093190595
:10A33000EEA5FFA5FA93EA930E94C0DB22960C9447
:10A34000A37C8CE40E94FAF0E0E2F1E003E0A88153
:10A35000B9810E9459F5A881B981E8E8FEEE0E9412
:10A36000DDF30E94ADF50FB68CE4481A8827580A31
:10A3700022960FBE11F00C94EA51A0E2B1E00E94C7
:10A38000A7F5EA2FFB2F3297F0400FEFAC8DBD8D74
:10A390000E9459F5AC8DBD8D8C9180538C93E7E272
:10A3A000F8E0AC8DBD8D7BE70E9467F50E94167FBB
:10A3B0008EE980936D040AEAAC8DBD8D4C91040F3B
:10A3C000AEE6B4E00C9384E0809385040E94F11221
:10A3D0000C94A37C81E0A8A1B9A18C93A8A1B9A1F8
:10A3E0000C91053018F011F00C94A552A8EBB3E0D5
:10A3F000E8A1F9A10E94B4F4A8EBB3E00E940EF02A
:10A40000ECE8FEEE0E94DDF30E9497F18CE40E94DE
:10A41000FAF0E0E2F1E003E0A881B9810E9459F589
:10A42000E8EBF3E0A881B9810E94AFF50FB68CE4A8
:10A43000481A8827580A22960FBE11F00C949D5294
:10A44000A0E2B1E00E94A7F5EA2FFB2F3297F0407F
:10A450000FEFAC8DBD8D0E9459F5AC8DBD8D8C91EB
:10A4600080538C938EE180936B0489E280936C041B
:10A47000A8A1B9A18C9180936D04AC8DBD8D0C9178
:10A48000033010F00C946752E8A1F9A1A190BB240D
:10A49000EEEAF0E0EA0DFB1DAC8DBD8D7BE70E947E
:10A4A00067F5AC8DBD8D8C91A8A1B9A1AD90BB24F1
:10A4B000A3E0B6E0AA0DBB1D8C930AEAAC8DBD8D5E
:10A4C0004C91040FAEE6B4E00C930C949652A8A104
:10A4D000B9A10C9141E0040FAA8DBB8D0C93AA8DFC
:10A4E000BB8D8C91A9E3B0E00E94D7F30E94CDF31D
:10A4F0000C900822689409F4E894A88DB98D8827F7
:10A5000080F98C93A88DB98D0C91013011F00C94C9
:10A510008C528FE780936E04A88DB98D0C9100301A
:10A5200011F00C9496528DE880936E0484E0809331
:10A5300085040E94F1120C94A37CA8A1B9A18C916E
:10A540008F5F8C9310F40C94EE5181E0AE81BF814B
:10A550008C93AE81BF810C91073018F011F00C94F0
:10A56000A353A8EBB3E0E6E4FEEE0E94DDF30E9405
:10A5700097F1A8EBB3E00E940EF0EE81FF810E94FC
:10A58000B4F48CE40E94FAF0E0E2F1E003E0A88188
:10A59000B9810E9459F5E8EBF3E0A881B9810E94E6
:10A5A000AFF50FB68CE4481A8827580A22960FBEDA
:10A5B00011F00C949B5382E380936B0483E28093AD
:10A5C0006C04AE81BF818C9180936D0484E0809394
:10A5D000850484EF91E00E94EBF0A0E2B1E00E94DC
:10A5E000A7F5EA2FFB2F3297F0400FEFAC8DBD8D12
:10A5F0000E9459F5AC8DBD8D8C9180538C93AC8DA0
:10A60000BD8D0C91003011F00C94195380E0AE8197
:10A61000BF81AD90BB24A9E2B5E0AA0DBB1D8C9310
:10A620008AEA80936E040E94F1120E94B0100C948A
:10A630009953AC8DBD8D0C91013011F00C944853A1
:10A6400081E0AE81BF81AD90BB24A9E2B5E0AA0D47
:10A65000BB1D8C93AE81BF810C9141E0041BAC818A
:10A66000BD810C93AC81BD819C91AE81BF81AD90C9
:10A67000BB24A9E2B5E0AA0DBB1D0E94A6F18BEA9E
:10A6800080936E040E94F1120E94B0100C949953B2
:10A69000AC8DBD8D0C91023011F00C9499538DE26C
:10A6A00080936E040E94F11280E0AE81BF81AD9074
:10A6B000BB24A9E2B5E0AA0DBB1D8C930E94B0108B
:10A6C00081E0AE81BF81AD90BB24A9E2B5E0AA0DC7
:10A6D000BB1D8C93AE81BF810C9141E0041BAC810A
:10A6E000BD810C93AC81BD819C91AE81BF81AD9049
:10A6F000BB24A9E2B5E0AA0DBB1D0E94A6F184E629
:10A7000090E00E94EBF00E94B01080E0AE81BF812B
:10A71000AD90BB24A9E2B5E0AA0DBB1D8C9384E6E5
:10A7200090E00E94EBF00E94B0108AEF90E00E944F
:10A73000EBF00C94A37CAE81BF818C918F5F8C93E6
:10A7400010F40C94A9528CE40E94FAF0E0E2F1E0DB
:10A7500003E0A881B9810E9459F5A881B981E0E997
:10A76000FEEE0E94DDF30E94ADF50FB68CE4481AB0
:10A770008827580A22960FBE11F00C94F054A0E2DC
:10A78000B1E00E94A7F5EA2FFB2F3497F0400FEFBE
:10A79000AEA5BFA50E9459F585E08093850482E3AC
:10A7A00080936B0483E280936C0482E280936D0457
:10A7B00085E380936E0481E380936F04EEA5FFA58B
:10A7C00002E0ACA5BDA50E9459F5ACA5BDA50E94AF
:10A7D000FEF4AC8DBD8D0C93AC8DBD8D0C91003114
:10A7E00018F011F00C94F6530C94F8530C949B7CD5
:10A7F000AEA5BFA50E94A7F5EA2FFB2F3297F04028
:10A800000FEFAA8DBB8D0E9459F5AA8DBB8D8C913F
:10A8100080538C93AA8DBB8D0C91013081E009F09F
:10A8200080E08F93AA8DBB8D0C91023081E009F0FE
:10A8300080E09F91892B882311F40C94295481E0A6
:10A84000AC8DBD8DAD90BB24A1E3B5E0AA0DBB1DC1
:10A850008C93AA8DBB8D0C91003011F00C943A545E
:10A8600080E0AC8DBD8DAD90BB24A1E3B5E0AA0D19
:10A87000BB1D8C93AC8DBD8D0C91003018F011F088
:10A880000C9444540C945354AC8DBD8D0C910930F0
:10A8900010F00C945354AC8DBD8D0C9141E0041B11
:10A8A000A885B9850C93AC8DBD8D0C91083018F03E
:10A8B00011F00C945D540C946C54AC8DBD8D0C91C6
:10A8C000013110F00C946C54AC8DBD8D0C9149E0AD
:10A8D000041BA885B9850C93AC8DBD8D8C9180939C
:10A8E00043070E94FC7CA5E8B4E08C918F5F8C93B9
:10A8F0000AEAAA8DBB8D4C91040FA5E8B4E0AD9097
:10A90000BB24AAE6B4E0AA0DBB1D0C93AA8DBB8D97
:10A910000C91023011F00C9497548DE2A5E8B4E04C
:10A92000AD90BB24AAE6B4E0AA0DBB1D8C930E9497
:10A93000F112AA8DBB8D0C91023011F00C94DF54F2
:10A9400080E0AC8DBD8DAD90BB24A1E3B5E0AA0D38
:10A95000BB1D8C930E94B01081E0AC8DBD8DAD907D
:10A96000BB24A1E3B5E0AA0DBB1D8C93A885B985D6
:10A970009C91AC8DBD8DAD90BB24A1E3B5E0AA0D3B
:10A98000BB1D0E94A6F184E690E00E94EBF00E94BD
:10A99000B01080E0AC8DBD8DAD90BB24A1E3B5E0DF
:10A9A000AA0DBB1D8C9384E690E00E94EBF00E9400
:10A9B000B0108AEF90E00E94EBF00C94EE54A88562
:10A9C000B9859C91AC8DBD8DAD90BB24A1E3B5E064
:10A9D000AA0DBB1D0E94A6F10E94B0100C94A37C8E
:10A9E000AEEEB6E08C9181FB16F00C94F9540C9409
:10A9F000A37C8CE40E94FAF0E0E2F1E002E0A8819E
:10AA0000B9810E9459F5A881B981E4E9FEEE0E945E
:10AA1000DDF30E94ADF50FB68CE4481A8827580A7A
:10AA200022960FBE11F00C943455A0E2B1E00E94C2
:10AA3000A7F5082F42E0041BA885B9850C93A0E276
:10AA4000B1E00E94A7F5EA2FFB2FA885B9850C91EC
:10AA50003197E01BF0400FEFA0E2B1E00E9459F502
:10AA60000E94FFB60C94A37CA0E2B1E00E94A7F57F
:10AA7000A885B9858C93A885B9850C91053010F00F
:10AA80000C9444550C94A37CE0E2F1E001E0AEA10B
:10AA9000BFA10E9459F5AEA1BFA1E8E9FEEE0E9458
:10AAA000DDF30E94ADF511F40C9458550C94A37C81
:10AAB00082E0E0E2F1E001E00A93AFA1B8A50E94D4
:10AAC00052F5AEA1BFA10E94FEF4AC85BD850C93EA
:10AAD0008EEF90E0AA85BB858D939C93A885B98560
:10AAE0000C91053018F011F00C9478550C94B35576
:10AAF000E0E2F1E005E0A8A5B9A50E9459F5A88516
:10AB0000B9850D91112745E050E0041B150BA8896C
:10AB1000B9890D931C93A0E2B1E00E94A7F5EA2F3A
:10AB2000FB2FA889B9890C913197E01BF0400FEFFA
:10AB3000ACA1BDA10E9459F5A8A5B9A50E94A7F591
:10AB4000EA2FFB2F3497F0400FEFAEA5BFA50E9470
:10AB500059F5AEA5BFA50E94FEF4AA85BB850D934D
:10AB60001C930C94B5550C94A37CAC85BD850C91BD
:10AB7000013011F00C945D5AAA85BB850D911C9192
:10AB8000003050E0150711F00C941056ACA1BDA197
:10AB90000E94FEF4AC8DBD8D0C93E2EDF4E0A1902B
:10ABA000BB24EFE0F0E0EA0DFB1DAC8DBD8D7BE733
:10ABB0000E9467F5AC8DBD8D8C91A2EDB4E0AD9097
:10ABC000BB24A6E0B4E0AA0DBB1D8C93AC8DBD8D5B
:10ABD0000C91013010F00C94F75580E0A2EDB4E038
:10ABE000AD90BB24A8E0B5E0AA0DBB1D8C9385E217
:10ABF00080936B048EE180936C048BE280936D04F0
:10AC000084E280936E0484ED80936F0483EC8093E0
:10AC1000700486E0809385040E94F1120C945B5AC4
:10AC2000013050E0150711F00C944A56ACA1BDA1BB
:10AC30000E94FEF4AA89BB890D931C93E2EDF4E017
:10AC4000A190BB24E4EAF0E0AA0CBB1CEA0DFB1DBA
:10AC5000AA89BB897BE70E9469F5AA89BB898D9186
:10AC60009C91A2EDB4E0AD90BB24A4E2B4E0AA0CA8
:10AC7000BB1CAA0DBB1D8D939C9383ED80936B042D
:10AC800083EC80936C0482E0809385040E94F1122F
:10AC90000C945B5A023050E0150711F00C948E565C
:10ACA000ACA1BDA10E94FEF4AC8DBD8D0C93E2ED74
:10ACB000F4E0A190BB24E2E1F0E0EA0DFB1DAC8DD5
:10ACC000BD8D7BE70E9467F5AC8DBD8D0D91112781
:10ACD0004CE350E00E948DF1A2EDB4E0AD90BB24B6
:10ACE000AFE9B4E0AA0CBB1CAA0DBB1D0D931C93CD
:10ACF00086E280936B0486E280936C0481E2809309
:10AD00006D0484ED80936E0483EC80936F0485E082
:10AD1000809385040E94F1120C945B5A033050E03A
:10AD2000150711F00C94D256ACA1BDA10E94FEF4FF
:10AD3000AC8DBD8D0C93E2EDF4E0A190BB24E5E178
:10AD4000F0E0EA0DFB1DAC8DBD8D7BE70E9467F541
:10AD5000AC8DBD8D0D9111274CE350E00E948DF11B
:10AD6000A2EDB4E0AD90BB24A5EAB4E0AA0CBB1CF4
:10AD7000AA0DBB1D0D931C938DE280936B0486E29C
:10AD800080936C0481E280936D0484ED80936E0463
:10AD900083EC80936F0485E0809385040E94F11218
:10ADA0000C945B5A043050E0150711F00C940857CE
:10ADB000ACA1BDA10E94FEF4AC8DBD8D0C93E0EB67
:10ADC000F6E0AC8DBD8D7BE70E9467F5AC8DBD8D47
:10ADD0000D9111274CE350E00E948DF1ADECB4E0F1
:10ADE0000D931C9383E280936B048EE180936C043B
:10ADF0008BE280936D0484ED80936E0483EC8093EA
:10AE00006F0485E0809385040E94F1120C945B5AD4
:10AE1000053050E0150711F00C944A57ACA1BDA1C4
:10AE20000E94FEF4AC8DBD8D0C93E2EDF4E0A19098
:10AE3000BB24E6E9F0E0EA0DFB1DAC8DBD8D7BE7A0
:10AE40000E9467F5AC8DBD8D0D9111274CE350E04C
:10AE50000E948DF1A2EDB4E0AD90BB24AAEBB4E06A
:10AE6000AA0CBB1CAA0DBB1D0D931C9385EB8093F4
:10AE70006B048091D20480936C0484ED80936D0404
:10AE800083EC80936E0484E0809385040E94F11229
:10AE90000C945B5A063050E0150711F00C948A5759
:10AEA000ACA1BDA10E94FEF4AA89BB890D931C939D
:10AEB000E2EDF4E0A190BB24EDE1F0E0AA0CBB1CB4
:10AEC000EA0DFB1DAA89BB897BE70E9469F5AA8967
:10AED000BB898D919C91A2EDB4E0AD90BB24A3EC15
:10AEE000B4E0AA0CBB1CAA0DBB1D8D939C9387EDEF
:10AEF00080936B048EE980936C0484ED80936D04E1
:10AF000083EC80936E0484E0809385040E94F112A8
:10AF10000C945B5A073050E0150711F00C94E15780
:10AF2000ACA1BDA10E94FEF4AC8DBD8D0C93AC8D87
:10AF3000BD8D0C91013010F00C94A25781E0AC8DC6
:10AF4000BD8D8C93E2EDF4E0A190BB24EFE9F0E03D
:10AF5000EA0DFB1DAC8DBD8D7BE70E9467F5AC8DC6
:10AF6000BD8D8C91A2EDB4E0AD90BB24ACE0B4E01B
:10AF7000AA0DBB1D8C938DE280936B0489E28093B4
:10AF80006C0484ED80936D0483EC80936E0484E004
:10AF9000809385040E94F112AC8DBD8D0C910E3F03
:10AFA00011F00C94DF5780E0A2EDB4E0AD90BB242B
:10AFB000A0E0B4E0AA0DBB1D8C930E94B0100C94CD
:10AFC0005B5AAA85BB850D911C910D3050E0150789
:10AFD00080E00CF081E08F93AA85BB850D911C91D8
:10AFE0000F3050E0150781E014F009F080E09F91E8
:10AFF0008923882311F40C944158ACA1BDA10E946F
:10B00000FEF4AA89BB890D931C93AA85BB850C917C
:10B010004CE0041BAA8DBB8D0C93EA8DFB8DA19097
:10B02000BB24EFE8F0E0AA0CBB1CEA0DFB1DAA89CB
:10B03000BB897BE70E9469F5AA89BB898D919C91A8
:10B04000AA8DBB8DAD90BB24A9E4B5E0AA0CBB1CB6
:10B05000AA0DBB1D8D939C9387E480936B04AA8DEE
:10B06000BB8D8C9180936C0484ED80936D0483EC94
:10B0700080936E0484E0809385040E94F1120C9406
:10B080005B5A013150E0150711F00C94B758ECA150
:10B09000FDA101E0AEA5BFA50E9459F5AEA5BFA5D3
:10B0A0000E94FEF4AC8DBD8D0C93ACA1BDA10E949D
:10B0B000A7F5082F41E0041BAE8DBF8D0C9382E0F5
:10B0C000ECA1FDA1AE8DBF8D0C910A93AFA5B8A9DF
:10B0D0000E9452F5AEA5BFA50E94FEF4AA89BB89C5
:10B0E0000D931C93EC8DFD8DA190BB24E6E2F8E05E
:10B0F000AA0CBB1CEA0DFB1DAA89BB897BE70E9439
:10B1000069F5AA89BB898D919C91AC8DBD8DAD905F
:10B11000BB24A4EFB6E0AA0CBB1CAA0DBB1D8D93EB
:10B120009C93AA89BB890D911C91003050E01507B2
:10B1300011F00C94A55880E0AC8DBD8DAD90BB2472
:10B14000A2EFB6E0AA0DBB1D8C9384ED80936B0437
:10B15000AC8DBD8D8C9180936C0483EC80936D04D9
:10B1600083E0809385040E94F1120C945B5A0231B3
:10B1700050E0150711F00C94FA58ACA1BDA10E9443
:10B18000FEF4AA89BB890D931C93E2EDF4E0A19033
:10B19000BB24E6E2F0E0AA0CBB1CEA0DFB1DAA8969
:10B1A000BB897BE70E9469F5AA89BB898D919C9137
:10B1B000A2EDB4E0AD90BB24A7E2B6E0AA0CBB1CA4
:10B1C000AA0DBB1D8D939C9388E280936B0480E253
:10B1D00080936C0483E280936D0484ED80936E040D
:10B1E00083EC80936F0485E0809385040E94F112C4
:10B1F0000C945B5A033150E0150711F00C943C5944
:10B20000ACA1BDA10E94FEF4AA89BB890D931C9339
:10B21000E2EDF4E0A190BB24E0E6FFE0AA0CBB1C49
:10B22000EA0DFB1DAA89BB897BE70E9469F5AA8903
:10B23000BB898D919C91A2EDB4E0AD90BB24A0E5BB
:10B24000B6E0AA0CBB1CAA0DBB1D8D939C930E945B
:10B25000F87E8DE28093700486E28093710481E22F
:10B260008093720483EC8093730489E08093850457
:10B270000E94F1120C945B5A043150E0150711F052
:10B280000C948959ACA1BDA10E94FEF4AA89BB8986
:10B290000D931C93E2EDF4E0A190BB24E6E8FFE0FF
:10B2A000AA0CBB1CEA0DFB1DAA89BB897BE70E9487
:10B2B00069F5AA89BB898D919C91A2EDB4E0AD900E
:10B2C000BB24A6E6B6E0AA0CBB1CAA0DBB1D8D9341
:10B2D0009C9381E380936B048AE280936C0484EDF9
:10B2E00080936D0483EC80936E04AA89BB890D91D1
:10B2F0001C91003050E0150711F00C9482598AEA35
:10B3000080936E0484E0809385040E94F1120C9473
:10B310005B5A053150E0150711F00C94CB59ACA1E4
:10B32000BDA10E94FEF4AC8DBD8D0C93ACA1BDA15E
:10B330008C91AC8DBD8D8C93AC8DBD8D8C918053DB
:10B340008C93E2EDF4E0A190BB24EAE3F0E0EA0D97
:10B35000FB1DAC8DBD8D7BE70E9467F58BE2809372
:10B360006B0489E580936C0484ED80936D048FE712
:10B3700080936E04AC8DBD8D0C91003011F00C9457
:10B38000C4598DE880936E0484E0809385040E9404
:10B39000F1120C945B5A063150E0150711F00C9431
:10B3A000F759ACA1BDA10E94FEF4AA89BB890D93F7
:10B3B0001C93E9E3F0E0AA89BB897BE70E9469F569
:10B3C000AA89BB898D919C91A5E7B6E08D939C934A
:10B3D0000E94F87E84ED8093700483EC8093710466
:10B3E00087E0809385040E94F1120C945B5A083127
:10B3F00050E0150711F00C942A5AA8EDB6E0EAE9DE
:10B40000FEEE0E94DDF30E9497F1ECA1FDA1A8EDF4
:10B41000B6E00E940EF00E9447F5A8EDB6E00E944B
:10B420000EF0E2EFFDEE0E94DDF30E9497F10E9424
:10B43000167F84ED80936D0483EC80936E0484E02A
:10B44000809385040E94F112A8EDB6E00E948EF070
:10B450000C945B5A093150E0150711F00C945B5ABB
:10B46000A8EDB6E0EEE9FEEE0E94DDF30E9497F152
:10B47000ECA1FDA1A8EDB6E00E940EF00E9447F5F8
:10B48000A8EDB6E00E940EF0E2EFFDEE0E94DDF3C3
:10B490000E9497F10E94167F80E480936D0483ECF4
:10B4A00080936E0484E0809385040E94F112A8EDDD
:10B4B000B6E00E948EF00C94A37CAC85BD850C9107
:10B4C000023011F00C94FA66AA85BB850D911C918F
:10B4D000023350E0150711F00C941A5BACA1BDA12A
:10B4E0000E94A7F5082F033010F00C94795A0C94A1
:10B4F0009B7CECA1FDA102E0AEA5BFA50E9459F581
:10B50000AEA5BFA50E94FEF4AC8DBD8D0C93AC8D95
:10B51000BD8D0C91013081E008F080E08F93AC8DFF
:10B52000BD8D0C910A3580E010F009F081E09F910B
:10B53000892B882311F40C949F5A0C949B7CACA10A
:10B54000BDA10E94A7F5082F42E0041BA885B9857C
:10B550000C93ACA1BDA10E94A7F5EA2FFB2FA885F3
:10B56000B9850C913197E01BF0400FEFAEA5BFA558
:10B570000E9459F5EEA5FFA5FA93EA930E941FE2F7
:10B580002296AC8DBD8D0C91093210F00C94DB5AD3
:10B59000EC8DFD8D0191112745E050E00E948DF169
:10B5A000E7E4FCE0E00FF11FADE4B6E07BE70E94CA
:10B5B00078F50C94EC5AEC8DFD8D0191108145E0ED
:10B5C00050E00E948DF1E1E4FDE0E00FF11FADE4F9
:10B5D000B6E07BE70E9478F5AC8DBD8D8C918093B1
:10B5E000430780913E07806280933E070E94FC7C67
:10B5F000A5E8B4E08C918F5F8C9389E5A5E8B4E071
:10B60000AD90BB24AAE6B4E0AA0DBB1D8C93A5E8BF
:10B61000B4E08C918F5F8C9383ECA5E8B4E0AD909F
:10B62000BB24AAE6B4E0AA0DBB1D8C930E94F112C4
:10B630000C94F866033350E0150711F00C94465B48
:10B64000ACA1BDA10E94FEF4AC8DBD8D0C93E8E3CE
:10B65000F0E0AC8DBD8D7BE70E9467F584E08093C0
:10B66000850483ED80936B048BE880936C0485EBF9
:10B6700080936D040AEAAC8DBD8D4C91040FAEE64B
:10B68000B4E00C930E94F1120C94F8660C3350E075
:10B69000150711F00C948A5BACA1BDA10E94A7F51F
:10B6A000082F043018F011F00C94585B0C945A5B7E
:10B6B0000C949B7CACA1BDA1E4EAFDEE0E94DDF3FD
:10B6C0000E94ADF511F00C94745BA42DB52DE2EA47
:10B6D000FEEE0E94DDF30E9497F1ECE6FFE0A42D60
:10B6E000B52D7BE70E9478F5ECE6FFE0ACA1BDA1AB
:10B6F0007BE70E9478F50E94247F89E580936D04A2
:10B7000083EC80936E0484E0809385040E94F112A0
:10B710000C94F8660D3350E0150711F00C94B45BEF
:10B72000ACA1BDA10E94A7F5082F043018F011F0BC
:10B730000C949C5B0C949E5B0C949B7CEAEFFFE06A
:10B74000ACA1BDA17BE70E9478F50E94167F89E538
:10B7500080936D0483EC80936E0484E08093850471
:10B760000E94F1120C94F8660E3350E0150711F0A8
:10B770000C940E5CECA1FDA1A8EDB6E00E9447F58B
:10B7800087E10E94FAF0E8EDF6E0A881B9810E9415
:10B7900047F5A8EDB6E0E6EAFEEE0E94DDF30E9472
:10B7A00097F1E881F981A8EDB6E00E940EF00E94C1
:10B7B00047F5A8EDB6E00E940EF0E2EFFDEE0E9424
:10B7C000DDF30E9497F187E1481A8827580A2296EC
:10B7D0000E94167F81E380936D0489E280936E045A
:10B7E00086EA80936F04E8EDF6E003E0AEA5BFA51E
:10B7F0000E9459F5AEA5BFA50E94FEF4A3E4B7E0F0
:10B800000C930E94FC7C83EC809370040E94F112E4
:10B81000A8EDB6E00E948EF00C94F8660F3350E06D
:10B82000150711F00C94635CECA1FDA1A8EDB6E046
:10B830000E9447F5A8EDB6E00E94A7F5082F0F304B
:10B8400018F011F00C94265C0C94285C0C949B7CF2
:10B8500087E10E94FAF0E8EDF6E0A881B9810E9444
:10B8600047F5A8EDB6E0EAEAFEEE0E94DDF30E949D
:10B8700097F1E881F981A8EDB6E00E940EF00E94F0
:10B8800047F5A8EDB6E00E940EF0E2EFFDEE0E9453
:10B89000DDF30E9497F187E1481A8827580A22961B
:10B8A0000E94167F89E580936D0483EC80936E047B
:10B8B00084E0809385040E94F112A8EDB6E00E9416
:10B8C0008EF00C94F866003450E0150711F00C94DB
:10B8D000915CACA1BDA10E94A7F5082F0C3010F01F
:10B8E0000C94745C0C949B7CAEA5BFA5EEEAFEEEB6
:10B8F0000E94DDF30E9497F1ECA1FDA1FA93EA9377
:10B900000E940BCD2296EEA5FFA5FA93EA930E9422
:10B9100031D422968091B70380688093B7030C944A
:10B92000F866013450E0150711F00C94B45CAEA534
:10B93000BFA5EEEAFEEE0E94DDF30E9497F1ECA1B6
:10B94000FDA1FA93EA930E9480DC2296EEA5FFA562
:10B95000FA93EA930E9431D422968091B7038068CB
:10B960008093B7030C94F866023450E0150711F089
:10B970000C94C85CECA1FDA1FA93EA930E9448D90B
:10B9800022968091B70380688093B7030C94F86681
:10B99000023550E0150711F00C94EC5CACA1BDA190
:10B9A0000E94FEF4AC8DBD8D0C93E4E1F8E0AC8D0B
:10B9B000BD8D7BE70E9467F589EB80936B0485EB77
:10B9C00080936C0481EC80936D0483E08093850404
:10B9D0000E94F1120C94F866033550E0150711F03F
:10B9E0000C94125DACA1BDA10E94FEF4AC8DBD8D86
:10B9F0000C93EEEAF6E0AC8DBD8D7BE70E9467F517
:10BA000089EB80936B04AC8DBD8D8C9180936C041D
:10BA100081EC80936D0483E0809385040E94F11291
:10BA20000C94F866043550E0150711F00C94385D5D
:10BA3000ACA1BDA10E94FEF4AC8DBD8D0C93EFEACC
:10BA4000F6E0AC8DBD8D7BE70E9467F589EB8093B6
:10BA50006B0481EC80936C04AC8DBD8D8C918093D4
:10BA60006D0483E0809385040E94F1120C94F866C3
:10BA7000063550E0150711F00C94A95DACA1BDA1ED
:10BA80000E94FEF4AC8DBD8D0C93AC8DBD8D0C91E0
:10BA9000013081E008F080E08F93AC8DBD8D0C917A
:10BAA0000A3080E010F009F081E09F91892B882313
:10BAB00011F40C945D5D0C949B7CEC8DFD8D0191DB
:10BAC000112748E050E00E948DF1E9E8FFE0E00F27
:10BAD000F11FAAE1B5E07BE70E9478F5EC8DFD8DC2
:10BAE000A190BB24E0EEFFE0EA0DFB1DA3E2B5E070
:10BAF0007BE70E9467F5EC8DFD8DA190BB24EAEEFB
:10BB0000FFE0EA0DFB1DA7E2B5E07BE70E9467F5C9
:10BB1000EC8DFD8DA190BB24E5E1F8E0EA0DFB1D65
:10BB2000A5E2B5E07BE70E9467F50E94247F8AE2E8
:10BB300080936D04AC8DBD8D8C9180936E0483ECED
:10BB400080936F0485E0809385040E94F1120C9429
:10BB5000F866073550E0150711F00C940B5EACA1A8
:10BB6000BDA10E94A7F5082F013081E008F080E018
:10BB70008F93ACA1BDA10E94A7F5082F033080E0F0
:10BB800010F009F081E09F91892B882311F40C9427
:10BB9000CB5D0C949B7CACA1BDA10E94A7F5AE8DA2
:10BBA000BF8D8C93ACA1BDA10E94A7F5EA2FFB2FFE
:10BBB000AE8DBF8D0C913197E01BF0400FEFAEA51D
:10BBC000BFA50E9459F5AEA5BFA50E94FEF4AC8D9D
:10BBD000BD8D0C93AC8DBD8D8C9180937A06809138
:10BBE00026058260809326050E94247F87EB809340
:10BBF0006D0486EA80936E048BEE80936F048091CF
:10BC00007A06809343070E94FC7C0E94F1120E94F6
:10BC10000D7E0C94F866083550E0150711F00C9471
:10BC2000525EACA1BDA10E94FEF4AC8DBD8D0C9303
:10BC3000AC8DBD8D0C91013018F011F00C94225E8A
:10BC40000C94245E0C949B7CE2EDF4E0A190BB2468
:10BC5000E1E3F0E0EA0DFB1DAC8DBD8D7BE70E94BA
:10BC600067F58BE280936B0489E580936C0481EE29
:10BC700080936D0484E080936E0480E280936F046F
:10BC800081E3809370040AEAAC8DBD8D4C91040F62
:10BC9000A1E7B4E00C9387E0809385040E94F11241
:10BCA0000C94F866093550E0150711F00C94A25E6B
:10BCB000ACA1BDA10E94FEF4AC8DBD8D0C93AC8DEA
:10BCC000BD8D0C91013018F011F00C94695E0C944C
:10BCD0006B5E0C949B7CE2EDF4E0A190BB24EEE261
:10BCE000F0E0EA0DFB1DAC8DBD8D7BE70E9467F592
:10BCF000AC8DBD8D8C91A2EDB4E0AD90BB24ABE7D3
:10BD0000B6E0AA0DBB1D8C938BE280936B0489E592
:10BD100080936C0484E080936D0486E280936E04CB
:10BD200081E280936F040AEAAC8DBD8D4C91040FC3
:10BD3000A0E7B4E00C9386E0809385040E94F112A2
:10BD40000C94F8660A3550E0150711F00C94D05E9B
:10BD5000ACA1BDA10E94FEF4AC8DBD8D0C93AC8D49
:10BD6000BD8D0C91013010F00C94B85E0C949B7C4E
:10BD7000EEE2F0E0AC8DBD8D7BE70E9467F50E949E
:10BD8000EB7E8EE980936F04AC8DBD8D8C9180939A
:10BD9000700486E0809385040E94F1120C94F8668A
:10BDA0000B3550E0150711F00C94245FACA1BDA138
:10BDB0000E94FEF4AC8DBD8D0C93AC8DBD8D0C91AD
:10BDC000013018F011F00C94E75E0C94E95E0C94CD
:10BDD0009B7CE5E1F8E0AC8DBD8D7BE70E9467F5CB
:10BDE000AC8DBD8D0C91013011F00C94105FE8A169
:10BDF000F9A1A190BB24ECE9F0E0EA0DFB1DA0E164
:10BE0000BB2780E08C937BE70E9467F580E0A8A1C8
:10BE1000B9A1AD90BB24ABE1B6E0AA0DBB1D8C93DC
:10BE20000E94F87E8EEA809370040AEAAC8DBD8D84
:10BE30004C91040FA1E7B4E00C9387E08093850454
:10BE40000E94F1120C94F8660C3550E0150711F0C1
:10BE50000C947D5FECA1FDA101E0AC8DBD8D0E9435
:10BE600059F5AC8DBD8D8C9180538C93ACA1BDA147
:10BE70000E94A7F5082F41E0041BAE8DBF8D0C93E7
:10BE800082E0ECA1FDA1AE8DBF8D0C910A93AFA510
:10BE9000B8A90E9452F5AEA5BFA50E94FEF4AA8DD6
:10BEA000BB8D0C93EC8DFD8DA190BB24E9E0F0E0FF
:10BEB000EA0DFB1DAA8DBB8D7BE70E9467F5AA8D5D
:10BEC000BB8D8C91AC8DBD8DAD90BB24ABEFB6E03E
:10BED000AA0DBB1D8C9384ED80936B04AC8DBD8D3E
:10BEE0008C9180936C0483EC80936D0483E0809349
:10BEF00085040E94F1120C94F8660D3550E0150788
:10BF000011F00C94A05FE4E0F0E0ACA1BDA17BE7F0
:10BF10000E9478F581E380936B0481E380936C0445
:10BF20008DE280936D0489E580936E0483EC8093A9
:10BF30006F0485E0809385040E94F1120C94F866EA
:10BF4000043650E0150711F00C941560ECA1FDA12A
:10BF500001E0AC8DBD8D0E9459F5AC8DBD8D8C91ED
:10BF600080538C93AC8DBD8D0C91013081E008F035
:10BF700080E08F93AC8DBD8D0C91033080E010F08C
:10BF800009F081E09F91892B882311F40C94CA5FFA
:10BF90000C949B7CA889B9890E9494EFA889B989DF
:10BFA0000D911C91013050E015070CF402C00C9467
:10BFB000DB5F0C949B7CACA1BDA10E94A7F5EA2F8E
:10BFC000FB2FA889B9890C913197E01BF0400FEF46
:10BFD000AEA5BFA50E9459F5AEA5BFA50E94FEF46F
:10BFE000AA8DBB8D0C93EC8DFD8DA190BB24E5E457
:10BFF000F0E0EA0DFB1DAA8DBB8D7BE70E9467F583
:10C0000087E480936B04AC8DBD8D8C9180936C0420
:10C0100085EB80936D0483EC80936E0484E08093C1
:10C0200085040E94F1120C94F866053650E015075D
:10C0300011F00C94A860AEA5BFA50E94BFF3ECA1BF
:10C04000FDA101E0AC8DBD8D0E9459F5AC8DBD8D7B
:10C050008C9180538C93AC8DBD8D0C91013081E01F
:10C0600008F080E08F93AC8DBD8D0C91053080E0A1
:10C0700010F009F081E09F91892B882311F40C9432
:10C0800043600C949B7CA889B9890E9494EFA8898D
:10C09000B9890D911C91013050E015070CF402C0D4
:10C0A0000C9454600C949B7CACA1BDA10E94A7F59C
:10C0B000EA2FFB2FA889B9890C913197E01BF0403A
:10C0C0000FEFAEA5BFA50E9459F5AEA5BFA50E9472
:10C0D000FEF4AA8DBB8D0C93AA8DBB8D0C91013003
:10C0E00081E008F080E08F93AA8DBB8D0C910A351A
:10C0F00080E010F009F081E09F91892B882311F4F2
:10C100000C9484600C949B7CEC8DFD8DA190BB24E1
:10C11000E3EBF0E0EA0DFB1DAA8DBB8D7BE70E94EF
:10C1200067F58EE180936B0489E280936C04AC8D9B
:10C13000BD8D8C9180936D048DE880936E040E9478
:10C14000327F89E0809385040E94F1120C94F86696
:10C15000063650E0150711F00C943B61AEA5BFA563
:10C160000E94BFF3ECA1FDA101E0AC8DBD8D0E944A
:10C1700059F5AC8DBD8D8C9180538C93AC8DBD8D5C
:10C180000C91013081E008F080E08F93AC8DBD8D83
:10C190000C91053080E010F009F081E09F91892B2F
:10C1A000882311F40C94D6600C949B7CA889B989DF
:10C1B0000E9494EFA889B9890D911C91013050E03B
:10C1C00015070CF402C00C94E7600C949B7CACA1A6
:10C1D000BDA10E94A7F5EA2FFB2FA889B9890C9170
:10C1E0003197E01BF0400FEFAEA5BFA50E9459F5B7
:10C1F000AEA5BFA50E94FEF4AA8DBB8D0C93AA8D9F
:10C20000BB8D0C91013081E008F080E08F93AA8D06
:10C21000BB8D0C910A3580E010F009F081E09F9110
:10C22000892B882311F40C9417610C949B7CEC8D62
:10C23000FD8DA190BB24E8EBF0E0EA0DFB1DAA8D7B
:10C24000BB8D7BE70E9467F58EE180936B0489E2EA
:10C2500080936C04AC8DBD8D8C9180936D048FE7C1
:10C2600080936E040E94327F89E0809385040E944F
:10C27000F1120C94F866073650E0150711F00C9493
:10C280001662AEA5BFA50E94BFF3ECA1FDA102E01E
:10C29000AEA5BFA50E9459F5AEA5BFA50E94FEF4AC
:10C2A000A88DB98D0C93A88DB98D0C91013081E0CA
:10C2B00008F080E08F93A88DB98D0C91083280E052
:10C2C00010F009F081E09F91892B882311F40C94E0
:10C2D0006B610C949B7CACA1BDA10E94A7F5082FBB
:10C2E00042E0041BA885B9850C93ACA1BDA10E94B6
:10C2F000A7F5EA2FFB2FA885B9850C913197E01B94
:10C30000F0400FEFAEA5BFA50E9459F5AEA5BFA5A1
:10C310000E94A7F5A885B9858C9380E0AA8DBB8D76
:10C320008C93ACA5BDA50E94BFF381E0AC81BD811B
:10C330008C93A885B9854C91AC81BD810C91041773
:10C3400018F011F00C94E361AC81BD818C91EEA5E5
:10C35000FFA503E00A93ABA5BCA50E9452F5AAA5D0
:10C36000BBA50E94FEF4AC89BD890C93AC89BD8944
:10C370000C91003011F00C94C1618FEFAC89BD8934
:10C380008C93AC89BD898C91ACA5BDA58F930E947F
:10C390000EF08F918D9388278C93ACA5BDA50E943C
:10C3A000A7F5082F093018F011F00C94D9610C94FE
:10C3B000DB610C949B7CAC81BD818C918D5F8C93F7
:10C3C00010F40C949961E88DF98D019111274AE0E0
:10C3D00050E00E948DF1E9E2F8E0E00FF11FACA51A
:10C3E000BDA57BE70E9478F5A88DB98D8C918093CF
:10C3F000430780913E07806280933E070E94FC7C49
:10C400000E94F11284E690E00E94EBF0A3E4B7E012
:10C410000D9111274AEB50E0040F151FACE0B5E079
:10C420000D931C930E943B850C94F866083650E0EF
:10C43000150711F00C944662ACA1BDA10E94A7F5AE
:10C44000082F063018F011F00C9428620C942A6220
:10C450000C949B7CE1EBF6E0ACA1BDA17BE70E94D4
:10C4600078F50E94EB7E8DE280936F048FE28093DB
:10C47000700482E28093710483EC8093720488E0FC
:10C48000809385040E94F1120C94F866093650E0FE
:10C49000150711F00C94C962AEA5BFA50E94BFF3A9
:10C4A000ECA1FDA102E0AEA5BFA50E9459F5AEA585
:10C4B000BFA50E94FEF4A88DB98D0C93A88DB98DEF
:10C4C0000C91013081E008F080E08F93A88DB98D48
:10C4D0000C91043180E010F009F081E09F91892BEC
:10C4E000882311F40C9476620C949B7CACA1BDA1C2
:10C4F0000E94A7F5082F42E0041BA885B9850C937C
:10C50000ACA1BDA10E94A7F5EA2FFB2FA885B98594
:10C510000C913197E01BF0400FEFAEA5BFA50E9434
:10C5200059F5AEA5BFA50E94A7F5A885B9858C933E
:10C53000A885B9850C910A3018F011F00C94A2620C
:10C540000C94A4620C949B7CE88DF98D01911127C9
:10C550004BE050E00E948DF1E1EBF6E0E00FF11FBF
:10C56000AEA5BFA57BE70E9478F50E94EB7E86EA28
:10C5700080936F04A88DB98D8C918093700483ECA7
:10C580008093710487E0809385040E94F1120C94DB
:10C59000F8660A3650E0150711F00C94EF62ACA172
:10C5A000BDA10E94FEF4AC8DBD8D0C93EAEBF6E0CC
:10C5B000AC8DBD8D7BE70E9467F50E94EB7E8BEA18
:10C5C00080936F0482ED8093700483EC80937104F8
:10C5D00087E0809385040E94F1120C94F8660B3674
:10C5E00050E0150711F00C941563ACA1BDA10E9499
:10C5F000FEF4AC8DBD8D0C93EBEBF6E0AC8DBD8DF8
:10C600007BE70E9467F50E94EB7E8AEA80936F04C5
:10C6100082ED8093700483EC8093710487E08093B3
:10C6200085040E94F1120C94F8660C3650E0150750
:10C6300011F00C945B63ACA1BDA10E94A7F5082F7B
:10C64000033018F011F00C9427630C9429630C94B8
:10C650009B7CACA1BDA1E4EAFDEE0E94DDF30E944B
:10C66000ADF511F00C943863ACA1BDA10E94BFF3ED
:10C67000E0E0F0E0ACA1BDA17BE70E9478F580E2AC
:10C6800080936B048AE280936C0481E280936D0452
:10C690008DE280936E048FE280936F0482E2809338
:10C6A000700483EC8093710487E0809385040E947A
:10C6B000F1120C94F8660D3650E0150711F00C9449
:10C6C000A163ACA1BDA10E94A7F5082F043018F00A
:10C6D00011F00C946D630C946F630C949B7CACA173
:10C6E000BDA1E4EAFDEE0E94DDF30E94ADF511F07C
:10C6F0000C947E63ACA1BDA10E94BFF3EEE2F8E012
:10C70000ACA1BDA17BE70E9478F58DE280936B041C
:10C7100084E280936C048AE280936D048DE28093BE
:10C720006E048FE280936F0482E28093700483EC46
:10C730008093710487E0809385040E94F1120C9429
:10C74000F8660E3650E0150711F00C946A64ACA13F
:10C75000BDA10E94A7F5082F023010F00C94B2631F
:10C760000C949B7CECA1FDA101E0AC8DBD8D0E94E1
:10C7700059F5AC8DBD8D8C9180538C93AC8DBD8D56
:10C780000C91013081E008F080E08F93AC8DBD8D7D
:10C790000C91033080E010F009F081E09F91892B2B
:10C7A000882311F40C94D6630C949B7CACA1BDA19E
:10C7B0000E94A7F5A88DB98D8C93A88DB98D0C9189
:10C7C00041E0041BA885B9850C93ACA1BDA10E94D2
:10C7D000A7F5EA2FFB2FA885B9850C913197E01BAF
:10C7E000F0400FEFAEA5BFA50E9459F5AEA5BFA5BD
:10C7F0000E94FEF4AA8DBB8D0C93AA8DBB8D0C916B
:10C80000013081E008F080E08F93AA8DBB8D0C9100
:10C81000083280E010F009F081E09F91892B882395
:10C8200011F40C9415640C949B7C0091D20401309B
:10C8300011F00C942A64EC8DFD8DA190BB24EBE7E4
:10C84000FFE0EA0DFB1DAA8DBB8D7BE70E9467F51B
:10C850000C944E64023011F00C943D64EC8DFD8D0F
:10C86000A190BB24EEE7FFE0EA0DFB1DAA8DBB8D76
:10C870007BE70E9467F50C944E64033011F00C9432
:10C880004E64EC8DFD8DA190BB24E1E8FFE0EA0D44
:10C89000FB1DAA8DBB8D7BE70E9467F585EB80931E
:10C8A0006B048091D20480936C0481E380936D04C7
:10C8B0008AE280936E04AC8DBD8D8C9180936F0461
:10C8C00083EC8093700486E0809385040E94F112CB
:10C8D0000C94F8660F3650E0150711F00C94B6640E
:10C8E000ACA1BDA10E94FEF4AC8DBD8D0C93AC8DAE
:10C8F000BD8D0C91033018F011F00C9481640C94F0
:10C9000083640C949B7CE2EDF4E0A190BB24E4E80A
:10C91000FFE0EA0DFB1DAC8DBD8D7BE70E9467F546
:10C9200085EB80936B048091D20480936C0481E347
:10C9300080936D048AE280936E0481EC80936F048F
:10C94000AC8DBD8D8C9180937004AC8DBD8D0C91A0
:10C95000003011F00C94AF648AEA8093700486E092
:10C96000809385040E94F1120C94F866003750E021
:10C97000150711F00C94FF64ACA1BDA10E94FEF458
:10C98000AC8DBD8D0C93AC8DBD8D0C910E3F18F010
:10C9900011F00C94CD640C94CF640C949B7CE2ED6C
:10C9A000F4E0A190BB24EDE8FFE0EA0DFB1DAC8DA7
:10C9B000BD8D7BE70E9467F5AC8DBD8D8C91A2ED9E
:10C9C000B4E0AD90BB24A0E7B6E0AA0DBB1D8C93EC
:10C9D00085EB80936B048091D20480936C0481E397
:10C9E00080936D048AE280936E0484E780936F04E1
:10C9F00085E0809385040E94F1120C94F86601375B
:10CA000050E0150711F00C945365ACA1BDA10E9434
:10CA1000FEF4AC8DBD8D0C93AC8DBD8D0C910130B1
:10CA200018F011F00C9416650C9418650C949B7C0E
:10CA3000E2EDF4E0A190BB24E4E3F0E0EA0DFB1D9D
:10CA4000AC8DBD8D7BE70E9467F5AC8DBD8D8C9163
:10CA5000A2EDB4E0AD90BB24AAE8B6E0AA0DBB1DE0
:10CA60008C9385EB80936B048091D20480936C044B
:10CA700082EA80936D048DEB80936E0486E280934E
:10CA80006F0481E2809370040AEAAC8DBD8D4C91F5
:10CA9000040FA1E7B4E00C9387E0809385040E9423
:10CAA000F1120C94F866023750E0150711F00C945F
:10CAB0009765ACA1BDA10E94FEF4AA89BB890D9324
:10CAC0001C93AA89BB898D919C91A2EDB4E0AD9095
:10CAD000BB24AFE7B6E0AA0CBB1CAA0DBB1D8D930F
:10CAE0009C93E2EDF4E0A190BB24EEE1F8E0AA0C07
:10CAF000BB1CEA0DFB1DAA89BB897BE70E9469F577
:10CB000085EB80936B048091D20480936C0489E35D
:10CB100080936D0487EB80936E0483EC80936F04A5
:10CB200085E0809385040E94F1120C94F866033727
:10CB300050E0150711F00C940D66ECA1FDA103E087
:10CB4000AEA5BFA50E9459F5ACA1BDA10E94A7F555
:10CB5000082F43E0041BAE8DBF8D0C93EEA5FFA5FF
:10CB6000A8EDB6E00E9447F584E0ECA1FDA1AE8DF2
:10CB7000BF8D0C910A93A8EDB6E00E940EF00E94C2
:10CB800052F587E10E94FAF0E8EDF6E0A881B9815C
:10CB90000E9447F5A8EDB6E0E2EBFEEE0E94DDF361
:10CBA0000E9497F1E881F981A8EDB6E00E940EF0AD
:10CBB0000E9447F5A8EDB6E00E940EF0E2EFFDEE10
:10CBC0000E94DDF30E9497F187E1481A8827580AEE
:10CBD000229685E0809385040E94167F8AE28093E6
:10CBE0006D0483EC80936E0486EA80936F04AEA597
:10CBF000BFA50E94FEF4A3E4B7E00C9380913E072A
:10CC00008F7D80933E070E94FC7C0E94F112A8ED6C
:10CC1000B6E00E948EF00C94F866043750E01507D9
:10CC200011F00C944F66ACA1BDA10E94FEF4AC8D36
:10CC3000BD8D0C93ACA1BDA10E94A7F5082F0330B8
:10CC400018F011F00C9426660C9428660C949B7CCA
:10CC5000E6E2F8E0AC8DBD8D7BE70E9467F5AC8D18
:10CC6000BD8D8C918093F2060E94167F89E380939C
:10CC70006D048BEA80936E0485EB80936F04AC8D1A
:10CC8000BD8D8C918093430780913E078F7D80936B
:10CC90003E070E94FC7C0E94F1120C94F866053756
:10CCA00050E0150711F00C947266ACA1BDA10E9472
:10CCB000FEF4AC8DBD8D0C93E5EFFFE0AC8DBD8D2A
:10CCC0007BE70E9467F50E94EB7E85EB80936F0403
:10CCD00083EC8093700486E0809385040E94F112B7
:10CCE0000C94F866063750E0150711F00C94A16615
:10CCF000ACA1BDA10E94FEF4AC8DBD8D0C93AC8D9A
:10CD0000BD8D0C910A3518F011F00C9489660C94C5
:10CD10008B660C949B7CE6EFFFE0AC8DBD8D7BE7D2
:10CD20000E9467F50E94EB7E84E980936F0483EC98
:10CD30008093700486E0809385040E94F1120C9425
:10CD4000F866073750E0150711F00C94E166ACA1C6
:10CD5000BDA10E94FEF4AC8DBD8D0C93AC8DBD8D3C
:10CD60000C91013018F011F00C94B8660C94BA666E
:10CD70000C949B7CE9EBF6E0AC8DBD8D7BE70E94CB
:10CD800067F583E280936B048EE180936C048BE201
:10CD900080936D048EE580936E048AEA80936F041D
:10CDA000AC8DBD8D0C91013011F00C94DA668BEADC
:10CDB00080936F0485E0809385040E94F1120C94A7
:10CDC000F866073E53E0150711F00C94EB660E94DD
:10CDD00093EB0C94F866073C50E0150711F00C94A7
:10CDE000F86685E680935304E5E0F0E00E943CF0AD
:10CDF0000C94A37CAC85BD850C91033011F00C9490
:10CE0000526C81E0A881B9818C93A881B9810C9181
:10CE1000043018F011F00C942167A881B981AD900D
:10CE2000BB24A2E4B7E0AA0CBB1CAA0DBB1D0E9448
:10CE3000BFF3A881B9818C918F5F8C9310F40C940F
:10CE4000056781E0AA8DBB8D8C93AA8DBB8D9C91CB
:10CE50009A93ADA1BEA1E6EBFEEE0E94DDF32FEFAB
:10CE60000E94B6F1A88DB98D0C93A88DB98D0C9147
:10CE7000003018F011F00C943F670C94E367AE8516
:10CE8000BF850E94BFF381E0AA8DBB8D8C93AA8DD4
:10CE9000BB8D9C919A93ADA1BEA1E6EBFEEE0E94E4
:10CEA000DDF32FEF0E94B6F1A88DB98D0C93A88DFC
:10CEB000B98D0C91003011F00C947467A889B98970
:10CEC0004D915C91AA8DBB8D0D911127041715070B
:10CED0000CF402C00C947467A889B9890C9141E0E4
:10CEE000040FA88DB98D0C93A88DB98D0C910030CD
:10CEF00018F011F00C947E670C94CD67A88DB98D55
:10CF00000C91AA8DBB8D4C91041BAAA1BBA10C93C3
:10CF1000AA8DBB8D8C91ECA1FDA1AAA1BBA10C9106
:10CF20000A93AFA5B8A90E9452F5AAA1BBA10C9182
:10CF3000003011F00C94A067AEA5BFA50E94BFF30E
:10CF4000A88DB98D0C9141E0040FAA8DBB8D0C9377
:10CF5000AE85BF850E948DEFAE85BF850D911C917A
:10CF6000043050E015071CF011F00C94B9670C94D4
:10CF7000BB670C94E167AEA5BFA50E94FEF4AE8529
:10CF8000BF85AD90BC90A2E4B7E0AA0CBB1CAA0D73
:10CF9000BB1D0D931C930C94D367A889B9898C9100
:10CFA000AA8DBB8D8C93A889B9894D915C91AA8D6E
:10CFB000BB8D0D911127041715070CF002C00C94BE
:10CFC00047670C94626880E0AC8DBD8D8C93A88916
:10CFD000B9890D911C910C3050E0150781E009F0E2
:10CFE00080E08F93A889B9890D911C91003150E0A0
:10CFF000150781E009F080E09F91892B882311F4C7
:10D000000C94066881E0AC8DBD8D8C93AC8DBD8D8C
:10D010000C91003011F00C940F680C949B7CA88943
:10D02000B9890D911C9144E050E00E94C5EFAE8596
:10D03000BF854D935C9381E0A881B9818C93AE85C7
:10D04000BF854D915C91A881B9810D91112704177D
:10D0500015071CF011F00C946268A881B9810C913D
:10D0600044E0049FAA81BB810C92AA81BB818C9170
:10D0700084508C93AA81BB818C918F5F8C93AA8101
:10D08000BB818C91ECA1FDA104E00A93AFA5B8A9E6
:10D090000E9452F5AEA5BFA50E94FEF4A881B981F9
:10D0A000AD90BB24A2E4B7E0AA0CBB1CAA0DBB1D2B
:10D0B0000D931C93A881B9818C918F5F8C9310F490
:10D0C0000C941F68AA85BB850D911C91053650E014
:10D0D000150780E00CF081E08F93AA85BB850D9148
:10D0E0001C910E3650E0150781E014F009F080E045
:10D0F0009F918923882311F40C945269AA85BB85DA
:10D100000D911C9144E650E0041B150BAA89BB89C4
:10D110000D931C930091D204013011F00C94CE6851
:10D12000EA89FB89A190B080ECECF4E0AA0CBB1C6E
:10D13000EA0DFB1DA4E4B7E07BE70E9469F5EA89EC
:10D14000FB89A190B080ECEBF5E0AA0CBB1CEA0DCA
:10D15000FB1DA6E4B7E07BE70E9469F5EA89FB893D
:10D16000A190B080ECEEF2E0AA0CBB1CEA0DFB1D16
:10D17000A8E4B7E07BE70E9469F5EA89FB89A19002
:10D18000B080E8E2F3E0AA0CBB1CEA0DFB1DAAE4A8
:10D19000B7E07BE70E9469F50C945069023011F00A
:10D1A0000C941069EA89FB89A190B080E0EEF4E06C
:10D1B000AA0CBB1CEA0DFB1DA4E4B7E07BE70E94B0
:10D1C00069F5EA89FB89A190B080E0EDF5E0AA0C51
:10D1D000BB1CEA0DFB1DA6E4B7E07BE70E9469F5E6
:10D1E000EA89FB89A190B080E0E0F3E0AA0CBB1CC7
:10D1F000EA0DFB1DA8E4B7E07BE70E9469F5EA8928
:10D20000FB89A190B080ECE3F3E0AA0CBB1CEA0D13
:10D21000FB1DAAE4B7E07BE70E9469F50C94506916
:10D22000033011F00C945069EA89FB89A190B08019
:10D23000E4EFF4E0AA0CBB1CEA0DFB1DA4E4B7E08C
:10D240007BE70E9469F5EA89FB89A190B080E4EE52
:10D25000F5E0AA0CBB1CEA0DFB1DA6E4B7E07BE7DA
:10D260000E9469F5EA89FB89A190B080E4E1F3E0CE
:10D27000AA0CBB1CEA0DFB1DA8E4B7E07BE70E94EB
:10D2800069F5EA89FB89A190B080E0E5F3E0AA0C9A
:10D29000BB1CEA0DFB1DAAE4B7E07BE70E9469F521
:10D2A0000C94206CAA85BB850D911C91093C50E023
:10D2B000150780E00CF081E08F93AA85BB850D9166
:10D2C0001C91023D50E0150781E014F009F080E068
:10D2D0009F918923882311F40C94426AAA85BB8507
:10D2E0000D911C9148EC50E0041B150BAA89BB89D9
:10D2F0000D931C930091D204013011F00C94BE697F
:10D30000EA89FB89A190B080E8E0F5E0AA0CBB1C9B
:10D31000EA0DFB1DA4E4B7E07BE70E9469F5EA890A
:10D32000FB89A190B080E8EFF5E0AA0CBB1CEA0DE8
:10D33000FB1DA6E4B7E07BE70E9469F5EA89FB895B
:10D34000A190B080E4E6F3E0AA0CBB1CEA0DFB1D43
:10D35000A8E4B7E07BE70E9469F5EA89FB89A19020
:10D36000B080E0EAF3E0AA0CBB1CEA0DFB1DAAE4C6
:10D37000B7E07BE70E9469F50C94406A023011F037
:10D380000C94006AEA89FB89A190B080ECE1F5E099
:10D39000AA0CBB1CEA0DFB1DA4E4B7E07BE70E94CE
:10D3A00069F5EA89FB89A190B080ECE0F6E0AA0C6F
:10D3B000BB1CEA0DFB1DA6E4B7E07BE70E9469F504
:10D3C000EA89FB89A190B080E8E7F3E0AA0CBB1CD6
:10D3D000EA0DFB1DA8E4B7E07BE70E9469F5EA8946
:10D3E000FB89A190B080E4EBF3E0AA0CBB1CEA0D32
:10D3F000FB1DAAE4B7E07BE70E9469F50C94406A44
:10D40000033011F00C94406AEA89FB89A190B08046
:10D41000E0E3F5E0AA0CBB1CEA0DFB1DA4E4B7E0B9
:10D420007BE70E9469F5EA89FB89A190B080E0E280
:10D43000F6E0AA0CBB1CEA0DFB1DA6E4B7E07BE7F7
:10D440000E9469F5EA89FB89A190B080ECE8F3E0DD
:10D45000AA0CBB1CEA0DFB1DA8E4B7E07BE70E9409
:10D4600069F5EA89FB89A190B080E8ECF3E0AA0CA9
:10D47000BB1CEA0DFB1DAAE4B7E07BE70E9469F53F
:10D480000C94206CAA85BB850D911C910D3251E046
:10D49000150780E00CF081E08F93AA85BB850D9184
:10D4A0001C91063351E0150781E014F009F080E08B
:10D4B0009F918923882311F40C94326BAA85BB8534
:10D4C0000D911C914CE251E0041B150BAA89BB89FC
:10D4D0000D931C930091D204013011F00C94AE6AAC
:10D4E000EA89FB89A190B080E4E4F5E0AA0CBB1CBA
:10D4F000EA0DFB1DA4E4B7E07BE70E9469F5EA8929
:10D50000FB89A190B080E4E3F6E0AA0CBB1CEA0D15
:10D51000FB1DA6E4B7E07BE70E9469F5EA89FB8979
:10D52000A190B080ECEDF3E0AA0CBB1CEA0DFB1D52
:10D53000A8E4B7E07BE70E9469F5EA89FB89A1903E
:10D54000B080E8E1F4E0AA0CBB1CEA0DFB1DAAE4E4
:10D55000B7E07BE70E9469F50C94306B023011F064
:10D560000C94F06AEA89FB89A190B080E8E5F5E0C7
:10D57000AA0CBB1CEA0DFB1DA4E4B7E07BE70E94EC
:10D5800069F5EA89FB89A190B080E8E4F6E0AA0C8D
:10D59000BB1CEA0DFB1DA6E4B7E07BE70E9469F522
:10D5A000EA89FB89A190B080E0EFF3E0AA0CBB1CF4
:10D5B000EA0DFB1DA8E4B7E07BE70E9469F5EA8964
:10D5C000FB89A190B080ECE2F4E0AA0CBB1CEA0D50
:10D5D000FB1DAAE4B7E07BE70E9469F50C94306B71
:10D5E000033011F00C94306BEA89FB89A190B08074
:10D5F000ECE6F5E0AA0CBB1CEA0DFB1DA4E4B7E0C9
:10D600007BE70E9469F5EA89FB89A190B080ECE58F
:10D61000F6E0AA0CBB1CEA0DFB1DA6E4B7E07BE715
:10D620000E9469F5EA89FB89A190B080E4E0F4E00A
:10D63000AA0CBB1CEA0DFB1DA8E4B7E07BE70E9427
:10D6400069F5EA89FB89A190B080E0E4F4E0AA0CD6
:10D65000BB1CEA0DFB1DAAE4B7E07BE70E9469F55D
:10D660000C94206CAA85BB850D911C91013951E069
:10D67000150780E00CF081E08F93AA85BB850D91A2
:10D680001C910A3951E0150781E014F009F080E09F
:10D690009F918923882311F40C94206CAA85BB8563
:10D6A0000D911C9140E951E0041B150BAA89BB891F
:10D6B0000D931C930091D204013011F00C949E6BD9
:10D6C000EA89FB89A190B080E0E8F5E0AA0CBB1CD8
:10D6D000EA0DFB1DA4E4B7E07BE70E9469F5EA8947
:10D6E000FB89A190B080E0E7F6E0AA0CBB1CEA0D34
:10D6F000FB1DA6E4B7E07BE70E9469F5EA89FB8998
:10D70000A190B080E4E5F4E0AA0CBB1CEA0DFB1D7F
:10D71000A8E4B7E07BE70E9469F5EA89FB89A1905C
:10D72000B080E0E9F4E0AA0CBB1CEA0DFB1DAAE402
:10D73000B7E07BE70E9469F50C94206C023011F091
:10D740000C94E06BEA89FB89A190B080E4E9F5E0F4
:10D75000AA0CBB1CEA0DFB1DA4E4B7E07BE70E940A
:10D7600069F5EA89FB89A190B080E4E8F6E0AA0CAB
:10D77000BB1CEA0DFB1DA6E4B7E07BE70E9469F540
:10D78000EA89FB89A190B080E8E6F4E0AA0CBB1C12
:10D79000EA0DFB1DA8E4B7E07BE70E9469F5EA8982
:10D7A000FB89A190B080E4EAF4E0AA0CBB1CEA0D6E
:10D7B000FB1DAAE4B7E07BE70E9469F50C94206C9E
:10D7C000033011F00C94206CEA89FB89A190B080A1
:10D7D000E8EAF5E0AA0CBB1CEA0DFB1DA4E4B7E0E7
:10D7E0007BE70E9469F5EA89FB89A190B080E8E9AE
:10D7F000F6E0AA0CBB1CEA0DFB1DA6E4B7E07BE734
:10D800000E9469F5EA89FB89A190B080ECE7F4E019
:10D81000AA0CBB1CEA0DFB1DA8E4B7E07BE70E9445
:10D8200069F5EA89FB89A190B080E8EBF4E0AA0CE5
:10D83000BB1CEA0DFB1DAAE4B7E07BE70E9469F57B
:10D8400080E280936B0481E380936C04AA89BB8996
:10D850008C9180936D0480E380936E0482E28093C8
:10D860006F0484E280937004AA85BB850D911C919E
:10D8700044E650E00E94C5EFAA89BB894D935C93B2
:10D88000AA89BB898C91809371048CE28093720485
:10D8900088E28093730489E0809385040E94F112EA
:10D8A0000C94A37CAC85BD850C91043011F00C94D4
:10D8B0007172AA85BB850D911C91013050E015074E
:10D8C00011F00C94816DACA1BDA10E94A7F5082FA9
:10D8D000093010F00C946E6C0C949B7C81E0ECA1F0
:10D8E000FDA102E00A93AFA5B8A90E9452F5AEA52A
:10D8F000BFA50E94FEF4AC8DBD8D0C93AC8DBD8D8B
:10D900000C91013081E008F080E08F93AC8DBD8DEB
:10D910000C91043180E010F009F081E09F91892B97
:10D92000882311F40C94966C0C949B7CACA1BDA143
:10D930000E94A7F5082F093011F00C94C56C83E004
:10D94000ECA1FDA101E00A93AFA5B8A90E9452F590
:10D9500084E0ECA1FDA102E00A93ADA5BEA50E9462
:10D9600052F586E0ECA1FDA102E00A93ABA5BCA5AF
:10D970000E9452F588E0ECA1FDA102E00A93AFA15C
:10D98000B8A50E9452F50C94E96C83E0ECA1FDA1CE
:10D9900002E00A93AFA5B8A90E9452F585E0ECA178
:10D9A000FDA102E00A93ADA5BEA50E9452F587E055
:10D9B000ECA1FDA102E00A93ABA5BCA50E9452F523
:10D9C00089E0ECA1FDA102E00A93AFA1B8A50E94F5
:10D9D00052F5AEA5BFA50E94FEF4AA8DBB8D0C9397
:10D9E000ACA5BDA50E94FEF4A88DB98D0C93AAA587
:10D9F000BBA50E94FEF4AE89BF890C93AEA1BFA166
:10DA00000E94FEF4AC89BD890C93EC8DFD8DA19034
:10DA1000BB24E9E8F2E0EA0DFB1DAA8DBB8D7BE794
:10DA20000E9467F5ACA5BDA5E8EBFEEE0E94DDF314
:10DA30000E94ADF511F00C94216D8EEFA88DB98D7B
:10DA40008C93EC8DFD8DA190BB24EDE9F2E0EA0D05
:10DA5000FB1DA88DB98D7BE70E9467F5AE89BF8954
:10DA60000C910B3318F011F00C94386D0C943A6D46
:10DA70000C949B7CEC8DFD8DA190BB24E1EBF2E03E
:10DA8000EA0DFB1DAE89BF897BE70E9467F5AC8973
:10DA9000BD890C91013081E008F080E08F93AC8962
:10DAA000BD890C910A3580E010F009F081E09F916A
:10DAB000892B882311F40C945F6D0C949B7CEC8D66
:10DAC000FD8DA190BB24E5ECF2E0EA0DFB1DAC89D5
:10DAD000BD897BE70E9467F583EC80936B0484EB40
:10DAE00080936C04AC8DBD8D8C9180936D0483EC20
:10DAF00080936E0484E0809385040E94F1120C945C
:10DB00006F72023050E0150711F00C94D06EACA18A
:10DB1000BDA10E94A7F5082F053010F00C94926D5E
:10DB20000C949B7C81E0ECA1FDA102E00A93AFA5DF
:10DB3000B8A90E9452F5AEA5BFA50E94FEF4A88D1B
:10DB4000B98D0C93A88DB98D0C91013081E008F04E
:10DB500080E08F93A88DB98D0C910A3580E010F08C
:10DB600009F081E09F91892B882311F40C94BA6D00
:10DB70000C949B7CACA1BDA10E94A7F5082F42E0AC
:10DB8000041BA885B9850C93ACA1BDA10E94A7F583
:10DB9000EA2FFB2FA885B9850C913197E01BF04047
:10DBA0000FEFAEA5BFA50E9459F5AEA5BFA50E9477
:10DBB000A7F5A885B9858C9380E0AA8DBB8D8C9341
:10DBC000ACA5BDA50E94BFF381E0AC81BD818C9363
:10DBD000A885B9854C91AC81BD810C91041718F0D2
:10DBE00011F00C944F6EAC81BD818C91EEA5FFA518
:10DBF00003E00A93ABA5BCA50E9452F5AAA5BBA55C
:10DC00000E94FEF4AA89BB890D931C93AA89BB8943
:10DC10000D911C910F3F50E0150711F00C94126EFE
:10DC20000C949B7CAA89BB890D911C910E3F50E0FE
:10DC300015071CF011F00C941F6E0C94356E8FEFCD
:10DC4000ACA5BDA58F930E940EF08F918D93882770
:10DC50008C93AA89BB890D911C914FEF50E0041B56
:10DC6000150BAA89BB890D931C93AA89BB898C913A
:10DC7000AC89BD898C93AC89BD898C91ACA5BDA5BF
:10DC80008F930E940EF08F918D9388278C93AC8197
:10DC9000BD818C918D5F8C9310F40C94E86DA88DF0
:10DCA000B98D0C91093210F00C94776EACA5BDA51E
:10DCB0000E94A7F5082F0F3018F011F00C94626E37
:10DCC0000C94646E0C949B7CE88DF98D0191112766
:10DCD00040E150E00E948DF1ECEBF9E0E00FF11F24
:10DCE000ACA5BDA57BE70E9478F50C949E6EACA513
:10DCF000BDA50E94A7F5082F043018F011F00C9470
:10DD0000836E0C94856E0C949B7CA88DB98D0C91C0
:10DD100048E2041BAC8DBD8D0C93EC8DFD8D019103
:10DD2000112745E050E00E948DF1EFE0FDE0E00FAB
:10DD3000F11FACA5BDA57BE70E9478F5A88DB98D34
:10DD40008C918093430780913E07806280933E07C9
:10DD5000A1E0B1E08C9186FB16F40C94B16E0E94A8
:10DD6000FC7CA5E8B4E08C918F5F8C9383ECA5E8F4
:10DD7000B4E0AD90BB24AAE6B4E0AA0DBB1D8C9321
:10DD8000A1E0B1E08C9186FB16F40C94C96E0E9460
:10DD9000F1128091B70380688093B7030C946F727F
:10DDA000033050E0150711F00C944F6FACA1BDA1EA
:10DDB0000E94FEF4AC8DBD8D0C93AC8DBD8D0C918D
:10DDC000013081E008F080E08F93AC8DBD8D0C9127
:10DDD0000A3580E010F009F081E09F91892B8823BB
:10DDE00011F40C94F56E0C949B7CAC8DBD8D0C9154
:10DDF000093210F00C94176FA42DB52DECEBFEEE4C
:10DE00000E94DDF30E9497F1EC8DFD8D01911127A9
:10DE100040E150E00E948DF1ECEBF9E0E00FF11FE2
:10DE2000A42DB52D7BE70E9478F50C94306FA42DBE
:10DE3000B52DECEBFEEE0E94DDF30E9497F1EC8D28
:10DE4000FD8D0191108145E050E00E948DF1E7E4E5
:10DE5000FCE0E00FF11FA42DB52D7BE70E9478F5C3
:10DE6000AC8DBD8D8C918093430780913E0780627D
:10DE700080933E070E94FC7CA5E8B4E08C918F5F04
:10DE80008C9387E5A5E8B4E0AD90BB24AAE6B4E0A6
:10DE9000AA0DBB1D8C930E94F1120C946F7204307A
:10DEA00050E0150711F00C94C36F81E0AC8DBD8D6F
:10DEB0008C93AC8DBD8D0C91083218F011F00C9440
:10DEC000826FA42DB52DECEBFEEE0E94DDF30E94D7
:10DED00097F1EC8DFD8D0191112740E150E00E94FA
:10DEE0008DF1ECEBF9E0E00FF11FA42DB52D7BE7F0
:10DEF0000E9478F5AC8DBD8D8C918F5F8C9310F462
:10DF00000C94596F81E0AC8DBD8D8C93AC8DBD8D23
:10DF10000C91023318F011F00C94AF6FA42DB52DB5
:10DF2000ECEBFEEE0E94DDF30E9497F1EC8DFD8D8F
:10DF30000191112745E050E00E948DF1EFE0FDE0F6
:10DF4000E00FF11FA42DB52D7BE70E9478F5AC8D75
:10DF5000BD8D8C918F5F8C9310F40C94866F8091A3
:10DF60003E07806280933E070E94FC7C87E5809399
:10DF700070048CE38093710487E0809385040E9491
:10DF8000F1120C946F72053050E0150711F00C94EB
:10DF90005970ACA1BDA10E94A7F5082F033010F065
:10DFA0000C94D46F0C949B7C81E0ECA1FDA102E069
:10DFB0000A93AFA5B8A90E9452F5AEA5BFA50E94CD
:10DFC000FEF4A88DB98D0C93A88DB98D0C910130FC
:10DFD00081E008F080E08F93A88DB98D0C910A350F
:10DFE00080E010F009F081E09F91892B882311F4E3
:10DFF0000C94FC6F0C949B7CACA1BDA10E94A7F576
:10E00000082F42E0041BA885B9850C93ACA1BDA1E3
:10E010000E94A7F5EA2FFB2FA885B9850C913197AF
:10E02000E01BF0400FEFAEA5BFA50E9459F5AEA5CD
:10E03000BFA50E94FEF4AA8DBB8D0C93E88DF98DCF
:10E04000A190BB24E7E0FFE0EA0DFB1DAA8DBB8D8C
:10E050007BE70E9467F5A88DB98D8C91809343076B
:10E0600080913E07806280933E070E94FC7CA5E879
:10E07000B4E08C918F5F8C9385EBA5E8B4E0AD9014
:10E08000BB24AAE6B4E0AA0DBB1D8C93A5E8B4E0BE
:10E090008C918F5F8C9383ECA5E8B4E0AD90BB24AA
:10E0A000AAE6B4E0AA0DBB1D8C930E94F1120C9459
:10E0B0006F72063050E0150711F00C94A17081E0EA
:10E0C000AC8DBD8D8C93AC8DBD8D0C910A3518F047
:10E0D00011F00C948270EC8DFD8DA190BB24E7E0D3
:10E0E000FFE0EA0DFB1DA0E1BB278BE78C937BE7EC
:10E0F0000E9467F5AC8DBD8D8C918F5F8C9310F471
:10E100000C9463708AE280936B048EE180936C04BC
:10E1100080E280936D048FE280936E048CE28093A2
:10E120006F0485EB8093700487E5809371048CE322
:10E130008093720488E0809385040E94F1120C940D
:10E140006F72073050E0150711F00C94F67081E003
:10E15000AC8DBD8D8C93AC8DBD8D0C91043118F0C0
:10E1600011F00C94E370EC8DFD8DA190BB24EDE9D2
:10E17000F2E0EA0DFB1DA0E1BB2789E18C937BE770
:10E180000E9467F5EC8DFD8DA190BB24E9EDF2E0D6
:10E19000EA0DFB1DA0E1BB2780E08C937BE70E948A
:10E1A00067F580E0AC8DBD8DAD90BB24A4E5B4E0F7
:10E1B000AA0DBB1D8C93AC8DBD8D8C918F5F8C9304
:10E1C00010F40C94AB7083EC80936B0484EB80931D
:10E1D0006C0487E580936D048CE380936E0484E087
:10E1E000809385040E94F1120C946F72083050E005
:10E1F000150711F00C944B72ACA1BDA10E94FEF466
:10E20000AC8DBD8D0C93AC8DBD8D0C910A3518F085
:10E2100011F00C940D710C940F710C949B7C8091F7
:10E220003E07806280933E07AC8DBD8D8C918093BC
:10E2300043070E94FC7C0E94F112AC8DBD8D0C91B5
:10E24000003018F011F00C9427710C944D71AC8DC6
:10E25000BD8D0C91093210F00C944D71EC8DFD8D3B
:10E260000191112740E150E00E948DF1ECEBF9E0C3
:10E27000E00FF11FA0E1B4E09FE00E948DF5AE8DAC
:10E28000BF8D0C910F3018F011F00C9449710C9463
:10E290004D718FE0AE8DBF8D8C93AC8DBD8D0C918B
:10E2A000083218F011F00C9457710C947D71AC8DFC
:10E2B000BD8D0C910B3510F00C947D71EC8DFD8DA6
:10E2C0000191108145E050E00E948DF1E7E4FCE00F
:10E2D000E00FF11FA0E1B4E094E00E948DF5AE8D57
:10E2E000BF8D0C91043018F011F00C9479710C94DE
:10E2F0007D7184E0AE8DBF8D8C93A0E1B4E00E946F
:10E30000A7F5AE8DBF8D8C93AE8DBF8D0C91003077
:10E3100018F011F00C948E710C94497281E0A8856C
:10E32000B9858C93A885B9858C91E0E1F4E001E092
:10E330000A93AAE4B4E00E9452F5AAE4B4E08C91F6
:10E34000A9E4B4E08C93A9E4B4E08C91A889B989DC
:10E350008D9388278C93A885B9858C918F5F8C933A
:10E36000009149040F3F11F00C94DA71A885B9852A
:10E370008C91E0E1F4E001E00A93AAE4B4E00E94A9
:10E3800052F5AAE4B4E08C91A9E4B4E08C93A88996
:10E39000B9890D911C91A9E4B4E04D915527040F62
:10E3A000151FA889B9890D931C93A885B9858C91EF
:10E3B0008F5F8C93AEA5BFA5E889F9890E94ADF463
:10E3C000AEA5BFA50E94A7F5082F033010F00C944E
:10E3D000077286E30E94FAF0E8A9F9A9A881B98139
:10E3E0000E9447F5A8A9B9A9E4EAFDEE0E94DDF371
:10E3F0000E9497F1E881F981A8A9B9A90E940EF0BD
:10E400000E9447F586E3481A8827580A229681E039
:10E41000AC8DBD8D8C93AC8DBD8D0C91033018F0FF
:10E4200011F00C943372AC8DBD8D8C91EEA5FFA5CF
:10E4300001E00A93ADA5BEA50E9452F5ACA5BDA50D
:10E440000E94FEF4AC8DBD8DAD90BB24AAE6B4E075
:10E45000AA0DBB1D0C93AC8DBD8D8C918F5F8C93E1
:10E4600010F40C940B7283E08093850484E690E0B2
:10E470000E94EBF00E94F112AE8DBF8D4C91A885E9
:10E48000B9850C91041718F011F00C9449720C9492
:10E4900092710C946F72093050E0150711F00C94D2
:10E4A0006F72ECA1FDA1A5E1B7E00E9447F5EEE394
:10E4B000F0E0ACA1BDA17BE70E9478F583EC8093EE
:10E4C0006B048AE280936C048CE280936D0488E292
:10E4D00080936E0484E0809385040E94F1120C9472
:10E4E000A37CA8A5B9A5EEEBFEEE0E94DDF30E9489
:10E4F000ADF511F00C94C47286E0E0E2F1E002E0C8
:10E500000A93AFA5B8A90E9452F5AEA5BFA50E9477
:10E510000EF0E4ECFEEE0E94DDF30E9497F188E03D
:10E52000E0E2F1E002E00A93AFA5B8A90E940EF084
:10E530000E9452F5AEA5BFA50E940EF0E4ECFEEEDF
:10E540000E94DDF30E9497F1EEA5FFA5A1E1B1E0E5
:10E550000E9447F50E940FF1A1E1B1E00E940EF088
:10E56000E6ECFEEE0E94DDF30E9497F10E940FF1AF
:10E5700080E080938A0480916904846080936904B8
:10E580000E94159C0C94A37CA8A5B9A5EAECFEEE0C
:10E590000E94DDF30E94ADF511F00C941D7386E02E
:10E5A000E0E2F1E002E00A93AFA5B8A90E9452F5BB
:10E5B000AEA5BFA50E940EF0E0EDFEEE0E94DDF3D9
:10E5C0000E9497F188E0E0E2F1E002E00A93AFA553
:10E5D000B8A90E940EF00E9452F5AEA5BFA50E94F8
:10E5E0000EF0E0EDFEEE0E94DDF30E9497F18AE06E
:10E5F000E0E2F1E002E00A93AFA5B8A90E940EF0B4
:10E600000E9452F5EEA5FFA5A8E0B1E00E9447F5F3
:10E610000E9409F18091690482608093690480916D
:10E6200069048160809369040E94E79E8091690477
:10E630008E7F809369040C94A37CA8A5B9A5E2ED14
:10E64000FEEE0E94DDF30E94ADF511F00C945D73B7
:10E65000ACA1BDA10E94FEF4AC8DBD8D0C93AC8D20
:10E66000BD8D0C91013018F011F00C9439730C949D
:10E670003B730C949B7CEBE7FFE0AC8DBD8D7BE79F
:10E680000E9467F586E380936B0482E280936C04BA
:10E690008EE180936D048FE280936E040AEAAC8D64
:10E6A000BD8D4C91040FAFE6B4E00C9385E08093F0
:10E6B00085040E94F1120C94A37CA8A5B9A5E8EDED
:10E6C000FEEE0E94DDF30E94ADF511F00C949D73F7
:10E6D000ACA1BDA10E94FEF4AC8DBD8D0C93AC8DA0
:10E6E000BD8D0C91013018F011F00C9479730C94DD
:10E6F0007B730C949B7CE8EBF6E0AC8DBD8D7BE7E7
:10E700000E9467F588E580936B0484E180936C0434
:10E7100084E080936D0481E880936E040AEAAC8DF6
:10E72000BD8D4C91040FAFE6B4E00C9385E080936F
:10E7300085040E94F1120C94A37CA8A5B9A5EEED66
:10E74000FEEE0E94DDF30E94ADF511F00C94D9733A
:10E75000ACA1BDA10E94FEF4AC8DBD8D0C93AC8D1F
:10E76000BD8D0C91013018F011F00C94B9730C941C
:10E77000BB730C949B7CEFE0F0E0AC8DBD8D7BE730
:10E780000E9467F50E94F87E88E58093700481E816
:10E79000809371040AEAAC8DBD8D4C91040FA2E701
:10E7A000B4E00C9388E0809385040E94F1120C94ED
:10E7B000A37CA8A5B9A5E4EEFEEE0E94DDF30E94BD
:10E7C000ADF511F00C94717486E0E0E2F1E001E047
:10E7D0000A93AFA5B8A90E9452F5AEA5BFA5EAEE6F
:10E7E000FEEE0E94DDF30E94ADF511F00C943E7434
:10E7F000AEA5BFA50E94A7F5AE8DBF8D8C93AE8D43
:10E80000BF8D0C9141E0041BA885B9850C9382E073
:10E81000ECA1FDA1A885B9850C910A93AFA5B8A973
:10E820000E9452F5AEA5BFA50E94FEF4AA89BB893D
:10E830000D931C93AA89BB890D911C910B3350E059
:10E8400015071CF011F00C9427740C9429740C9487
:10E850009B7CAA89BB890D911C914FEF5FEF0E94B1
:10E860008DF1AA89BB890D931C93E9E7FFE0AA8982
:10E87000BB897BE70E9469F50C945C74ACA1BDA1D7
:10E880000E94FEF4AA89BB890D931C93AA89BB89B7
:10E890000D911C910B3350E015071CF011F00C94F6
:10E8A00053740C9455740C949B7CE9E7FFE0AA899F
:10E8B000BB897BE70E9469F50E94469E88E58093AC
:10E8C0006B0480E580936C048CE280936D0488E295
:10E8D00080936E0484E0809385040E94F1120C946E
:10E8E000A37CAC85BD850C91073011F00C94A57606
:10E8F000AA85BB850D911C91013050E0150711F0E0
:10E900000C948275ACA1BDA10E94FEF4AC8DBD8DAE
:10E910000C930E94D6CC00915204013010F00C945C
:10E92000A77481E08093500483E08093850482EA99
:10E9300080936B0482ED80936C0488E880936D046F
:10E940000E94F112809119058F77809319058091AB
:10E950002605806180932605E2E5F4E0FA93EA93C8
:10E960000E94A97C229688E880936B048BEE8093AA
:10E970006C048AEB80936D0483E08093850480911E
:10E9800026058F7E809326050E94F112A1E0B1E05A
:10E990008C9186FB16F00C941E755A924A9281E077
:10E9A000A42DB52D8C9381E00E9485EF5A924A9256
:10E9B00083E0A42DB52D8C9381E00E9485EF5A92BF
:10E9C0004A9284E0A42DB52D8C9381E00E9485EFBE
:10E9D0000E9421DE269683E00E9481EF81E08093F1
:10E9E0005004EC8DFD8DFA93EA930E9496C722960F
:10E9F0005A924A9280E0A42DB52D8C9381E00E941A
:10EA000085EF5A924A9283E0A42DB52D8C9381E034
:10EA10000E9485EF5A924A9284E0A42DB52D8C93E2
:10EA200081E00E9485EF0E9421DE269683E00E940D
:10EA300081EF81E0809344050C94807580911905E5
:10EA40008068809319055A924A9281E0A42DB52DD1
:10EA50008C9381E00E9485EF5A924A928091F00354
:10EA6000A42DB52D8C9381E00E9485EF5A924A9295
:10EA700084E0A42DB52D8C9381E00E9485EF0E9447
:10EA800021DE269683E00E9481EF81E0809350048E
:10EA9000EC8DFD8DFA93EA930E9496C722965A92C6
:10EAA0004A9280E0A42DB52D8C9381E00E9485EFE1
:10EAB0005A924A928091F003A42DB52D8C9381E057
:10EAC0000E9485EF5A924A9284E0A42DB52D8C9332
:10EAD00081E00E9485EF0E9421DE269683E00E945D
:10EAE00081EF81E0A1E5B4E0AD90BB24A1E4B5E005
:10EAF000AA0DBB1D8C93809119058F778093190502
:10EB00000C94A376023050E0150711F00C94C975EF
:10EB100080912605806180932605ACA1BDA10E944D
:10EB2000FEF4AC8DBD8D0C93EC8DFD8DFA93EA93C4
:10EB30000E947BC9229681E280936B0483E38093D9
:10EB40006C048FE280936D0487E580936E04AC8D36
:10EB5000BD8D8C9180936F0485E0809385040E9425
:10EB6000F1120E94D6CCE2E5F4E0FA93EA930E9417
:10EB7000A97C229688E880936B0481E080938504C9
:10EB8000809126058F7E809326050E94F1120C94B9
:10EB9000A376033050E0150711F00C940676ACA173
:10EBA000BDA10E94FEF4AC8DBD8D0C93AC8DBD8DCE
:10EBB0000C91033611F00C9404760E9463CC81E230
:10EBC00080936B0483E380936C048FE280936D04E5
:10EBD00087E580936E048CE380936F0485E08093D7
:10EBE00085040E94F1120E94D6CCE2E5F4E0FA938B
:10EBF000EA930E94A97C229688E880936B0481E0C6
:10EC0000809385040E94F1120C94A376043050E0A6
:10EC1000150711F00C944976ACA1BDA10E94FEF439
:10EC2000AC8DBD8D0C93EC8DFD8DA190BB24EAEED7
:10EC3000F7E0AA0CBB1CEA0DFB1DAA89BB890E9448
:10EC400085F5AA89BB890D911C9141E050E0041B18
:10EC5000150BAA89BB890D931C93EC8DFD8DA1909A
:10EC6000BB24EAEEF7E0AA0CBB1CEA0DFB1DAA8947
:10EC7000BB897BE70E9469F582E08093850488E97F
:10EC800080936B0481E080936C040E94F1120C94D9
:10EC9000A376053050E0150711F00C948C76ACA1EA
:10ECA000BDA10E94FEF4AC8DBD8D0C93EC8DFD8D4D
:10ECB000A190BB24EAEEF7E0AA0CBB1CEA0DFB1DF9
:10ECC000AA89BB890E9485F5AA89BB890D911C91EF
:10ECD00041E050E0040F151FAA89BB890D931C93D6
:10ECE000EC8DFD8DA190BB24EAEEF7E0AA0CBB1CD5
:10ECF000EA0DFB1DAA89BB897BE70E9469F582E0CA
:10ED00008093850483EB80936B0481E080936C0493
:10ED10000E94F1120C94A376063050E0150711F012
:10ED20000C94A3760E94D6CCE2E5F4E0FA93EA9341
:10ED30000E94A97C229688E880936B0481E08093EE
:10ED400085040E94F1120C94A37CAC85BD850C91C6
:10ED5000083011F00C94DC7BAA85BB850D911C91C9
:10ED6000003050E0150711F00C94EF76ACA1BDA176
:10ED70000E94FEF4AC8DBD8D0C93AC8DBD8D0C91BD
:10ED8000053010F00C94C87685E0AC8DBD8D8C9369
:10ED9000AC8DBD8D0C91023318F011F00C94D2762D
:10EDA0000C94D67682E3AC8DBD8D8C93E2EDF4E0CD
:10EDB000A190BB24E8E7F0E0EA0DFB1DAC8DBD8D12
:10EDC0007BE70E9467F50E942B7F80E380936D04B0
:10EDD00083E0809385040E94F1120C94DA7B013069
:10EDE00050E0150711F00C94617781E0ECA1FDA1D2
:10EDF00004E00A93AFA5B8A90E9452F5AEA5BFA53D
:10EE00000E94FEF4AA89BB890D931C93E2EDF4E005
:10EE1000A190BB24EBE6F0E0AA0CBB1CEA0DFB1DA5
:10EE2000AA89BB897BE70E9469F5E2EDF4E0A19035
:10EE3000BB24E1E7F0E0AA0CBB1CEA0DFB1D00E0DF
:10EE400010E0A0E1BB277BE70E9469F5ACA1BDA162
:10EE50000E94A7F5082F043018F011F00C943277B7
:10EE60000C94527785E0ECA1FDA104E00A93AFA5D4
:10EE7000B8A90E9452F5AEA5BFA50E94FEF4AA89CA
:10EE8000BB890D931C93E2EDF4E0A190BB24E1E774
:10EE9000F0E0AA0CBB1CEA0DFB1DAA89BB897BE72D
:10EEA0000E9469F50E942B7F87ED80936D0484E7B3
:10EEB00080936E0484E0809385040E94F1120C9488
:10EEC000DA7B023050E0150711F00C941378A88912
:10EED000B9890D911C9142E050E00E94C5EFAE85CA
:10EEE000BF854D935C9381E0A881B9818C93AE85F9
:10EEF000BF854D915C91A881B9810D9111270417AF
:10EF000015071CF011F00C94F477AE85BF850D91B8
:10EF10001C910F3050E015071CF011F00C94927703
:10EF20000C9494770C949B7CA881B9810C9142E05D
:10EF3000049FAA81BB810C92AA81BB818C918C5FBA
:10EF40008C93AA81BB818C91E0E2F1E002E00A930C
:10EF5000AFA5B8A90E9452F5AEA5BFA50E94FEF4C8
:10EF6000AC8DBD8D0C930091D204013011F00C9446
:10EF7000C877E881F981A190BB24E9E6F1E0EA0DC8
:10EF8000FB1DAC8DBD8D7BE70E9467F50C94EC7783
:10EF9000023011F00C94DB77E881F981A190BB2459
:10EFA000E8E7F1E0EA0DFB1DAC8DBD8D7BE70E942B
:10EFB00067F50C94EC77033011F00C94EC77E88152
:10EFC000F981A190BB24E7E8F1E0EA0DFB1DAC8DCF
:10EFD000BD8D7BE70E9467F5A881B9818C918F5F19
:10EFE0008C9310F40C947777E2EDF4E0A190BB24BD
:10EFF000EBE7F0E0EA0DFB1DAE85BF857BE70E94E5
:10F0000067F50E942B7F86E280936D0481E28093F6
:10F010006E0481E080936F0485E0809385040E94F4
:10F02000F1120C94DA7B033050E0150711F00C94C8
:10F03000C578A889B9890D911C9142E050E00E94E1
:10F04000C5EFAE85BF854D935C9381E0A881B98102
:10F050008C93AE85BF854D915C91A881B9810D914E
:10F060001127041715071CF011F00C94A678AE8533
:10F07000BF850D911C910F3050E015071CF011F069
:10F080000C9444780C9446780C949B7CA881B981AC
:10F090000C9142E0049FAA81BB810C92AA81BB81A2
:10F0A0008C918C5F8C93AA81BB818C91E0E2F1E022
:10F0B00002E00A93AFA5B8A90E9452F5AEA5BFA57C
:10F0C0000E94FEF4AC8DBD8D0C930091D2040130F2
:10F0D00011F00C947A78E881F981A190BB24E6E9DB
:10F0E000F1E0EA0DFB1DAC8DBD8D7BE70E9467F55D
:10F0F0000C949E78023011F00C948D78E881F9819F
:10F10000A190BB24E5EAF1E0EA0DFB1DAC8DBD8DBD
:10F110007BE70E9467F50C949E78033011F00C9405
:10F120009E78E881F981A190BB24E4EBF1E0EA0D3F
:10F13000FB1DAC8DBD8D7BE70E9467F5A881B98171
:10F140008C918F5F8C9310F40C942978E2EDF4E0AD
:10F15000A190BB24EEE7F0E0EA0DFB1DAE85BF8574
:10F160007BE70E9467F50E942B7F86E280936D0407
:10F1700081E280936E0482E080936F0485E0809347
:10F1800085040E94F1120C94DA7B043050E01507DC
:10F1900011F00C947579A889B9890D911C9143E0FF
:10F1A00050E00E94C5EFAE85BF854D935C93AE8560
:10F1B000BF850D911C91063150E015071CF011F030
:10F1C0000C94E4780C94E6780C949B7C81E0A88104
:10F1D000B9818C93AE85BF854D915C91A881B98131
:10F1E0000D911127041715071CF011F00C94587994
:10F1F000A881B9810C9143E0049FAA81BB810C9244
:10F20000AA81BB818C918D5F8C93AA81BB818C91EB
:10F21000E0E2F1E003E00A93AFA5B8A90E9452F53D
:10F22000AEA5BFA50E94FEF4AC8DBD8D0C930091E0
:10F23000D204013011F00C942C79E881F981A1906D
:10F24000BB24E3ECF1E0EA0DFB1DAC8DBD8D7BE74B
:10F250000E9467F50C945079023011F00C943F79BC
:10F26000E881F981A190BB24E9EDF1E0EA0DFB1DF5
:10F27000AC8DBD8D7BE70E9467F50C94507903300F
:10F2800011F00C945079E881F981A190BB24EFEE44
:10F29000F1E0EA0DFB1DAC8DBD8D7BE70E9467F5AB
:10F2A000A881B9818C918F5F8C9310F40C94EA78CB
:10F2B000E2EDF4E0A190BB24E1E8F0E0EA0DFB1DF3
:10F2C000AE85BF857BE70E9467F586E280936B047D
:10F2D00081E280936C0481E080936D0483E08093ED
:10F2E00085040E94F1120C94DA7B053050E015077A
:10F2F00011F00C94257AA889B9890D911C9143E0ED
:10F3000050E00E94C5EFAE85BF854D935C93AE85FE
:10F31000BF850D911C91063150E015071CF011F0CE
:10F320000C9494790C9496790C949B7C81E0A88140
:10F33000B9818C93AE85BF854D915C91A881B981CF
:10F340000D911127041715071CF011F00C94087A81
:10F35000A881B9810C9143E0049FAA81BB810C92E2
:10F36000AA81BB818C918D5F8C93AA81BB818C918A
:10F37000E0E2F1E003E00A93AFA5B8A90E9452F5DC
:10F38000AEA5BFA50E94FEF4AC8DBD8D0C9300917F
:10F39000D204013011F00C94DC79E881F981A1905C
:10F3A000BB24E5E0F2E0EA0DFB1DAC8DBD8D7BE7F3
:10F3B0000E9467F50C94007A023011F00C94EF79FA
:10F3C000E881F981A190BB24EBE1F2E0EA0DFB1D9D
:10F3D000AC8DBD8D7BE70E9467F50C94007A0330FD
:10F3E00011F00C94007AE881F981A190BB24E1E34B
:10F3F000F2E0EA0DFB1DAC8DBD8D7BE70E9467F549
:10F40000A881B9818C918F5F8C9310F40C949A79B8
:10F41000E2EDF4E0A190BB24E4E8F0E0EA0DFB1D8E
:10F42000AE85BF857BE70E9467F586E280936B041B
:10F4300081E280936C0482E080936D0483E080938A
:10F4400085040E94F1120C94DA7B063050E0150717
:10F4500011F00C94DE7AA889B9890D911C9143E0D2
:10F4600050E00E94C5EFAE85BF854D935C93AE859D
:10F47000BF850D911C91063150E015071CF011F06D
:10F480000C94447A0C94467A0C949B7C81E0A8817D
:10F49000B9818C93AE85BF854D915C91A881B9816E
:10F4A0000D911127041715071CF011F00C94B87A70
:10F4B000A881B9810C9143E0049FAA81BB810C9281
:10F4C000AA81BB818C918D5F8C93AA81BB818C9129
:10F4D000E0E2F1E003E00A93AFA5B8A90E9452F57B
:10F4E000AEA5BFA50E94FEF4AC8DBD8D0C9300911E
:10F4F000D204013011F00C948C7AE881F981A1904A
:10F50000BB24E7E4F2E0EA0DFB1DAC8DBD8D7BE78B
:10F510000E9467F50C94B07A023011F00C949F7A37
:10F52000E881F981A190BB24EDE5F2E0EA0DFB1D35
:10F53000AC8DBD8D7BE70E9467F50C94B07A0330EB
:10F5400011F00C94B07AE881F981A190BB24E3E733
:10F55000F2E0EA0DFB1DAC8DBD8D7BE70E9467F5E7
:10F56000A881B9818C918F5F8C9310F40C944A7AA6
:10F57000A889B9890C9143E00E9497F5AC8DBD8DA7
:10F580000C93E2EDF4E0A190BB24E7E8F0E0EA0D93
:10F59000FB1DAE85BF857BE70E9467F586E2809301
:10F5A0006B0481E280936C0483E080936D0483E0BC
:10F5B000809385040E94F1120C94DA7B073050E0AE
:10F5C000150711F00C948E7BECA1FDA101E0AC8D30
:10F5D000BD8D0E9459F5AC8DBD8D8C9180538C935F
:10F5E000AC8DBD8D0C91013081E008F080E08F93EF
:10F5F000AC8DBD8D0C91033080E010F009F081E0FE
:10F600009F91892B882311F40C94087B0C949B7C8C
:10F61000A889B9890C9141E0041BAAA1BBA10C9354
:10F6200082E0ECA1FDA1AAA1BBA10C910A93AFA518
:10F63000B8A90E9452F5AEA5BFA50E94FEF4A88D00
:10F64000B98D0C930091D20443E0049FAE89BF8929
:10F650000C92AE89BF890C91AC8DBD8D4C91040F7D
:10F66000AC89BD890C93AC89BD890C9143E0041B26
:10F67000AE89BF890C93AE89BF890C91093080E0B7
:10F6800010F009F081E08F93AE89BF890C910130B1
:10F6900081E008F080E09F91892B8F93A88DB98D30
:10F6A0000C910B3080E010F009F081E09F91892BE4
:10F6B000882311F40C945E7B0C949B7CEE89FF896B
:10F6C000A190BB24E2ECF9E0EA0DFB1DA88DB98DF9
:10F6D0007BE70E9467F586E280936B0481E280936A
:10F6E0006C04AC8DBD8D8C9180936D0485E380930B
:10F6F0006E04A88DB98D8C9180936F0482ED8093F8
:10F70000700484E98093710483EC8093720488E030
:10F71000809385040E94F1120C94DA7B083050E04B
:10F72000150711F00C94DA7BECA1FDA101E0AC8D82
:10F73000BD8D0E9459F5AC8DBD8D8C9180538C93FD
:10F74000AC8DBD8D0C91013018F011F00C94AA7B9A
:10F750000C94AC7B0C949B7CE2EDF4E0A190BB2478
:10F76000E7E6FFE0EA0DFB1DAC8DBD8D7BE70E9457
:10F7700067F5AC8DBD8D8C91A2EDB4E0AD90BB244E
:10F78000A3E4B6E0AA0DBB1D8C930E94F87E86E22E
:10F790008093700481E2809371040AEAAC8DBD8D80
:10F7A0004C91040FA2E7B4E00C9388E080938504A9
:10F7B0000E94F1120C94A37CAC85BD850C9109309C
:10F7C00011F00C949B7CAA85BB850D911C91003097
:10F7D00050E0150711F00C94197CACA1BDA10E945A
:10F7E000A7F5082F083018F011F00C94F97B0C9451
:10F7F000FB7B0C949B7CE2EDF4E00191112749E046
:10F8000050E00E948DF1E6E4F0E0E00FF11FACA1C2
:10F81000BDA17BE70E9478F589E580936B0483ECBA
:10F8200080936C0482E0809385040E94F1120C9412
:10F83000997C0A3050E0150711F00C944A7CACA179
:10F84000BDA10E94A7F5082F043018F011F00C9408
:10F850002B7C0C942D7C0C949B7CE2E7FFE0ACA10C
:10F86000BDA17BE70E9478F5ECA1FDA1A8E5B6E07B
:10F870000E9447F58CE880936B0489E580936C04C3
:10F8800083EC80936D0483E0809385040E94F112E1
:10F890000C94997C043150E0150711F00C94997C7C
:10F8A000ACA1BDA10E94A7F5082F013018F011F0FE
:10F8B0000C945C7C0C945E7C0C949B7CE7E7FFE0F2
:10F8C000ACA1BDA17BE70E9478F5ECA1FDA1ADE55F
:10F8D000B6E00E9447F50E94EB7E88EC80936F04AF
:10F8E00089E58093700483EC8093710487E08093B2
:10F8F00085040E94F112A8EDB6E0E6EAFEEE0E9451
:10F90000DDF30E9497F1EDE5F6E0A8EDB6E00E9488
:10F910000EF00E9447F5A8EDB6E00E940EF0E2EF6F
:10F92000FDEE0E94DDF30E9497F1A8EDB6E00E9483
:10F930008EF00C94A37C81E0809385048FE6809305
:10F940006B040E94F1128CEA481A8827580AE09644
:10F95000089581E00E94FAF08BEE80936B04AA81F7
:10F96000BB810C91043110F00C94BD7CAA81BB8149
:10F970008C9180936C040C94EE7CAA81BB810C91D9
:10F980004AE00E9497F5A881B9810C93AA81BB81B6
:10F990000C914AE00E9497F58C93AA81BB810C914F
:10F9A000003018F011F00C94D77C0C94E67C02E146
:10F9B000A881B9814C91040FABE6B4E00C93AA8105
:10F9C000BB818C9180936C040C94EE7C02E1A88145
:10F9D000B9814C91040FACE6B4E00C9380EC8093B9
:10F9E0006D0483E0809385040E94F11281E0481A3F
:10F9F0008827580A2296089581E00E94FAF081E053
:10FA00000E94FAF081E00E94FAF082E00E94FAF08F
:10FA100082E00E94FAF082E00E94FAF084E00E9404
:10FA2000FAF0AEE3B7E08C9185FB16F00C942C7DD8
:10FA300080913E078F7D80933E078AE280936B041E
:10FA40008EE180936C0480E280936D048FE280935A
:10FA50006E048CE280936F04A881B981E3E4F7E03F
:10FA60000E94B4F4E881F98101E0AE81BF810E9477
:10FA700059F582E0E881F98101E00A93AD81BE8108
:10FA80000E9452F5A881B9810E94A7F5EA2FFB2FA9
:10FA90003297F0400FEFAA81BB810E9459F5AE81E9
:10FAA000BF810E94FEF4AC85BD850C93AC81BD8105
:10FAB0000E94FEF4AA85BB850C93AA81BB810E949B
:10FAC000FEF4A885B9850C93A881B9810E94A7F599
:10FAD000082F033011F00C94817DAC85BD858C918D
:10FAE00080937004AA85BB858C9180937104A8854E
:10FAF000B9858C918093720488E0809385040C947E
:10FB0000B47D00914307053110F00C94907D8091F5
:10FB100043078093700486E0809385040C94B47D41
:10FB2000AA85BB850C91003011F00C94A47D02E1F4
:10FB3000AC85BD854C91040FA0E7B4E00C9386E042
:10FB4000809385040C94B47D02E1AC85BD854C9115
:10FB5000040FA0E7B4E00C93AA85BB858C91809339
:10FB6000710487E0809385048DE0481A8827580A3D
:10FB70002E96089581E00E94FAF081E0A881B98173
:10FB80008C93A881B9810C91033018F011F00C947A
:10FB9000027EA881B981AD90BB24A4EFB3E0AA0D89
:10FBA000BB1D0C91013011F00C94FA7D5A924A92CF
:10FBB00080E0A42DB52D8C9381E00E9485EF5A92B0
:10FBC0004A92AC81BD818C91A42DB52D8C9381E09E
:10FBD0000E9485EF5A924A928091F003A42DB52D90
:10FBE0008C9381E00E9485EF0E9421DE269683E0BF
:10FBF0000E9481EFA881B9818C918F5F8C9310F462
:10FC00000C94C17D8091EE0680688093EE0681E0C1
:10FC1000481A8827580A22960895EEEAF6E0A0E1ED
:10FC2000B0E00E9483F5013011F00C941B7E0E941D
:10FC30006FA10C94597E023011F00C94237E0E9427
:10FC4000D1AC0C94597E033011F00C942B7E0E94A1
:10FC5000A6AF0C94597E043011F00C94337E0E94B0
:10FC6000B0A20C94597E053011F00C943B7E0E949A
:10FC7000E6B30C94597EEEEAF6E0A0E1B0E00E9413
:10FC800083F5073081E008F480E08F93EEEAF6E038
:10FC9000A0E1B0E00E9483F5083081E010F009F0A7
:10FCA00080E09F918923882311F40C94597E0E944F
:10FCB000B0A284E690E00E94EBF00E9419F0AFE75A
:10FCC000B6E08D9388278C930E9415F0082F0030A2
:10FCD00011F00C945D7E8091EE068F778093EE0696
:10FCE00008955A924A9280E0A42DB52D8C9381E01C
:10FCF0000E9485EF5A924A9288E0A42DB52D8C93EC
:10FD000081E00E9485EF5A924A928091F003A42DDF
:10FD1000B52D8C9381E00E9485EF0E9421DE26960E
:10FD200083E00E9481EF5A924A9280E0A42DB52D83
:10FD30008C9381E00E9485EF5A924A928091F00361
:10FD4000A42DB52D8C9381E00E9485EF5A924A92A2
:10FD500084E0A42DB52D8C9381E00E9485EF0E9454
:10FD600021DE269683E00E9481EF88EC90E00E94DD
:10FD7000EBF0AEEEB6E08C9183FB16F00C94D17EE6
:10FD800086EA80936B0484EA80936C048CE280930F
:10FD90006D0488E280936E0484E0809385040C9463
:10FDA000D97E0E94167F89E680936D0483E080935C
:10FDB00085040E94F1128091EE068F7E8093EE06FC
:10FDC00080E0A0EFB3E0AD90BB24A3E0B4E0AA0DC7
:10FDD000BB1D8C93089581E280936B0481E3809333
:10FDE0006C048AE280936D0483E280936E0408952C
:10FDF00080E380936B048DE280936C0482E28093B5
:10FE00006D048EE180936E0488E280936F04089500
:10FE10008CE980936B0485EB80936C04089586E7EE
:10FE200080936E0485EB80936F04089585E480933E
:10FE30006B048FEA80936C0408958BE880936B04C5
:10FE400085EB80936C0408958CEB80936B048BE4BA
:10FE500080936C04089580E280936B0484E3809324
:10FE60006C0408958AE280936F048EE1809370049D
:10FE700080E2809371048FE2809372048CE280931D
:10FE80007304089582E00E94FAF082E00E94FAF082
:10FE900082E00E94FAF082E00E94FAF081E00E9483
:10FEA000FAF081E00E94FAF081E00E94FAF081E02D
:10FEB0008093D90485E08093DA048BE08093DB049F
:10FEC00082E18093DC048CE18093DD0487E28093FF
:10FED000DE0483E38093DF048FE38093E0048BE40C
:10FEE0008093E10487E58093E20482E68093E30453
:10FEF0008CE68093E40483E78093E50489E78093AC
:10FF0000E6048DE78093E7048EE78093E8048DE7AD
:10FF10008093E90489E78093EA0483E78093EB0404
:10FF20008CE68093EC0482E68093ED0487E5809371
:10FF3000EE048BE48093EF048FE38093F00483E37B
:10FF40008093F10487E28093F2048CE18093F304C0
:10FF500082E18093F4048BE08093F50485E0809344
:10FF6000F60481E08093F70481E08093F80480E058
:10FF700087BD84EF86BD80EC8FBD81E18EBDA7E398
:10FF8000B0E08C9180648C93AA85BB850E94BFF3FE
:10FF9000A885B9850E94BFF381E090E0AE81BF8162
:10FFA0008D939C93A7EDB4E04D915C91AE81BF81A0
:10FFB0000D911C91041715071CF011F00C9478801A
:10FFC00081E0AC81BD818C93AC81BD810C910F31FE
:10FFD00018F011F00C947280AA85BB850D911C91CC
:10FFE000A3EDB4E04D915C91040F151FAA85BB856C
:10FFF0000D931C93AA85BB850D911C914FEF5FE774
:020000021000EC
:1000000004231523AA85BB850D931C93A885B98568
:100010000D911C91A5EDB4E04D915C91040F151F5D
:10002000A885B9850D931C93A885B9850D911C9160
:100030004FEF5FE704231523A885B9850D931C9323
:10004000AA85BB8511968C91AA81BB818C9392E085
:10005000AA81BB810E94AEF1AA81BB818C918F5F86
:100060008C93A885B98511968C91A881B9818C93C0
:1000700092E0A881B9810E94AEF1A881B9818C91EA
:100080008F5F8C93AA81BB81AD90BB24A8EDB4E0B7
:10009000AA0DBB1D0D911127A881B981AD90BB247C
:1000A000A8EDB4E0AA0DBB1D4D915527040F151FF7
:1000B000AC85BD850D931C9386B782FFFDCFAC85C3
:1000C000BD858D919C9190934B0080934A0086B79B
:1000D000846086BFAC81BD818C918F5F8C9310F45E
:1000E0000C94E47FAE81BF810E948DEF0C94D27F8F
:1000F000A7E3B0E08C918F7B8C938BE0481A882724
:10010000580A2E960895A9EFB4E08D919C91A3ED25
:10011000B4E08D939C93ABEFB4E08D919C91A5EDF1
:10012000B4E08D939C93ACE4B7E08D919C91A7EDE6
:10013000B4E08D939C930E94427FACE4B7E08D9134
:100140009C910E94EBF00895A9EFB4E08D919C91F1
:10015000A3EDB4E08D939C93ABEFB4E08D919C91B3
:10016000A5EDB4E08D939C93AEE4B7E08D919C91A6
:10017000A7EDB4E08D939C930E94427FACE4B7E07E
:100180008D919C910E94EBF00895AEE4B7E00D9143
:100190001C914EE150E0041B150BA7EDB4E00D934C
:1001A0001C93A7EDB4E08D919C910E94EBF0089513
:1001B00082E00E94FAF081E00E94FAF081E00E9461
:1001C000FAF081E00E94FAF081E00E94FAF081E00A
:1001D0000E94FAF081E00E94FAF081E00E94FAF0B9
:1001E00081E00E94FAF081E00E94FAF081E00E9432
:1001F000FAF081E00E94FAF081E00E94FAF081E0DA
:100200000E94FAF081E0AA81BB818C93AA81BB8114
:100210000C91033018F011F00C944D82AA81BB812F
:10022000AD90BB24A2E0B5E0AA0DBB1D0C9101303E
:1002300011F00C942C81AA81BB81AD90BB24ABE45E
:10024000B4E0AA0DBB1D0C91003011F00C942C8170
:1002500081E0A881B9818C935A924A9280E0A42DC2
:10026000B52D8C9381E00E9485EF5A924A9285E0E9
:10027000A42DB52D8C9381E00E9485EF5A924A926D
:10028000A885B9858C91A42DB52D8C9381E00E9411
:1002900085EF0E9421DE269683E00E9481EFAA81ED
:1002A000BB81AD90BB24ABE7B6E0AA0DBB1D0C91A2
:1002B000003011F00C946E81AA81BB81AD90BB24FB
:1002C000ACE0B4E0AA0DBB1D8C91AA81BB81AD90BE
:1002D000BB24A9E0B4E0AA0DBB1D8C935A924A92AC
:1002E000AC81BD818C91A42DB52D8C9381E00E94B1
:1002F00085EF5A924A92AE81BF81AD90BB24ABE7A5
:10030000B6E0AA0DBB1D8C91A42DB52D8C9381E078
:100310000E9485EF0E94BB2A249682E00E9481EF12
:1003200080916904806280936904AA81BB81AD9049
:10033000BB24A2E0B5E0AA0DBB1D0C91013011F069
:100340000C94458281E0AA81BB81AD90BB24AEECC8
:10035000B4E0AA0DBB1D8C93EA81FB81A190BB2464
:10036000E8E7F0E0EA0DFB1DA88DB98D0E9483F54A
:10037000EA81FB81A190BB24EBE6F0E0AA0CBB1C58
:10038000EA0DFB1DA9EFB4E00E9485F5EA81FB812F
:10039000A190BB24E1E7F0E0AA0CBB1CEA0DFB1D19
:1003A000ABEFB4E00E9485F5A9EFB4E00D911C918C
:1003B000003050E0150711F00C94EC81ABEFB4E085
:1003C0000D911C91003050E0150711F00C94EC8158
:1003D0000E94E1830C94DB83AA81BB81AD90BB2496
:1003E000ACEFB4E0AA0DBB1D0C91013011F00C94E0
:1003F0000782EA81FB81A190BB24EBE7F0E0EA0DE4
:10040000FB1DAC89BD890E9483F50C942082AA81D2
:10041000BB81AD90BB24ACEFB4E0AA0DBB1D0C9129
:10042000023011F00C942082EA81FB81A190BB2460
:10043000EEE7F0E0EA0DFB1DAC89BD890E9483F573
:100440005A924A9281E0A42DB52D8C9381E00E94AE
:1004500085EF5A924A9285E0A42DB52D8C9381E0C8
:100460000E9485EF5A924A92A885B9858C91A42D55
:10047000B52D8C9381E00E9485EF0E9421DE2696A7
:1004800083E00E9481EF0C944D82AA81BB818C9104
:100490008F5F8C9310F40C9406810091030501305A
:1004A00011F00C94568281E08093FE0300910405C4
:1004B000013011F00C945F8282E08093FF03009181
:1004C0000505013011F00C94688284E080930004EB
:1004D0000E94B010A881B9810C91013011F00C94E8
:1004E0009D8280E0A881B9818C93A5E7B6E00D914B
:1004F0001C914AE050E00E94C5EFAA8DBB8D4D9340
:100500005C9381E0AC81BD818C93AC81BD810C9109
:100510000A3018F011F00C949D82AA8DBB8D8D913C
:100520009C910E94EBF00E947D18AC81BD818C9162
:100530008F5F8C9310F40C948582AA81BB814C91BF
:1005400000911B06041711F00C94A98280E080939F
:100550001B0600EB14E0A88DB98D4D9155270E9424
:10056000C5EFACE4B7E04D935C93ACE4B7E00D911C
:100570001C9143E050E00E948DF1AEE4B7E00D9392
:100580001C9381E0AE89BF898C93AC89BD894C9165
:10059000AE89BF890C91041718F011F00C94D9831F
:1005A00000910305013011F00C94FA820091FD04D2
:1005B000013011F00C94E882EE89FF89A190BB24F0
:1005C000E9E6F1E0EA0DFB1DAA89BB890E9483F5EB
:1005D0000091FD04023011F00C94FA82EE89FF893B
:1005E000A190BB24E6E9F1E0EA0DFB1DAA89BB89D5
:1005F0000E9483F500910405013011F00C942483CE
:100600000091FE04013011F00C941283EE89FF89F1
:10061000A190BB24E8E7F1E0EA0DFB1DAA89BB89A4
:100620000E9483F50091FE04023011F00C942483A3
:10063000EE89FF89A190BB24E5EAF1E0EA0DFB1DFC
:10064000AA89BB890E9483F500910505013011F04C
:100650000C944E830091FF04013011F00C943C8304
:10066000EE89FF89A190BB24E7E8F1E0EA0DFB1DCC
:10067000AA89BB890E9483F50091FF04023011F022
:100680000C944E83EE89FF89A190BB24E7E8F1E04A
:10069000EA0DFB1DAA89BB890E9483F5E8E1FAE017
:1006A0000E94DDF3AA89BB898C919927AA85BB8515
:1006B0000E94BCF380E8A889B9898C9380E0AE855C
:1006C000BF858C93AA85BB850C91003011F00C94EA
:1006D00071830E94C5800E94AC840E94C5800C94E6
:1006E000D18381E0AE81BF818C93AE81BF810C91BB
:1006F000083018F011F00C94CD830E94AC84AA85C8
:10070000BB850C91A889B9894C910423AC81BD812A
:100710000C93AC81BD810C91003018F011F00C9459
:1007200093830C94998381E0AC85BD858C930C9464
:100730009D8380E0AC85BD858C93AE85BF850C9193
:10074000013011F00C94B383AC85BD850C91013060
:1007500011F00C94AF830E94A4800C94B1830E948A
:1007600083800C94BE83AC85BD850C91013011F063
:100770000C94BE8381E0AE85BF858C93A889B9892E
:100780000C9142E00E9497F50C93AE81BF818C9151
:100790008F5F8C9310F40C9475830E94AC840E943C
:1007A000C580AE89BF898C918F5F8C9310F40C94B7
:1007B000C5820E94E1838FE0481A8827580A6C9608
:1007C000089581E00E94FAF081E0A881B9818C93BC
:1007D000A881B9810C91033018F011F00C949F841A
:1007E000A881B981AD90BB24A8E3B4E0AA0DBB1DDC
:1007F0000C91003011F00C942C8480E0A881B98118
:10080000AD90BB24ADEFB3E0AA0DBB1D8C93A881C6
:10081000B981AD90BB24ACEFB4E0AA0DBB1D8C91A7
:100820008F5F8C93A881B981AD90BB24ACEFB4E00D
:10083000AA0DBB1D0C91023018F011F00C9422840B
:100840000C942C8481E0A881B981AD90BB24ACEFDD
:10085000B4E0AA0DBB1D8C93A881B981AD90BB24D7
:10086000A2E0B5E0AA0DBB1D0C91013011F00C9473
:1008700066845A924A9280E0A42DB52D8C9381E033
:100880000E9485EF5A924A9285E0A42DB52D8C9353
:1008900081E00E9485EF5A924A92AE81BF818C918D
:1008A000A42DB52D8C9381E00E9485EF0E9421DE5E
:1008B000269683E00E9481EF80E0A881B981AD9007
:1008C000BB24A2E0B5E0AA0DBB1D8C9380E0A881FB
:1008D000B981AD90BB24AEECB4E0AA0DBB1D8C93E6
:1008E000A881B981AD90BB24ABE7B6E0AA0DBB1DD2
:1008F0000C91013011F00C9497845A924A92AA817B
:10090000BB818C91A42DB52D8C9381E00E9485EF45
:100910005A924A9280E0A42DB52D8C9381E00E94DA
:1009200085EF0E94BB2A249682E00E9481EFA88175
:10093000B9818C918F5F8C9310F40C94E8830E94A2
:10094000B010809169048F7D8093690481E0481A1A
:100950008827580A229608950E947D18A1E0B1E0E8
:100960008C9185FB81E00EF080E08F930091F30382
:10097000013081E009F080E09F91892B882311F4F8
:100980000C94C4840E945C2DA1E0B1E08C9184FBA6
:1009900081E00EF080E08F930091F403013081E05C
:1009A00009F080E09F91892B882311F40C94DA845C
:1009B0000E94122EA1E0B1E08C9183FB81E00EF049
:1009C00080E08F930091F203013081E009F080E034
:1009D0009F91892B882311F40C94F0840E94A62CFB
:1009E000A1E0B1E08C9182FB16F00C94F9840E9496
:1009F000122EA1E0B1E08C9181FB16F00C940285DF
:100A00000E94A62CA1E0B1E08C9180FB16F00C9422
:100A10000B850E945C2D08953F2F2723212030381D
:100A20003C3E3900322A7314141414144C05181A5D
:100A3000141414141414140C021214141414141492
:100A4000140E100414141414141414170D14141484
:100A5000141414144507060F141414141414161D3A
:100A60000A0814141414141414030911141414147B
:100A700014141C0B191B81E00E94FAF081E00E9403
:100A8000FAF08AE00E94FAF08AE00E94FAF0ACE004
:100A9000B5E00D911C91003050E0150781E009F0A0
:100AA00080E08F93ACE0B5E00D911C91043F51E0E4
:100AB000150780E014F009F081E09F91892B8823CD
:100AC00011F40C9465850C940F9C8091EE06806463
:100AD0008093EE06ACE0B5E00D911C91003050E043
:100AE00015071CF011F00C9477850C949185ACE0FF
:100AF000B5E00D911C91043050E015070CF402C0D4
:100B00000C949185ECE0F5E0A190B080EAE8F0E08B
:100B1000EA0DFB1DA0E1BB2781E08C937BE70E94DF
:100B200067F5ACE0B5E00D911C91033050E015077E
:100B30001CF011F00C949E850C94BF85ACE0B5E0E0
:100B40000D911C91073050E015070CF402C00C9475
:100B5000BF8500910C0543E0041BAE81BF810C935F
:100B6000EE81FF81A190BB24EAE8F0E0EA0DFB1DD5
:100B7000A0E1BB2780E08C937BE70E9467F5ACE0A7
:100B8000B5E00D911C91063050E015071CF011F0F6
:100B90000C94CC850C94ED85ACE0B5E00D911C91E6
:100BA0000A3050E015070CF402C00C94ED8500915A
:100BB0000C0546E0041BAE81BF810C93EE81FF81E2
:100BC000A190BB24EBE1F0E0EA0DFB1DA0E1BB2707
:100BD00081E08C937BE70E9467F5ACE0B5E00D9176
:100BE0001C910B3050E015071CF011F00C94FA85A5
:100BF0000C941B86ACE0B5E00D911C910D3050E0DB
:100C000015070CF402C00C941B8600910C054BE0F8
:100C1000041BAE81BF810C93EE81FF81A190BB24A8
:100C2000EBE1F0E0EA0DFB1DA0E1BB2780E08C9337
:100C30007BE70E9467F5ACE0B5E00D911C910C30AC
:100C400050E015071CF011F00C9428860C9449868E
:100C5000ACE0B5E00D911C91003150E015070CF4AB
:100C600002C00C94498600910C054CE0041BAE8137
:100C7000BF810C93EE81FF81A190BB24E8E1F0E0FD
:100C8000EA0DFB1DA0E1BB2781E08C937BE70E946E
:100C900067F5ACE0B5E00D911C910F3050E0150701
:100CA0001CF011F00C9456860C947786ACE0B5E0FD
:100CB0000D911C91033150E015070CF402C00C9407
:100CC000778600910C054FE0041BAE81BF810C9329
:100CD000EE81FF81A190BB24E8E1F0E0EA0DFB1D6D
:100CE000A0E1BB2780E08C937BE70E9467F5ACE036
:100CF000B5E00D911C91033150E0150711F00C94F3
:100D0000B08681E08093B904809101018062809374
:100D100001010091F503013011F00C94B0865A9254
:100D20004A9281E0A42DB52D8C9381E00E9485EF3D
:100D30005A924A9281E0A42DB52D8C9381E00E94B5
:100D400085EF5A924A9282E0A42DB52D8C9381E0D2
:100D50000E9485EF0E9421DE269683E00E9481EFAB
:100D6000ACE0B5E00D911C91043150E0150711F095
:100D70000C94E98681E08093B9048091010180613F
:100D8000809301010091F503013011F00C94E98684
:100D90005A924A9281E0A42DB52D8C9381E00E9455
:100DA00085EF5A924A9281E0A42DB52D8C9381E073
:100DB0000E9485EF5A924A9283E0A42DB52D8C9320
:100DC00081E00E9485EF0E9421DE269683E00E944A
:100DD00081EFACE0B5E00D911C91053150E01507B5
:100DE00011F00C942787809101018F7D8093010180
:100DF0005A924A9280E0A42DB52D8C9381E00E94F6
:100E000085EF5A924A9281E0A42DB52D8C9381E012
:100E10000E9485EF5A924A9282E0A42DB52D8C93C0
:100E200081E00E9485EF0E9421DE269683E00E94E9
:100E300081EF80E08093400400911006003011F0B3
:100E40000C94278780E08093FF030E94B010ACE0F1
:100E5000B5E00D911C91063150E0150711F00C948E
:100E60006587809101018F7E809301015A924A9299
:100E700080E0A42DB52D8C9381E00E9485EF5A92DD
:100E80004A9281E0A42DB52D8C9381E00E9485EFDC
:100E90005A924A9283E0A42DB52D8C9381E00E9452
:100EA00085EF0E9421DE269683E00E9481EF80E09C
:100EB0008093400400911106003011F00C94658776
:100EC00080E0809300040E94B010ACE0B5E00D918A
:100ED0001C91073150E0150711F00C949E8781E0BA
:100EE0008093BA0480910101886080930101009190
:100EF000F603013011F00C949E875A924A9281E0D9
:100F0000A42DB52D8C9381E00E9485EF5A924A92D0
:100F100082E0A42DB52D8C9381E00E9485EF5A923A
:100F20004A9281E0A42DB52D8C9381E00E9485EF3B
:100F30000E9421DE269683E00E9481EFACE0B5E0BE
:100F40000D911C91083150E0150711F00C94D787D2
:100F500081E08093BA048091010184608093010153
:100F60000091F603013011F00C94D7875A924A92FF
:100F700081E0A42DB52D8C9381E00E9485EF5A92DB
:100F80004A9282E0A42DB52D8C9381E00E9485EFDA
:100F90005A924A9283E0A42DB52D8C9381E00E9451
:100FA00085EF0E9421DE269683E00E9481EFACE06F
:100FB000B5E00D911C91093150E0150711F00C942A
:100FC0001B8880910101877F809301015A924A9288
:100FD00080E0A42DB52D8C9381E00E9485EF5A927C
:100FE0004A9282E0A42DB52D8C9381E00E9485EF7A
:100FF0005A924A9281E0A42DB52D8C9381E00E94F3
:1010000085EF0E9421DE269683E00E9481EF80E03A
:101010008093410480E08093F80380E08093F9039B
:1010200000910F06003011F00C941B8880E0809333
:10103000FE030E94B010ACE0B5E00D911C910A31A6
:1010400050E0150711F00C945F88809101018B7FAF
:10105000809301015A924A9280E0A42DB52D8C9381
:1010600081E00E9485EF5A924A9282E0A42DB52D2C
:101070008C9381E00E9485EF5A924A9283E0A42DDE
:10108000B52D8C9381E00E9485EF0E9421DE26968B
:1010900083E00E9481EF80E08093410480E08093B0
:1010A000F90380E08093FA0300911106003011F0FB
:1010B0000C945F8880E0809300040E94B010ACE044
:1010C000B5E00D911C910B3150E0150711F00C9417
:1010D000988881E08093BB048091010182608093B5
:1010E00001010091F703013011F00C9498885A9295
:1010F0004A9281E0A42DB52D8C9381E00E9485EF6A
:101100005A924A9283E0A42DB52D8C9381E00E94DF
:1011100085EF5A924A9281E0A42DB52D8C9381E0FF
:101120000E9485EF0E9421DE269683E00E9481EFD7
:10113000ACE0B5E00D911C910C3150E0150711F0B9
:101140000C94D18881E08093BB048091010181607F
:10115000809301010091F703013011F00C94D188C4
:101160005A924A9281E0A42DB52D8C9381E00E9481
:1011700085EF5A924A9283E0A42DB52D8C9381E09D
:101180000E9485EF5A924A9282E0A42DB52D8C934D
:1011900081E00E9485EF0E9421DE269683E00E9476
:1011A00081EFACE0B5E00D911C910D3150E01507D9
:1011B00011F00C941289809101018D7F80930101BF
:1011C0005A924A9280E0A42DB52D8C9381E00E9422
:1011D00085EF5A924A9283E0A42DB52D8C9381E03D
:1011E0000E9485EF5A924A9281E0A42DB52D8C93EE
:1011F00081E00E9485EF0E9421DE269683E00E9416
:1012000081EF80E08093420480E08093FB030091B3
:101210000F06003011F00C94128980E08093FE03D9
:101220000E94B010ACE0B5E00D911C910E3150E081
:10123000150711F00C945389809101018E7F8093E2
:1012400001015A924A9280E0A42DB52D8C9381E041
:101250000E9485EF5A924A9283E0A42DB52D8C937B
:1012600081E00E9485EF5A924A9282E0A42DB52D2A
:101270008C9381E00E9485EF0E9421DE269683E018
:101280000E9481EF80E08093420480E08093FC0321
:1012900000911006003011F00C94538980E0809387
:1012A000FF030E94B010ACE0B5E00D911C910E312F
:1012B00050E015071CF011F00C9460890C948189A2
:1012C000ACE0B5E00D911C91023250E015070CF432
:1012D00002C00C94818900910C054EE1041BAE8183
:1012E000BF810C93EE81FF81A190BB24EDE8F0E07B
:1012F000EA0DFB1DA0E1BB2780E08C937BE70E94F9
:1013000067F5ACE0B5E00D911C91013250E0150796
:101310001CF011F00C948E890C94AF89ACE0B5E010
:101320000D911C91053250E015070CF402C00C948D
:10133000AF8900910C0541E2041BAE81BF810C9383
:10134000EE81FF81A190BB24EDE8F0E0EA0DFB1DEA
:10135000A0E1BB2781E08C937BE70E9467F5ACE0BE
:10136000B5E00D911C91043250E015071CF011F00E
:101370000C94BC890C94D889ACE0B5E00D911C911B
:10138000083250E015070CF402C00C94D889009183
:101390000C0544E2041BAE81BF810C9381E0AE8159
:1013A000BF81AD90BB24AEE0B6E0AA0DBB1D8C930F
:1013B000ACE0B5E00D911C91073250E015071CF030
:1013C00011F00C94E5890C94018AACE0B5E00D9124
:1013D0001C910B3250E015070CF402C00C94018AEA
:1013E00000910C0547E2041BAE81BF810C9380E0A5
:1013F000AE81BF81AD90BB24AEE0B6E0AA0DBB1DAF
:101400008C93ACE0B5E00D911C910A3250E01507C9
:101410001CF011F00C940E8A0C942A8AACE0B5E012
:101420000D911C910E3250E015070CF402C00C9483
:101430002A8A00910C054AE2041BAE81BF810C93FD
:1014400081E0AE81BF81AD90BB24ABE1B6E0AA0DD7
:10145000BB1D8C93ACE0B5E00D911C910D3250E0BA
:1014600015071CF011F00C94378A0C94538AACE0E9
:10147000B5E00D911C91013350E015070CF402C04A
:101480000C94538A00910C054DE2041BAE81BF8180
:101490000C9380E0AE81BF81AD90BB24ABE1B6E0A0
:1014A000AA0DBB1D8C93ACE0B5E00D911C910033EF
:1014B00050E015071CF011F00C94608A0C94728AAD
:1014C000ACE0B5E00D911C910B3350E015070CF426
:1014D00002C00C94728A00910C0540E3041BA9E041
:1014E000B5E00C93ACE0B5E00D911C910A3350E0EF
:1014F00015071CF011F00C947F8A0C94918AACE0D3
:10150000B5E00D911C91053450E015070CF402C0B4
:101510000C94918A00910C054AE3041BAAE0B5E003
:101520000C93ACE0B5E00D911C91043450E015072C
:101530001CF011F00C949E8A0C94B08AACE0B5E0DB
:101540000D911C910F3450E015070CF402C00C945F
:10155000B08A00910C0544E4041BABE0B5E00C93A9
:10156000ACE0B5E00D911C910E3450E015071CF075
:1015700011F00C94BD8A0C94DE8AACE0B5E00D91BC
:101580001C91023550E015070CF402C00C94DE8A61
:1015900000910C054EE4041BAE81BF810C93EE81DB
:1015A000FF81A190BB24EBEAF0E0EA0DFB1DA0E176
:1015B000BB2781E08C937BE70E9467F5ACE0B5E048
:1015C0000D911C91013550E015071CF011F00C94A1
:1015D000EB8A0C940C8BACE0B5E00D911C910535B9
:1015E00050E015070CF402C00C940C8B00910C0514
:1015F00041E5041BAE81BF810C93EE81FF81A19078
:10160000BB24EBEAF0E0EA0DFB1DA0E1BB2780E084
:101610008C937BE70E9467F5ACE0B5E00D911C91DF
:10162000053550E0150711F00C94D28B80916904B8
:101630008F7D8093690400913804013081E009F0C6
:1016400080E08F93009138040C3081E009F080E055
:101650009F91892B8F93009138040D3081E009F020
:1016600080E09F91892B8F93009138040B3781E0A4
:1016700009F080E09F91892B882311F40C94588BFA
:101680005A924A9281E0A42DB52D8C9381E00E945C
:1016900085EF5A924A9281E0A42DB52D8C9381E07A
:1016A0000E9485EF0E94BB2A249682E00E9481EF6F
:1016B00000913804023081E009F080E08F930091BE
:1016C00038040C3081E009F080E09F91892B8F93E2
:1016D00000913804073181E009F080E09F91892B67
:1016E0008F93009138040B3781E009F080E09F91DF
:1016F000892B882311F40C94958B5A924A9282E09C
:10170000A42DB52D8C9381E00E9485EF5A924A92C8
:1017100081E0A42DB52D8C9381E00E9485EF0E947D
:10172000BB2A249682E00E9481EF009138040330A6
:1017300081E009F080E08F93009138040D3081E062
:1017400009F080E09F91892B8F9300913804073135
:1017500081E009F080E09F91892B8F9300913804FC
:101760000B3781E009F080E09F91892B882311F4E9
:101770000C94D28B5A924A9283E0A42DB52D8C936F
:1017800081E00E9485EF5A924A9281E0A42DB52D06
:101790008C9381E00E9485EF0E94BB2A249682E010
:1017A0000E9481EFACE0B5E00D911C91063550E050
:1017B000150711F00C94FA8B8091EE068F7B8093C5
:1017C000EE065A924A9280913804A42DB52D8C933E
:1017D00081E00E9485EF5A924A9280E0A42DB52DB7
:1017E0008C9381E00E9485EF0E94BB2A249682E0C0
:1017F0000E9481EFACE0B5E00D911C91063550E000
:1018000015071CF011F00C94078C0C94268CACE09E
:10181000B5E00D911C910F3550E015070CF402C096
:101820000C94268C00910C0546E5041BAE81BF810B
:101830000C93AA81BB81EE81FF810E94B4F4EA81FE
:10184000FB81FA93EA930E944ED22296ACE0B5E077
:101850000D911C910E3550E015071CF011F00C9401
:10186000338C0C94668CACE0B5E00D911C9106367F
:1018700050E015070CF402C00C94668C00910C0526
:101880004EE5041BAE81BF810C9381E0AE81BF8128
:10189000AD90BB24A9E2B5E0AA0DBB1D8C93AE812F
:1018A000BF810C9141E0041BAC81BD810C93AC81E4
:1018B000BD819C91AE81BF81AD90BB24A9E2B5E012
:1018C000AA0DBB1D0E94A6F10E94B010ACE0B5E0CD
:1018D0000D911C91053650E015071CF011F00C9489
:1018E000738C0C94918CACE0B5E00D911C910D368D
:1018F00050E015070CF402C00C94918C00910C057B
:1019000045E6041BAE81BF810C9380E0AE81BF81B0
:10191000AD90BB24A9E2B5E0AA0DBB1D8C930E943B
:10192000B010ACE0B5E00D911C910C3650E01507FD
:101930001CF011F00C949E8C0C94F18CACE0B5E092
:101940000D911C91043750E015070CF402C00C9463
:10195000F18C00910C054CE6041BAE81BF810C9309
:1019600080E0AE81BF81AD90BB24A9E2B5E0AA0DB5
:10197000BB1D8C930E94B01081E0AE81BF81AD9001
:10198000BB24A9E2B5E0AA0DBB1D8C93AE81BF813B
:101990000C9141E0041BAC81BD810C93AC81BD81F5
:1019A0009C91AE81BF81AD90BB24A9E2B5E0AA0DA8
:1019B000BB1D0E94A6F184E690E00E94EBF00E941D
:1019C000B01080E0AE81BF81AD90BB24A9E2B5E04C
:1019D000AA0DBB1D8C9384E690E00E94EBF00E9460
:1019E000B010ACE0B5E00D911C91043750E0150744
:1019F00011F00C94FD8C0E94159CACE0B5E00D91AB
:101A00001C91053750E0150711F00C94098D0E94C8
:101A1000E79EACE0B5E00D911C91063750E015074C
:101A200011F00C94718D81E08093B90481E0809372
:101A3000BA048091010180628093010180910101CB
:101A40008860809301010091F503013011F00C943E
:101A50004A8D5A924A9281E0A42DB52D8C9381E053
:101A60000E9485EF5A924A9281E0A42DB52D8C9365
:101A700081E00E9485EF5A924A9282E0A42DB52D12
:101A80008C9381E00E9485EF0E9421DE269683E000
:101A90000E9481EF0091F603013011F00C94718DDA
:101AA0005A924A9281E0A42DB52D8C9381E00E9438
:101AB00085EF5A924A9282E0A42DB52D8C9381E055
:101AC0000E9485EF5A924A9281E0A42DB52D8C9305
:101AD00081E00E9485EF0E9421DE269683E00E942D
:101AE00081EFACE0B5E00D911C91073750E0150790
:101AF00011F00C94D98D81E08093B90481E080933A
:101B0000BB048091010180618093010180910101FA
:101B10008260809301010091F503013011F00C9473
:101B2000B28D5A924A9281E0A42DB52D8C9381E01A
:101B30000E9485EF5A924A9281E0A42DB52D8C9394
:101B400081E00E9485EF5A924A9283E0A42DB52D40
:101B50008C9381E00E9485EF0E9421DE269683E02F
:101B60000E9481EF0091F703013011F00C94D98DA0
:101B70005A924A9281E0A42DB52D8C9381E00E9467
:101B800085EF5A924A9283E0A42DB52D8C9381E083
:101B90000E9485EF5A924A9281E0A42DB52D8C9334
:101BA00081E00E9485EF0E9421DE269683E00E945C
:101BB00081EFACE0B5E00D911C91083750E01507BE
:101BC00011F00C94418E81E08093BA0481E08093FF
:101BD000BB04809101018460809301018091010127
:101BE0008160809301010091F603013011F00C94A3
:101BF0001A8E5A924A9281E0A42DB52D8C9381E0E1
:101C00000E9485EF5A924A9282E0A42DB52D8C93C2
